:020000040800F2
:1000000000060020B5050008B129000831290008C4
:1000100089290008312900085D290008B705000872
:10002000B7050008B7050008B70500084D3B0008F4
:10003000B7050008B7050008B7050008B7050008B0
:10004000B7050008B7050008B7050008B7050008A0
:10005000B7050008B7050008CD4A0008F94A0008AE
:10006000254B0008514B00087D4B0008B7050008E0
:10007000B7050008B7050008B7050008B705000870
:10008000B7050008B7050008B7050008792500087E
:10009000A12500088D250008B5250008A94B0008FA
:1000A000B7050008B7050008B7050008B705000840
:1000B000B7050008B7050008B7050008B705000830
:1000C000B7050008B7050008B7050008B705000820
:1000D000B7050008B7050008B7050008B705000810
:1000E0000D4C0008B7050008B7050008B705000863
:1000F000B7050008B7050008B7050008B7050008F0
:10010000B7050008B7050008814C0008B7050008CE
:10011000B7050008B7050008B7050008B7050008CF
:10012000B7050008B7050008B7050008B7050008BF
:10013000B7050008B7050008B7050008B7050008AF
:10014000B7050008B7050008B7050008B70500089F
:10015000B7050008B7050008B7050008B70500088F
:10016000B7050008B7050008B7050008B70500087F
:10017000B7050008B7050008B7050008B70500086F
:10018000B7050008B7050008B7050008B70500085F
:10019000B7050008B7050008B7050008B70500084F
:1001A000B7050008B7050008B7050008B70500083F
:1001B000B7050008B7050008B7050008B70500082F
:1001C000B7050008B7050008B7050008B70500081F
:1001D000B7050008B7050008B7050008B70500080F
:1001E000B7050008B7050008B7050008B7050008FF
:1001F000B7050008B7050008B7050008B7050008EF
:10020000B7050008B7050008B7050008B7050008DE
:10021000B7050008B7050008B7050008B7050008CE
:10022000B7050008B7050008B7050008B7050008BE
:10023000B7050008B7050008B7050008B7050008AE
:10024000B7050008B7050008B7050008B70500089E
:10025000B7050008B7050008B7050008B70500088E
:10026000B7050008B7050008B7050008B70500087E
:10027000B7050008B7050008B7050008B70500086E
:10028000B7050008B7050008B7050008B70500085E
:10029000B7050008B7050008B7050008B70500084E
:1002A0008D140008000000000000000000000000A5
:1002B00053B94AB9002908BF00281CBF4FF0FF31CD
:1002C0004FF0FF3000F074B9ADF1080C6DE904CEC9
:1002D00000F006F8DDF804E0DDE9022304B0704721
:1002E0002DE9F047089D04468E46002B4DD18A42E9
:1002F000944669D9B2FA82F252B101FA02F3C2F11C
:10030000200120FA01F10CFA02FC41EA030E9440AC
:100310004FEA1C48210CBEFBF8F61FFA8CF708FBCD
:1003200016E341EA034306FB07F199420AD91CEBA5
:10033000030306F1FF3080F01F81994240F21C81D7
:10034000023E63445B1AA4B2B3FBF8F008FB10331F
:1003500044EA034400FB07F7A7420AD91CEB040454
:1003600000F1FF3380F00A81A74240F20781644424
:10037000023840EA0640E41B00261DB1D4400023A9
:10038000C5E900433146BDE8F0878B4209D9002D0D
:1003900000F0EF800026C5E9000130463146BDE897
:1003A000F087B3FA83F6002E4AD18B4202D3824201
:1003B00000F2F980841A61EB030301209E46002DB0
:1003C000E0D0C5E9004EDDE702B9FFDEB2FA82F205
:1003D000002A40F09280A1EB0C014FEA1C471FFA63
:1003E0008CFE0126200CB1FBF7F307FB131140EA4A
:1003F00001410EFB03F0884208D91CEB010103F117
:10040000FF3802D2884200F2CB804346091AA4B2D8
:10041000B1FBF7F007FB101144EA01440EFB00FEAC
:10042000A64508D91CEB040400F1FF3102D2A64511
:1004300000F2BB800846A4EB0E0440EA03409CE7B0
:10044000C6F12007B34022FA07FC4CEA030C20FA5D
:1004500007F401FA06F31C43F9404FEA1C4900FA7D
:1004600006F3B1FBF9F8200C1FFA8CFE09FB1811FA
:1004700040EA014108FB0EF0884202FA06F20BD96D
:100480001CEB010108F1FF3A80F08880884240F2BD
:100490008580A8F102086144091AA4B2B1FBF9F001
:1004A00009FB101144EA014100FB0EFE8E4508D9FC
:1004B0001CEB010100F1FF346CD28E456AD9023881
:1004C000614440EA0840A0FB0294A1EB0E01A14266
:1004D000C846A64656D353D05DB1B3EB080261EBD4
:1004E0000E0101FA07F722FA06F3F1401F43C5E9AE
:1004F000007100263146BDE8F087C2F12003D840E4
:100500000CFA02FC21FA03F3914001434FEA1C4725
:100510001FFA8CFEB3FBF7F007FB10360B0C43EA17
:10052000064300FB0EF69E4204FA02F408D91CEBC7
:10053000030300F1FF382FD29E422DD902386344C5
:100540009B1B89B2B3FBF7F607FB163341EA034165
:1005500006FB0EF38B4208D91CEB010106F1FF38B4
:1005600016D28B4214D9023E6144C91A46EA0046AB
:1005700038E72E46284605E70646E3E61846F8E63D
:100580004B45A9D2B9EB020864EB0C0E0138A3E786
:100590004646EAE7204694E74046D1E7D0467BE767
:1005A000023B614432E7304609E76444023842E7DF
:1005B000704700BF02E000F000F8FEE772B63A486C
:1005C00080F30888394880F3098839484EF6085185
:1005D000CEF20001086040F20000CCF200004EF6BE
:1005E0003471CEF200010860BFF34F8FBFF36F8FFD
:1005F00040F20000C0F2F0004EF68851CEF2000149
:100600000860BFF34F8FBFF36F8F4FF00000E1EE34
:10061000100A4EF63C71CEF200010860062080F30D
:100620001488BFF36F8F03F0DDFF03F07FFF04F04A
:1006300009F84FF055301F491B4A91423CBF41F821
:10064000040BFAE71C49194A91423CBF41F8040BDC
:10065000FAE71A491A4A1B4B9A423EBF51F8040B5B
:1006600042F8040BF8E700201749184A91423CBFB2
:1006700041F8040BFAE703F097FF04F067F8144C15
:10068000144DAC4203DA54F8041B8847F9E700F034
:1006900041F8114C114DAC4203DA54F8041B884761
:1006A000F9E703F07FBF00000006002000220020D1
:1006B000000000080000002000060020785100081B
:1006C000002200208022002080220020B85F00202D
:1006D000A0020008A4020008A4020008A402000866
:1006E0002DE9F04F2DED108AC1F80CD0D0F80CD0C8
:1006F000BDEC108ABDE8F08F002383F311882846F3
:10070000A047002003F0D4FBFEE703F04DFB00DF21
:10071000FEE700002DE9F04103F0C8FE30B12F4B99
:1007200000220C211A725A729972DA7203F080FE5A
:10073000074603F0F1FE0546C0BB294B9F4235D06A
:1007400001339F4235D027F0FF02264B9A4234D125
:10075000A84642F21074F8B200F0E8FB00F06CFC1E
:1007600008B10024A04600F0E7FB064648B354BB9E
:10077000464635B11C4B9F4203D0002403F0C4FE13
:100780002646002003F05EFE0EB100F02FF800F0C8
:1007900077FC00F091FE02F013F90546B4B900F0C1
:1007A000BFFC4FF47A7003F089FBF7E7A8460024FA
:1007B000D4E704464FF00108D0E7804641F2883480
:1007C000CCE70446D5E74FF47A74D2E702F0F8F8A4
:1007D000431BA342E3D900F009F8DCE70022002024
:1007E000010007B0000008B0263A09B0F8B5444B44
:1007F000444A1C461968013100F081800433934259
:10080000F8D16268404B9A4279D9404B9B6803F11A
:10081000006303F580239A4271D203F049FE03F08E
:100820005BFE002000F06EFE0220394B187000F0D5
:10083000A5FE384B0021D3F8E820C3F8E810D3F820
:100840001021C3F81011D3F81021D3F8EC20C3F80D
:10085000EC10D3F81421C3F81411D3F81421D3F8F1
:10086000F020C3F8F010D3F81821C3F81811D3F80A
:10087000183172B64FF0E023C3F8084DD4E90004F4
:10088000BFF34F8FBFF36F8F234AC2F88410BFF3BB
:100890004F8F536923F480335361BFF34F8FD2F8E6
:1008A000803043F6E076C3F3C905C3F34E335B01F2
:1008B00003EA060C29464CEA81770139C2F87472C2
:1008C000F9D2203B13F1200FF2D1BFF34F8FBFF3CA
:1008D0006F8FBFF34F8FBFF36F8F536923F40033D4
:1008E00053610023C2F85032BFF34F8FBFF36F8FB5
:1008F000202383F31188854680F308882047F8BDBC
:100900000000040820000408FFFF03080022002064
:10091000802200200044025800ED00E0094A49F21C
:100920006900136899B21B0C00FB013344F250615B
:100930001360054B186882B2000C01FB02001860BE
:1009400080B27047182200201422002000211022BB
:1009500010B5044600F026FE034B03CB2060616017
:100960001868A06010BD00BF00E8F11F2DE9F0413C
:10097000ADF54C7D0D46002140F275126AAC07467C
:100980000CA80B9100F00EFE4FF4C472002120461B
:1009900000F008FE0DF12C0802F012F84FF47A7204
:1009A000264BB0FBF2F0186093E80700012384E8BF
:1009B00007000DF5E5702382FFF7C8FF41F204330D
:1009C0001F4906A8238404F041FA13230DF2DB2209
:1009D0000DF1280C84F8323106AB1E46083203CEE6
:1009E000664542F8080C42F8041C3346F5D13188BC
:1009F0002046B378118041469370012201F0E6FF52
:100A0000002380B2E97E0393AB7E029305F11903C4
:100A100001930123009307A3D3E90023CDE90480C8
:100A2000384602F039FC0DF54C7DBDE8F08100BF81
:100A3000AFF300809E6AC421818A46EE84220020A2
:100A40007C4E00082DE9F043224DBBB001F0B8FF09
:100A500040F2ED22AB68C31A934232D906AF2B465F
:100A600028220021A860384602F0FEFD05F10E00A4
:100A700000F090FD002604465FFA80F905F10E08AB
:100A8000F3B2F100994501F1280107D908EB0603FB
:100A900008223846013602F0E7FDF1E7082301227B
:100AA0000534297B0C48A4B2CDE902320B4B0193EB
:100AB0003023CDE90474009304A3D3E9002302F0AA
:100AC000EBFB3BB0BDE8F083AFF3008078F6339FDB
:100AD00093CACD8D285C00209C320020355C00201C
:100AE000F0B58B8AC9B006460C46013B9BB2C92BB8
:100AF00047D8274D2F7B27BB05F10C030822394629
:100B000000933B46204602F073FC7B1CFAB2D900EE
:100B10001F46A38A013B9A4205DA0E3200232A447B
:100B200000920822EEE700230022C5E900230023FB
:100B3000AB6085F8D730C5F8D8302B7B0BB9E37E96
:100B40002B7306AD8122002127A800F02BFD012286
:100B5000294627A802F006F8002380B2E17E03931D
:100B6000A37E029304F1190301932823CDE90450D5
:100B70000093304604A3D3E9002302F08DFBFFF776
:100B800061FF49B0F0BD00BF26417272DF25D7B7C3
:100B9000285C002070B50D4614461E4602F012FB7C
:100BA00050B9022E10D1012C0ED112A3D3E900238B
:100BB0000120C5E9002307E0282C10D005D8012C1E
:100BC00009D0052C0FD0002070BD302CFBD10BA319
:100BD000D3E90023ECE70BA3D3E90023E8E70BA359
:100BE000D3E90023E4E70BA3D3E90023E0E700BF48
:100BF000AFF30080401DA12026812A0B78F6339F99
:100C000093CACD8D9E6AC421818A46EE26417272B6
:100C1000DF25D7B7F017304A39059E5613B501F0D6
:100C2000CFFE19490B68C31A642B184B08D9184A10
:100C30001C8892F900200860C2EB021222441A803C
:100C4000B3F90020002A1BDA00221A8011490A6831
:100C5000821AB2F57A7F04D90D4C0860227852428C
:100C60002270B3F900300322002093FBF2F3DBB2D1
:100C700063F3070063F30F2063F3174002B010BD66
:100C8000962AE3DD9622E0E70C5D0020145D00204B
:100C900010220020105D00202DE9F04F8DB080461D
:100CA0000D4602AF02F08EFA044600285BD12B7E7F
:100CB000022B1BD1EB8A012B18D101F081FE0646D5
:100CC000FFF72CFE03464FF4C87006F51676DFF8E2
:100CD0001492B3FBF0F202FB103316FA83F3C9F857
:100CE0000030EB7E33B97A4B00221A702C37BD46A8
:100CF000BDE8F08FAB8AE6B20134013BB3420CD9B8
:100D000007F10803E100082228461E4401F0F8011B
:100D10000023009602F06CFBECE707F11800FFF7E8
:100D200015FE324607F1180107F1080004F010F82B
:100D30000028D8D10F2E08D8654B1E70D9F8003086
:100D4000A3F51673C9F80030D0E7FB1DF871014612
:100D5000072200930346284602F04AFBF9794046F1
:100D600002F028FAC2E7EB8A282B26D010D8012BF4
:100D70001ED0052BBAD1BFF34F8F5649564BCA68C8
:100D800002F4E0621343CB60BFF34F8F00BFFDE777
:100D9000302BABD16B7EE946504C0133627BDBB22A
:100DA000934203D1EA7E237B9A420BD0CD469DE746
:100DB00029464046FFF7DAFD98E729464046FFF707
:100DC0008FFE93E74FF0000807F118031022284622
:100DD000A7F8188041460093012302F009FBAE8A70
:100DE000023EB6B2F31C9B109B000733DB08A9EB55
:100DF000C3039D460DF1080A1FFA88F34FEAC801A4
:100E00009E4201F110010AD90AEB08030822284684
:100E100008F101080093002302F0EAFAECE794F8E5
:100E2000D70000F079FBD4F8D83005461BB994F808
:100E3000D70000F081FBD4F8D83033449D4204D26F
:100E400094F8D700013000F077FB4FEA960B4FF093
:100E500000081FFA88F18B45D4E9003209D90AEB62
:100E60008801012203EB880008F1010800F0A2FBD1
:100E7000EFE7F31894F8D70042F10002C4E900321A
:100E8000D4F8D83006EB0308C4F8D88000F044FB4F
:100E9000804509D394F8D730D4F8D8000133401BEB
:100EA00084F8D730C4F8D800FF2E0D4D09D80023A0
:100EB000237300F053FB01F097FE288108B9FFF778
:100EC00095FC23689B0A01332B810023A3606DE707
:100ED0009532002000ED00E00400FA05285C0020B7
:100EE0008422002098320020F8B50E4C02260E4FC6
:100EF000A4F5805343F8307C237E3BB965692DB15E
:100F0000284601F0D9FB284603F00AFF2046A4F545
:100F1000A55401F0D1FB012EA4F1100400D1F8BDBD
:100F20000126E5E7A85700207C4F0008014B187008
:100F3000704700BF90220020334BF0B51C7B85B07A
:100F400034B1324B0E221A810024204605B0F0BD88
:100F50002F4A02AB1068516803C308232D492E485D
:100F60000DEB030203F004FF054630B9274B0A22BC
:100F70002A481A8101F028FBE6E70169B1F5E01F74
:100F800006D9224B0B2226481A8101F01DFBDCE713
:100F9000438B40F21342934207D01C490C20088136
:100FA0001946204801F010FBCFE71F4A024402F126
:100FB0001003994204D2154B10221C481A81E4E711
:100FC000103920468E1A144901F0F8FD05F1180178
:100FD00007463246204601F0F1FDAB68BB4202D124
:100FE000EB6883420AD0094B0D221A813B460090E0
:100FF0000F48D5E9021201F0E7FAA5E70D480124F0
:1010000001F0E2FAA1E700BF285C00208422002062
:10101000214F0008DCFF1B0000000408904E000870
:101020009C4E0008AE4E00080800FCF7CC4E0008AD
:10103000E94E0008124F000810B54FF040540C4B19
:1010400022689A4212D1627D0A4B0B481A70C9225B
:10105000237D0E30094900F8023C00F091FAE022AD
:101060000021204600F09EFA012010BD0020FCE780
:101070009AAD44C590220020285C00201600003064
:1010800037B502231D4C1E4D012220461D496B71B0
:10109000236804F580545B689847D4F8B034012283
:1010A00018495B6804F596609847002316494FF489
:1010B00080520193154B16480093164B02F054F8DA
:1010C000154B197811B1124802F074F801F078FC50
:1010D0000446FFF723FC4FF4C873B0FBF3F202FBA6
:1010E000130304F5167010FA83F00C4B186003F02C
:1010F00013FA08B10F232B8103B030BDC832002092
:101100008422002040420F0094220020950B00080A
:101110009C320020990C0008902200209832002078
:101120002DE9F04F224D2DED028B93B0DFF88CA00E
:10113000204F284602F014F90346002846D0002428
:101140001D4E0E94A046ADF84440A146CDE90F4493
:10115000027B8DF844200FAA9968406803C21B687F
:1011600043F000430E93336804F22C54D3F810B0CC
:1011700001F028FC10EB0A02CDF80090304606F58D
:10118000A55641F100030EA9D84740F65823002880
:10119000C8BF48F0010810369C42E4D1B8F1000FF6
:1011A0000ED0284602F0E0F887F80090C1E700BFB3
:1011B0009C320020175D0020C832002040420F0002
:1011C0003B78072B00F2398101333B7000230DF18E
:1011D0002C084FF0010A0A93ADF834300B93C8F88D
:1011E00004309FED9B8B00269F4C374623684FF0C1
:1011F000000B0DF11D0207A920468DF81CA08DF8EB
:101200001DB08DED008BD3F808905B46C8479DF864
:101210001C90B9F1000F1ED0102259460EA800F004
:10122000C1F9236808AA0AA95F6920460DF11E03C7
:10123000B8470FAB4F4698E8030083E803009DF8DA
:1012400034300EA928468DF844300A9B0E93DDE910
:10125000082302F051FA06F22C5640F6582304F502
:10126000A5549E4204F11004C0D1002FBBD12846E2
:1012700001F0A8FF002840D17C4E01F0A1FB3368AB
:1012800098423AD301F09CFB0446FFF747FB4FF42A
:10129000C87304F516748DF82870B0FBF3F202FBE6
:1012A000130314FA83F33360714E377817B90123AF
:1012B0008DF82830C7F110040EA8FFF747FB0EABDE
:1012C000E4B20DF12900D919062C28BF06242246C4
:1012D000013400F055F90AABE4B228460393182311
:1012E00004940293634B0193012300935AA3D3E91F
:1012F000002301F069FF0023337001F061FB5E4AB7
:101300001368C31AB3F57A7F30D3106001F05AFB2B
:1013100002460B46284602F031F8284601F052FFFB
:1013200020B3564B0EAE564C1B7B002B14BF032331
:101330000223637101F044FB4FF47A7301223146BA
:10134000B0FBF3F02060204601F0E4FB182380B2EC
:1013500002934C4B019340F25513CDE90360009387
:1013600028463FA3D3E9002301F02EFFFFF756FCE8
:101370000826C0F307238DF838000022C0F3074089
:10138000DFF804914FF4807A8DF839308DF83A0007
:10139000A6F10807332F54D9A7F134041923B4FB5D
:1013A000F3F103FB1143002B4DD0641A4FF01808E2
:1013B000B4FBF8F890450BD0FFF730FCC0F30723DF
:1013C0008DF83800C0F307408DF839308DF83A00B9
:1013D0001822B4FBF2F302FB134312AA04F0070431
:1013E00002EBD3034246C4F1080413F8103C43FA5D
:1013F00004F404F00104002C07F10107A9F81AA075
:101400000CBF4FF000730023BE4243EA4424C9F8E6
:101410001840A9F818A0BDD10836A02EB8D1174C95
:10142000237B2BB1FFF70EFB237B002B7FF47EAEDB
:1014300013B0BDEC028BBDE8F08F284601F094FF9D
:10144000C4E60024D7E70124D5E700BFAFF300804E
:101450000000000000000000401DA12026812A0B92
:10146000F1C6A7C1D068080FC8320020983200200A
:101470009532002094320020085D0020285C002076
:1014800084220020165D00200004025808B506489A
:1014900000F0CCFB054800F0C9FB054A05490020D7
:1014A000BDE8084003F036BCC83200207847002071
:1014B000585D0020E90E000870B5104C0025104E54
:1014C00002F030FE20803068238883420CD800254B
:1014D0002088013802F022FE23880544013BB5F53F
:1014E000802F2380F4D370BD02F018FE33680544CA
:1014F0000133B5F5802F3360E5D3E8E7445D002084
:10150000185D002002F0ECBE00F10060920000F5D2
:10151000802002F069BE0000054B1A68054B1B884D
:101520009B1A834202D9104402F0F8BD0020704794
:10153000185D0020445D002038B5074D044628683A
:10154000204402F0F1FD28B928682044BDE8384065
:1015500002F0FCBD38BD00BF185D0020064991F8BF
:10156000243033B100230822086A81F82430FFF7C1
:10157000CBBF0120704700BF1C5D002070470000FA
:10158000002310B5934203D0CC5CC4540133F9E777
:1015900010BD000003460246D01A12F9011B0029B3
:1015A000FAD1704702440346934202D003F8011B6C
:1015B000FAE770472DE9F8431F4D14460746884661
:1015C00095F8242052BBDFF870909CB395F8243036
:1015D0002BB92022FF2148462F62FFF7E3FF95F841
:1015E00024004146C0F1080205EB8000A24228BF5A
:1015F0002246D6B29200FFF7C3FF95F82430A41B11
:1016000017441E449044E4B2F6B2082E85F82460D4
:10161000DBD1FFF7A3FF0028D7D108E02B6A03EB4B
:1016200082038342CFD0FFF799FF0028CBD100205F
:10163000BDE8F8830120FBE71C5D0020202383F335
:10164000118862B670470000002383F3118862B6E8
:1016500070470000012070477047000010B4134627
:10166000026814680022A4465DF8044B604700003D
:1016700000F5805090F859047047000000F5805044
:1016800090F852047047000000F5805090F958041B
:10169000704700004E20704700F5805208B5FFF7F4
:1016A000CDFFD2F89834D2F894041844D2F890348C
:1016B0001844D2F878341844D2F888341844D2F850
:1016C00084341844FFF7C0FF08BD00002DE9F74F30
:1016D0000C4600F580511F46054691F8523490465D
:1016E000BDF830909BB1D1F874340133C1F8743433
:1016F00023689A0006D4237B082B0BD9627B0AB19E
:101700000F2B07D9D1F878340133C1F878344FF072
:10171000FF300FE0FFF792FFEB6AD3F8C42012F41A
:10172000001A0AD0D1F87C3400200133C1F87C348F
:10173000FFF78AFF03B0BDE8F08F22684FF0480B37
:10174000D3F8C460002A6B6AC6F30446B4BF42F003
:10175000804292041BFB063BCBF8002023685B0011
:101760004FEA066344BF42F00052CBF80020227BD0
:1017700043EA02437201CBF80430607B18B343F4B0
:101780004013CBF80430D1F8A4340133C1F8A434A9
:10179000AB1803F58353197B41F020011973207BAB
:1017A000019200F06DFF0330019A80105FFA8AF316
:1017B0000AF1010A83420DDA04EB83010BEB830388
:1017C00049689960F2E7AB1803F58353197B60F31E
:1017D0004511E3E70121EB6A04F10C00B140C3F8C5
:1017E000D010AB18214603F58253C3E9048705EBFB
:1017F000461303F58253183351F804CB814243F862
:1018000004CBF9D109882A442846198041F268039B
:10181000D65002F5805209F0030392F86C1043F0A1
:10182000100321F01F010B43214682F86C30424621
:10183000FFF70AFF3B46CDF8309003B0BDE8F04F0C
:1018400000F0E4BE2DE9F04700F58056044696F816
:101850005254002D40F00181037C032B40F0928014
:101860002B4628462F465FFA83FC944510DA01EB9D
:10187000CC0E51F83CC0BCF1000F04DBDEF804C014
:10188000BCF1000F02DB01370133ECE70130FBE76D
:10189000FFF7D4FEE36AF0B9D3F8800040F002000D
:1018A000C3F880004E23E06A002F6ED1D0F880305C
:1018B00043F00103C0F88030694B6A4A1B6803F1AA
:1018C000805303F52C539B009342A36240F2AF80F8
:1018D000654801F06FF84D2842D8DFF884814FEA5F
:1018E000004EDFF88891D8F800C04EEA8C0EC3F89D
:1018F00084E00CF1805303F52C539B00636100EBF3
:101900000C03D4F82CC0C8F80030C0F14E03DCF84A
:10191000800040F03000CCF880004FF0000CD4F88C
:101920001480E6465FFA8CF08242BCDD01EBC00A0F
:1019300051F83000002810DBDAF804A0BAF1000FEB
:101940000BDA09EA00400AF07F0A40EA0A0040F098
:10195000084048F82E000EF1010E0CF1010CE1E7F1
:101960009A6922F001029A6101F02AF80646E36AB8
:101970009B69D90704D501F023F8831BFA2BF6D90C
:10198000FFF762FE2846BDE8F087B7EB530F3DD264
:10199000DFF8CCE04FEA074CDEF800304CEA830C6D
:1019A000C0F888C003F1805003EB4703002700F51F
:1019B0002C50CEF80030BC468000A061E06AD0F820
:1019C000803043F00C03C0F88030D4F818E0FBB24C
:1019D0009A427FF771AF51F8330001EBC30800283A
:1019E000D8F8043001DB002B0EDB20F0604023F040
:1019F000604340F0005043F000434EF83C000EEBD3
:101A0000CC000CF1010C43600137E0E7836923F05F
:101A10000103836100F0D4FF0646E36A9B69DA079D
:101A2000AED500F0CDFF831BFA2BF6D9A8E7E26A0A
:101A3000936923F00103936100F0C2FF0746E36A54
:101A40009B69DB0705D500F0BBFFC31BFA2BF6D95A
:101A500096E7012586F8525492E7002592E700BFE9
:101A6000545D0020FCB500402C4F00080000FF072B
:101A700013B500F580540191606C00F053FE1F28EF
:101A80000AD920220199606C00F0C2FEA0F1200367
:101A90005842584102B010BD0020FBE700F58050CD
:101AA00008B5FFF7CBFD406C00F010FEBDE8084024
:101AB000FFF7CABD002202608281426082607047E7
:101AC0000022002310B5C0E90023002304460C3097
:101AD00020F8043CFFF7EEFF204610BD2DE9F0474B
:101AE000074688B09A46884607F58054684691466E
:101AF000FFF7A4FDFFF7E4FF606C00F0F9FD1F287D
:101B00002DD920226946606C00F006FF202826D1DE
:101B100094F852341BB303AD444605AB2E4608344B
:101B200003CE9E4244F8080C44F8041C3546F5D117
:101B30003068414620603846B388A380DDE9002341
:101B4000C9E90023BDF808304A46AAF80030FFF77B
:101B50007BFD534608B0BDE8F04700F045BD0020CE
:101B6000FFF772FD08B0BDE8F08700002DE9F84FDF
:101B70000023064600F58154054688461034C0E926
:101B80000133274B46F8303B374638462037FFF7BE
:101B900097FFA742F9D105F580544FF4805305F51E
:101BA000A3594FF0000A26630026676405F58357A2
:101BB00009F110094FF0000B1037E663C4E90D3648
:101BC000012384F8403084F84830A7F1180020370A
:101BD00047E910ABFFF76EFF47F8286C4F45F4D18B
:101BE000B8F1010F84F85884A4F85A64A4F85C642E
:101BF000A4F85E6484F86064A4F86264A4F8646481
:101C0000A4F8666484F8686402D9064800F0D2FE3D
:101C1000054B284653F82830EB62BDE8F88F00BF2B
:101C20007C4F0008504F00086C4F0008044B10B563
:101C3000197804464A1C1A70FFF798FF204610BD19
:101C4000515D00202DE9F04700295FD0304F314829
:101C5000B7FBF1F581428CBF0A201120431EB5FB72
:101C6000F0FC00FB1C50DCB220B1022B1846F5D86A
:101C7000002037E00CF1FF35B5F5806F32D2C4EBB0
:101C8000C4094FF47A7009F103034FEAE308C3F380
:101C9000C70308F1010AA4EB030E08FB00085FFA72
:101CA0008EF65AFA8EFEB8FBFEFEBEF5617F1BDC97
:101CB0001FFA8EF4581C56FA80F00CFB00FCB7FBA0
:101CC000FCFC6145D4D1013BDBB20F2BD0D8711E97
:101CD0000020C9B2072905D8107101201480558051
:101CE00053719171BDE8F08709F1FF334FEAE30EBC
:101CF000C3F3C7030EF10108E41A0EFB0000E6B2BD
:101D000058FA84F4B0FBF4F4A4B2D3E70846E9E748
:101D100000B4C4043F420F0038B540F27772C36A82
:101D2000154CC3F8BC200722C36AC3F8C820226838
:101D3000C16A930043F4C023C1F8A03002F180537C
:101D400002F16C01C56A03F52C53EA3289009B004D
:101D5000226041F0E061094AC361C5F8C01003F593
:101D6000D87103F56A7341629342836202D90448D1
:101D700000F020FE38BD00BF545D0020FCB50040DF
:101D80002C4F00082DE9F04F00F58055994689B099
:101D9000044695F858348A469046022B04D9002709
:101DA000384609B0BDE8F08F9E4A52F8231009B9B1
:101DB00042F823009C49C4F80CA00B7884F81090DA
:101DC000C3B9FFF73BFC994BD3F8EC2042F4807287
:101DD000C3F8EC20D3F8942042F48072C3F8942026
:101DE000D3F8942022F48072C3F8942001230B705E
:101DF000FFF72AFC95F851346BB9FFF71FFC8C4AAA
:101E000095F85834D35CEBB1012B24D0012385F82D
:101E10005134FFF719FCFFF711FCE26A936923F0D4
:101E20001003936100F0CCFD0746E36A9E6916F04B
:101E3000080617D000F0C4FDC31BFA2BF5D9FFF735
:101E400003FCACE70221132001F0E2FE0221152081
:101E500001F0DEFEDAE70221142001F0D9FE0221B2
:101E60001620F5E79A6942F001029A6100F0A8FD98
:101E70000746E36A9A69D00705D400F0A1FDC31BA9
:101E8000FA2BF6D9DBE79A69002704F5825B42F06A
:101E900002020BF1100B9A61E36A5F65FFF7D4FB56
:101EA000686C00F013FC202200216846FFF77AFBE3
:101EB00002A8FFF7FFFD6A460BEB06030DF1180EB3
:101EC000069794460833BCE80300F44543F8080C31
:101ED00043F8041C6246F4D1DCF800002036186098
:101EE000B6F5806F9CF804201A71DCD1002304F54C
:101EF000A252514620461A3285F8503485F85334A0
:101F0000FFF7A0FE074690B9E26A936923F0010348
:101F1000936100F055FD0546E36A9B69D9077FF59B
:101F20003EAF00F04DFD431BFA2BF5D937E795F88E
:101F30005F6495F85E243602C5F86CA4E36A46EA4D
:101F4000426695F860241643B5F85C2446EA0246DA
:101F5000DE61B8F1000F29D004F5A35241462046B6
:101F60000232FFF76FFE90B9E26A936923F0010332
:101F7000936100F025FD0546E36A9B69DA077FF56A
:101F80000EAF00F01DFD431BFA2BF5D907E795F8BE
:101F9000683495F867141B01C5F87084E26A43EA57
:101FA0000123B5F8641443EA0143D360E36A0026D1
:101FB0002046C3F8BC60FFF7AFFE85F859646FF0A8
:101FC0004042E36AB9F1030F1A651A4AE36A5A6597
:101FD0004FF00222E36A9A654FF0FF32E36AC3F8DA
:101FE000E0204FF00302E36ADA65E26A936943F4A2
:101FF000407393613FF4D4AEE26A936923F0010326
:10200000936100F0DDFC0646E36A9B69DB0705D5BA
:1020100000F0D6FC831BFA2BF6D9C0E6012385F825
:102020005234BDE6485D0020505D00200044025857
:10203000644F0008550200022DE9F04F054689B0B3
:1020400090469946002741F2680A00F58056EB6AEF
:10205000D3F8D830FB40D8074AD505EB47124FEAF2
:10206000471B52441379190742D4D6F88034013300
:10207000C6F8803413799A0605EB0B0248BFD6F8F0
:10208000A834524444BF0133C6F8A834137943F04E
:1020900008031371DB0723D596F8533403B305F512
:1020A00082546846FFF70CFD03AB18345C4404F11E
:1020B000080C2068083454F8041C1A46644503C20E
:1020C0001346F6D12068694610602846A2889A8097
:1020D0000123ADF808302B68CDE90089DB6B984708
:1020E000D6F8543423B1D6F89C340133C6F89C3466
:1020F0000137202FABD109B0BDE8F08F2DE9F04FAB
:102100000F468DB0044600F05DFC82468946002FE4
:102110005BD1E36AD3F8A02012F4FE0F03D10020B4
:102120000DB0BDE8F08FD3F8A420920141BF04F5B3
:102130008051D1F894240132C1F89424D3F8A4201A
:102140005606ECD0D3F8A450E669C5F3052548231C
:10215000E8464FF0000B03FB05664046FFF7AAFC7C
:10216000326851004ABF22F06043C2F38A4343F011
:102170000043920048BF43F080430093736813F418
:1021800000131BBF012304F580528DF80D308DF82C
:102190000D301EBFD2F8AC340133C2F8AC34F38832
:1021A00003F00F038DF80C309DF80C0000F068FA76
:1021B0005FFA8BF3984225D9F2180CA90BF1010BA9
:1021C000127A0B4403F82C2CEEE7012FA7D1E36A17
:1021D000D3F8B02012F4FE0FA1D0D3F8B4209501AB
:1021E00041BF04F58051D1F894240132C1F8942400
:1021F000D3F8B420500692D0D3F8B450266AC5F371
:102200000525A4E7EFB9E36AC3F8A85004A807AD11
:10221000FFF756FC98E80F0007C52B8000232046E7
:1022200004A9ADF81830236804F58054DB6BCDE9C0
:1022300004A9984758B1D4F88C340133C4F88C34CD
:102240006EE7012FE2D1E36AC3F8B850DEE7D4F8B5
:10225000903401200133C4F8903461E7F8B50546A5
:102260000F4600F58054012639462846FFF746FF01
:1022700010B184F85364F7E7D4F8543423B1D4F898
:102280009C340133C4F89C34F8BD0000C36AF0B537
:102290001A6C12F47F0F2BD01B6C00F5805441F2A6
:1022A00068054FF0010CC4F8A0340023471900EB77
:1022B00043125E012A44117911F0020F15D049072B
:1022C00013D4B959C66A0CFA01F1D6F8CCE011EA78
:1022D0000E0F0AD0C6F8D410117941F00401117123
:1022E000D4F888240132C4F888240133202BDED1AD
:1022F000F0BD00002B4B70B51E561B5C012B30D877
:10230000294D2A4A55F8233052F8264013B349B3D1
:10231000236D9A0510D54FF40073236500F052FB2E
:1023200050EA01020B4602D0013861F10003024677
:1023300055F82600FFF780FE236D9B012CD54FF04A
:10234000007255F82630226503F58053012283F888
:10235000592421E001232365102323654FF4805382
:10236000236570BD236DDA0702D4236D5B0706D5A4
:102370000523002155F826002365FFF76FFF236D25
:10238000D80602D4236D590606D55023012155F8ED
:1023900026002365FFF762FF55F82600BDE8704070
:1023A000FFF774BF684F0008485D00206C4F0008BD
:1023B00008B5FFF743F9FFF769FFBDE80840FFF7ED
:1023C00043B90000C36AD3F8C00010F07C5005D0B8
:1023D000D3F8C40080F40010C0F3405070470000F0
:1023E00000F5805008B5FFF729F9406C00F080F93E
:1023F000FFF72AF943090CBF0120002008BD0000A7
:1024000000F5805393F8592462B1C16A8A6922F0B9
:1024100001028A61D3F898240132C3F8982400227B
:1024200083F85924704700002DE9F74300F58251E5
:1024300098460025FFF702F9103141F2680E4FF07F
:10244000010900F5805C00EB4514744423795E07B4
:102450001CD4DB061AD58E69C36A09FA06F6D3F8CE
:10246000CC703E4212D04F6801970F689742019F8F
:1024700077EB08070AD2C3F8D460237943F004034A
:102480002371DCF884340133CCF8843401352031F5
:10249000202DD8D103B0BDE8F043FFF7D5B8000038
:1024A000F8B51E4600230F46054613701446FFF785
:1024B00097FF80F0010038701EB12846FFF782FFB9
:1024C0002070F8BD2DE9F04F994685B00B780E4687
:1024D0008046174601931378DDE90EBA029300F0A7
:1024E00071FA337804460D4613B93B78002B41D07E
:1024F00022462B464046FFF797FFFFF759FFFFF7AD
:102500007FFF4B463A463146FFF7CAFF33782BB17F
:10251000019B1BB1012005B0BDE8F08F3B7813B1E2
:10252000029B002BF6D108F5805303935C4575EBB5
:102530000A031FD2039BD3F85404D8B1BBEB0402A7
:102540000368D9686AEB050388474B463A4631462B
:102550004046FFF7A5FF337813B1019B002BD9D17B
:102560003B7813B1029B002BD4D100F02BFA044628
:102570000D46DBE70020CEE7002108B50846FFF74F
:10258000B9FEBDE8084001F019BB000008B5012103
:102590000020FFF7AFFEBDE8084001F00FBB0000D0
:1025A00008B500210120FFF7A5FEBDE8084001F0B5
:1025B00005BB0000012108B50846FFF79BFEBDE8FA
:1025C000084001F0FBBA00000FB4002004B07047CF
:1025D00013B56C46031D84E8060094E8030083E805
:1025E0000500012002B010BD73B58568019155B199
:1025F0001B885B0707D4D0E900369B6B9847019A8C
:10260000C1B23046A847012002B070BDF0B586685F
:1026100089B005460C465EB1BDF838305B070AD478
:10262000D0E900379B6B98472246C1B23846B04785
:10263000012009B0F0BD0022002301F10806CDE918
:10264000002300230A46ADF8083003AB10680832B7
:1026500052F8041C1C46B24203C42346F6D110684B
:1026600020609288A28000F0AFF90423ADF8083012
:102670002B68CDE90001DB6B694628469847D7E710
:10268000082817D909280CD00A280CD00B280CD000
:102690000C280CD00D280CD00E2814BF4020302060
:1026A00070470C2070471020704714207047182086
:1026B000704720207047000010B5037C044613B912
:1026C000006802F03DFB204610BD00000023BFF370
:1026D0005B8FC360BFF35B8FBFF35B8F8360BFF320
:1026E0005B8F7047BFF35B8F0068BFF35B8F7047F2
:1026F00070B505460C30FFF7F5FF044605F10806F6
:102700003046FFF7EFFFA04206D96D683046FFF76D
:10271000E9FF2544281A70BD3046FFF7E3FF201A71
:10272000F9E7000070B505464068A0B105F10C0658
:1027300005F10800FFF7D6FF04463046FFF7D2FF49
:10274000844204F1FF34304694BF6D680025FFF7E2
:10275000C9FF2C44201A70BD38B50C460546FFF75A
:10276000C7FFA04210D305F10800FFF7BBFF0444E8
:102770006868BFF35B8FB4FBF0F100FB11440120EC
:10278000AC60BFF35B8F38BD0020FCE72DE9F04162
:10279000144607460D46FFF7C5FF844228BF04468E
:1027A000D4B1B84658F80C6B4046FFF79BFF304455
:1027B000286040467E68FFF795FF331A9C4203D895
:1027C00001206C60BDE8F081A41B6B603B68204475
:1027D000AB60E8600220F5E72046F3E738B50C4629
:1027E0000546FFF79FFFA04210D305F10C00FFF74D
:1027F00079FF04446868BFF35B8FB4FBF0F100FB22
:1028000011440120EC60BFF35B8F38BD0020FCE772
:102810002DE9FF418846694607466C46FFF7B6FF3B
:10282000002506B204EBC606B4420AD0626808EB83
:10283000050120680834FEF7A3FE54F8043C1D444B
:10284000F2E729463846FFF7C9FF284604B0BDE83D
:10285000F0810000F8B505460C300F46FFF742FF47
:1028600005F1080604463046FFF73CFFA04230461B
:1028700088BF6C68FFF736FF201A386020B12C68DB
:102880003046FFF72FFF2044F8BD000073B5144613
:1028900006460D46FFF72CFF8442019028BF0446F0
:1028A000DCB101A93046FFF7D5FF019B33B932688F
:1028B000C5E90233C5E9002401200CE09C422860F0
:1028C00038BF0194019884426860F5D93368241AAE
:1028D0000220AB60EC6002B070BD2046FBE7000058
:1028E0002DE9FF410F4669466C46FFF7CFFF00B266
:1028F000002604EBC005AC4209D0D4F80480B81916
:1029000054F8081B42464644FEF73AFEF3E73046C9
:1029100004B0BDE8F081000038B50546FFF7E0FFE0
:10292000044601462846FFF717FF204638BD000041
:1029300000B59BB0EFF3098168226846FEF720FEE0
:10294000EFF30583044B9A6BDA6A9A6A9A6A9A6A79
:102950009A6A9A6A9B6AFEE700ED00E000B59BB0B8
:10296000EFF3098168226846FEF70AFEEFF305835C
:10297000044B9A6B9A6A9A6A9A6A9A6A9A6A9B6AEA
:10298000FEE700BF00ED00E000B59BB0EFF309816A
:1029900068226846FEF7F4FDEFF30583034B5A6B9C
:1029A0009A6A9A6A9A6A9A6A9B6AFEE700ED00E060
:1029B000FEE700000FB408B5029801F019FAFEE72F
:1029C00001F0D6BC01F0AEBC01F0ACBC2DE9F04783
:1029D0000D46044600219046284640F27912FEF743
:1029E000E1FD234620220021284604F1220700F0C1
:1029F0003BFE231D022220212846C02600F034FE83
:102A0000631D03222221284600F02EFEA31D03226F
:102A10002521284600F028FE04F108031022282171
:102A2000284600F021FE04F1100308223821284630
:102A300000F01AFE04F1110308224021284600F09C
:102A400013FE04F1120308224821284600F00CFE70
:102A500004F1140320225021284600F005FE04F161
:102A6000180340227021284600F0FEFD04F12003E7
:102A70000822B021284600F0F7FD04F121030822C6
:102A8000B821284600F0F0FD314608363B460822C2
:102A90002846013700F0E8FDB6F5A07FF4D1002705
:102AA00004F1330A04F1320308223146284600F0CB
:102AB000DBFD94F832304FEAC7099F4209F5A4764E
:102AC00015D3B8F1000F08D1314609F24F1604F5BD
:102AD00099730722284600F0C7FD27463B1B94F850
:102AE000322193420CD3F01DC008BDE8F0870AEBF9
:102AF0000703082231462846013700F0B5FDD8E724
:102B000007F233133146082228460836013700F011
:102B1000ABFDE3E713B50446084600212022234617
:102B200001900160C0F8031000F09EFD231D019884
:102B30000222202100F098FD631D0198032222212A
:102B400000F092FDA31D01980322252100F08CFDC9
:102B5000019804F108031022282100F085FD0720C8
:102B600002B010BDF8B50E4605461446002181227C
:102B70003046FEF717FD2B4608220021304600F0B4
:102B800073FD7CB90F246B1C07220821304600F02E
:102B90006BFD01235F1C6A78013B934204D3E01D67
:102BA000C008F8BD0824F4E7EB1921460822304696
:102BB00000F05AFD08343B46ECE7000030B50A440B
:102BC000084D91420DD011F8013B5840082340F3C5
:102BD0000004013B2C4013F0FF0384EA5000F6D1BF
:102BE000EFE730BD2083B8ED384A73B510686B4607
:102BF00051686A4603C308233549364802F0B8F8DD
:102C0000044670B9344A6B46106851686A4603C37B
:102C1000082332492F4802F0ABF8044630BB0A20A3
:102C200022E00369B3F5E01FECD8418B40F2134278
:102C30009142E7D12A4A024402F110018B42E1D3CA
:102C4000103B244900209D1AFFF7B8FF04F118013A
:102C500006462A460020FFF7B1FFA3689E42D1D165
:102C6000E3689842CED1002002B070BD0369B3F58D
:102C7000E01F22D8B0F8661040F2134291421ED1F4
:102C8000174A024402F15C018B421AD35C3B1149A2
:102C900000209D1AFFF792FF04F1640106462A46C0
:102CA0000020FFF78BFFA268034696420BD1E06835
:102CB000834214BF0D200020D6E70B20D4E70C2060
:102CC000D2E71020D0E70D20CEE700BF214F00084B
:102CD000DCFF1B0000000408BC4F000890FF1B0035
:102CE0000800FCF72DE9F041C56915B9C161BDE8DF
:102CF000F0814B68AC4623F06047C3F38A464FEA45
:102D0000D37EC3F3807816EA230638BF3E462B46AF
:102D10005A68BEEBD27F22F060440AD0002A18DA4B
:102D2000A40CB44217D19D420FD10D60DEE71346CB
:102D3000EEE7A74207D102F08044C2F38072424519
:102D40000BD054B1EFE708D2EDE7CCF800100B60E0
:102D5000CDE7B44201D0B442E5D81A689C46002AB7
:102D6000E5D11960C3E700002DE9F047089D01F0A7
:102D7000070400EBD1004FF47F494FEAD508224405
:102D800005F00705944201D1BDE8F08704F007077C
:102D900005F0070A111B08EBD50E57453E4613F800
:102DA0000EC038BF5646C6F108068E4228BF0E46F2
:102DB000E108415C34443544B94029FA06F721FA68
:102DC0000AF1FFB28CEA010147FA0AF739408CEAAE
:102DD000010C03F80EC0D5E780EA0120082341F278
:102DE000210201B2013B4000002980B2B8BF50402F
:102DF00013F0FF03F5D1704738B50C468D18A54286
:102E000000D138BD14F8011BFFF7E6FFF7E700001B
:102E100002684AB1136801890360C38801339BB219
:102E20009942C38038BF03811046704770B588B09F
:102E3000044620220D4668460021FEF7B3FB2046DB
:102E40000495FFF7E5FF024660B16B46054608AE04
:102E50001C46083503CCB44245F8080C45F8041C60
:102E60002346F5D1104608B070BD0000082817D9D8
:102E700009280CD00A280CD00B280CD00C280CD018
:102E80000D280CD00E2814BF4020302070470C2095
:102E9000704710207047142070471820704720207A
:102EA00070470000082817D90C280CD910280CD915
:102EB00014280CD918280CD920280CD930288CBFFC
:102EC0000F200E207047092070470A2070470B2002
:102ED00070470C2070470D207047000010B54B68FC
:102EE00023B9CA8A63F30902CA8210BDC4681A688A
:102EF0001C60C360438A013B43824A60EFE70000E5
:102F00002DE9F84F1D46CB8A0F468146C3F30901D0
:102F1000924605290B4630D00020AAB207F11A04C8
:102F20009EB21FFA80F8042E0FD8904503F10103DA
:102F300006D30A44FB8A62F309030120FB821AE0EC
:102F40001AF800600130E654EAE79045F1D2A1F1A9
:102F5000050B1C237C68BBFBF3F203FB12BB1FFABF
:102F60008BF6002C45D14846FFF752FF044638B98E
:102F700078606FF00200BDE8F88F4FF00008E6E7D8
:102F8000002606607860ADB24FF0000B454510D9C1
:102F90000AEB0803221D13F8011B08F101089155E3
:102FA000B1B21FFA88F81B292BD0454506F101065E
:102FB000F1D8FB8AC3F30902154465F30903BCE7A2
:102FC00001321C4692B22368002BF9D16B1F0B44CF
:102FD0001C21B3FBF1F301339BB29A42D3D2BBF174
:102FE000000FD0D14846FFF713FF20B9C4F800B056
:102FF000BFE70122E7E7C0F800B05E462060044664
:10300000C1E74545D5D94846FFF702FF08B920601A
:10301000AFE7C0F800B0002620600446B6E7000025
:103020002DE9F04F2DED028B83B007469146BDF898
:103030003C50CDE90013002A00F092802DB10E9B88
:10304000002B00F08D80072D32D807F10C00FFF720
:10305000DFFE044638B96FF00204204603B0BDEC31
:10306000028BBDE8F08F14220021FEF79BFA2A465E
:103070000E9904F10800FEF783FA681CC0B2FFF74E
:1030800011FFFFF7F3FE207499F80030013803F0C8
:103090001F0314FA80F063F03F0303723846009B6D
:1030A00043F0004161602146FFF71CFE0124D4E794
:1030B0004FF0000800F10C034FF0800A46464446EA
:1030C00008EE103A18EE100AFFF7A2FE8346002819
:1030D000C1D014220021FEF765FAC6BB019B022075
:1030E000ABF808300E9B00F1080299195BFA82F2E6
:1030F0000130C0B2082801D0AE422AD3FFF7D2FE79
:10310000AE4208BF4FF0400AFFF7B0FE99F800202A
:10311000411E009B02F01F0201345BFA81F142EA7A
:10312000481288F0010824B24AEA020A43F0004239
:1031300081F808A059468BF810003846CBF80420D7
:103140004FF0000AFFF7CEFDAE42BBD185E700206D
:10315000C8E711F801CB013602F801CBB6B2C7E7D8
:103160006FF0010479E70000F8B515460E462822F5
:10317000002104461F46FEF715FA069BB5F5001F11
:10318000A760636004F10C00079B34BF6A094FF627
:10319000FF722362002397B29A4205D8002303608E
:1031A00027826382A382F8BD066001333046203651
:1031B000F2E7000003781BB94BB2002BC8BF0170C7
:1031C00070470000007870472DE9F74FDDF83C901C
:1031D000804692469B46BDF830500D9E9DF8384083
:1031E000BDF84070B9F1000F01D1002F51D11F2C53
:1031F0004FD898F80000B0B9072F47D835F003032F
:1032000047D13A4649464FF6FF702D02FFF7F4FDCD
:1032100020F0010045EA04644004400C44EA4024E4
:103220004FF6FF7321E040EA0520072F40EA0464CF
:10323000F6D900254FF6FF73C5F12000A5F1200255
:103240002AFA05F108350BFA00F02BFA02F20143D5
:1032500018461143C9B2FFF7BFFD402D0346EBD11D
:103260003A464946FFF7C8FD0346324621464046E6
:10327000CDE90097FFF7D4FE33780133DBB21F2B83
:1032800088BF0023337003B0BDE8F08F6FF00300F8
:10329000F9E76FF00100F6E72DE9F04F85B09246AF
:1032A00006469B46DDF848800F9D9DF840209DF81E
:1032B0004490BDF84C70B8F1000F01D1002F49D1F6
:1032C0001F2A47D83378002B47D00C029DF83810BE
:1032D000072F44EA026444EAC93444EA014444EA58
:1032E000030444F0800432D900234FF6FF72C3F187
:1032F000200CA3F120002AFA03F103930BFA0CFC33
:103300002BFA00F041EA0C0101431046C9B2FFF765
:1033100063FD039B02460833402BE8D13A46414601
:10332000FFF76AFD03462A4621463046CDE900876D
:10333000FFF776FEB9F1010F06D12B780133DBB22E
:103340001F2B88BF00232B7005B0BDE8F08F4FF610
:10335000FF73E8E76FF00100F6E76FF00300F3E7B3
:10336000C06900B104307047C3691A68C261C2689D
:103370001A60C360438A013B438270472DE9F041E4
:10338000D0F8188014461D46184E4146002709B94A
:10339000BDE8F081D1E90223A21A65EB030396424E
:1033A00077EB03031ED283698B420DD1FFF796FDA5
:1033B00083691B688361C3680B60438AC160013BFA
:1033C000816943828846E2E7FFF788FD0B68C8F809
:1033D0000030C3680B60438AC160013B4382D8F868
:1033E0000010D4E788460968D1E700BF80841E003A
:1033F0002DE9F04F8BB00D4614469B46DDF85090FA
:103400008046002800F01881B9F1000F00F0148107
:10341000531E3F2B00F21081012A03D1BBF1000F94
:1034200040F00A810023CDE90833B8F81430B5EB39
:10343000C30F4FEAC30703D300200BB0BDE8F08FE2
:103440002B199F42D8F80C3036BF7F1B2746FFB29E
:103450001BB9D8F81030002B7AD0272D4DD8C5F1E4
:10346000280600232946B742009308ABD8F8080085
:103470002CBFF6B23E46A7EB060A354432465FFA49
:103480008AFAFFF771FCB8F81430282103F10053D1
:10349000053BDB000493D8F80C300393039B13B176
:1034A000BAF1000F2CD1D8F8100040B1BAF1000FDA
:1034B00005D008AB5246691A0096FFF755FC38B2A2
:1034C000002FB9D066070AD00AAB624203EBD401E1
:1034D00002F0070211F8083C134101F8083C082CDF
:1034E0003DD9102C40F2B580202C40F2B780BBF1C2
:1034F000000F00F09C80082335E0BA460026C2E7A2
:10350000049BE02B28BFE02306930B44AB420593BA
:1035100015D95A1B0398691A0096924508AB00F119
:10352000040034BF5246D2B20792FFF71DFC079A3F
:103530001644AAEB020A1544F6B25FFA8AFA049B13
:10354000069A05999B1A0493039B1B680393A5E7AE
:1035500000933A4608AB2946D8F80800ADE7BBF11E
:10356000000F13D00123B4EBC30F6BD0082C12D87B
:103570009DF82030621E23FA02F2D50706D54FF0DF
:10358000FF3202FA04F423438DF820309DF82030F6
:1035900089F8003051E7102C12D8BDF82030621E97
:1035A00023FA02F2D10706D54FF0FF3202FA04F4F3
:1035B0002343ADF82030BDF82030A9F800303CE7B7
:1035C000202C0FD80899631E21FA03F3DA0705D5DA
:1035D0004FF0FF3202FA04F40C430894089BC9F838
:1035E00000302AE7402C2AD0611EC4F12102A4F148
:1035F0002103DDE9086526FA01F105FA02F225FA50
:1036000003F311431943CB0711D50122A4F1200381
:10361000C4F1200102FA03F322FA01F1A2400B43A4
:10362000524263EB430332432B43CDE90823DDE9E8
:103630000823C9E9002300E76FF00100FDE66FF001
:103640000800FAE6082CA1D9102CB4D9202CEED809
:10365000C4E7BBF1000FAED0022384E7BBF1000F3B
:10366000BCD004237FE70000012A30B5144638BFE0
:10367000012485B00025402C28BF4024012ACDE933
:10368000025518D81B788DF8083063070AD004ABB0
:10369000624203EBD40502F0070215F8083C9340A0
:1036A00005F8083C034600912246002102A8FFF7D6
:1036B0005BFB05B030BD082AE4D9102A03D81B886B
:1036C000ADF80830E1E7202A95BF1B68D3E9002355
:1036D0000293CDE90223D8E710B5CB681BB98B6004
:1036E0000B618B8210BDC4681A681C60C360438A7A
:1036F000013B4382CA60F0E72DE9F04F95B00446E4
:103700000D46CDE904230B681806C3F3C01147BF6B
:10371000C3F3C03BC3F306264FF0020B0E46002B4B
:1037200080F2018213F0C04940F0FD812A7B002A1B
:1037300000F0F981BBF1020F03D02078B04240F0D5
:10374000F581C3F30460089003F07F00069059B33D
:10375000C3F3074A7606069B2A4446EA0B4692F8CC
:103760000380002246EA83460023CDE90A235FEA6C
:10377000D81346EA0A0603936AD0069B52460AA962
:10378000204600935B466768B847002800F0D18167
:10379000A76987B9314604F10C00FFF747FB0746DC
:1037A000C8B96FF0020057E0C3F30F2A590608BFEB
:1037B0000AF0030ACEE73B699E420DD03F68002F16
:1037C000F9D1314604F10C00FFF730FB0746002821
:1037D000E7D0A3693B60A761FE7D08F01F03C6F335
:1037E00084060793F01A9B1B1FFA80FC0028B8BFC1
:1037F0000CF120001FFA83FCB8BF00B2002B099324
:10380000B8BF0CF12003D7E90221BCBF1BB209935A
:1038100052EA010335D0049EDFF8D4C2B21A059EE5
:1038200066EB01010026944576EB010329D395F858
:103830000DE097F81AC0E64516D1039B002B78D00F
:1038400001281EDCA948904276EB010316D338E02C
:10385000A76927B96FF00C0015B0BDE8F08F3B6980
:103860009E42B9D03F68F4E7A048904276EB01034E
:1038700001D30020F0E7039B002BFAD0099B0F2B0C
:1038800018DCFA7D4FEA88033946204602F003022D
:1038900003F07C031343FB75FFF720FB6B7BBB76C8
:1038A000039B3BB9FB7DC3F38402013262F38603C1
:1038B000FB75CFE76A7BBB7E9A42DAD1039B002B74
:1038C00037D04FEA9813022B33D0049B14220021E7
:1038D0000FA8BB60059BFB60FDF764FE049B0CA971
:1038E00020460C93059BADF846A00D932B1D8DF83B
:1038F00048B00E932B7B013BDBB2ADF84430079B05
:103900008DF84930089B8DF84A30069B8DF84B3076
:1039100094F8243083F001038DF84C30A368984765
:10392000FB7DC3F38403013303F01F039B02FB827F
:103930009FE7FB7DC8F34012B2EBD31F40F0FC8041
:10394000C3F38403079A934240F0F98003994FEA46
:1039500098122B7B00294DD0D2075DD4032B40F267
:10396000F180049BAE1D394604F10C00BB60324669
:10397000059BFB602B7B033BDBB2FFF7C1FA002802
:103980000CDA39462046FFF7A9FAFB7DC3F384031E
:10399000013303F01F039B02FB8202E7AB88DDE9E2
:1039A0000A843B834FF6FF73C9F12000A9F120027E
:1039B00028FA09F109F1080904FA00F024FA02F2E0
:1039C000014318461143C9B2FFF706FAB9F1400F97
:1039D0000346E9D1B88231462A7B033AD2B2FFF7D7
:1039E0000BFAFB7DB882DA43C2F3C01262F3C7134D
:1039F000FB753EE782B92E1D013B394604F10C00F0
:103A0000DBB23246FFF77CFA0028BADB2A7B31466C
:103A1000B88A013AD2B2E2E7F98A013BC1F309015F
:103A2000DAB204295CD8281D002307F11B069A424C
:103A300008D910F801CB013306F801C00131DBB21F
:103A40000529F4D1049993420C9138BF04330599A8
:103A50002CBF002355FA83F30D9107F11B010E9142
:103A6000796810930F91291DFB8AADF846A0C3F326
:103A700009038DF848B01A44079B8DF84930089B1C
:103A8000ADF844208DF84A30069B8DF84B3094F801
:103A9000243083F001038DF84C300023B88A7B601A
:103AA0002A7B013AFFF7A8F93B8BB882834203D106
:103AB000A3680CA92046984720460CA9FFF70CFEE6
:103AC000FB7DBA8AC3F38403013303F01F039B0217
:103AD000FB823B8B9A420CBF00206FF01000BBE6CC
:103AE0007B68002BAED0052006E000BF40420F00EF
:103AF00080841E001C3033461E68002EFAD1091A3D
:103B00002E1D081D184401EB090C5FFA89F3BCF166
:103B10001B0F97D89A4295D916F8013B09F1010974
:103B200000F8013BEFE76FF0090095E66FF00A003F
:103B300092E66FF00B008FE66FF00D008CE66FF0F1
:103B40000E0089E66FF00F0086E600BFEFF30983F1
:103B5000054968334A6B22F001024A6383F30988FE
:103B6000002383F31188704700EF00E0202080F3EA
:103B7000118862B60D4B0E4AD96821F4E061090440
:103B8000090C0A430B49DA60D3F8FC2042F080723A
:103B9000C3F8FC20084AC2F8B01F116841F00101C7
:103BA00011601022DA7783F82200704700ED00E000
:103BB0000003FA0555CEACC5001000E0202310B577
:103BC00083F311880E4B5B6813F4006314D0F1EE9D
:103BD000103AEFF309844FF08073683CE361094BBE
:103BE000DB6B236684F3098800F0B4F810B1064B50
:103BF000A36110BD054BFBE783F31188F9E700BF14
:103C000000ED00E000EF00E00B0700080E070008E1
:103C1000090100F16043012203F56143C9B283F851
:103C2000001300F01F039A4043099B0003F1604317
:103C300003F56143C3F880211A607047024B0022EC
:103C4000C3E900339A6070475C5D002000238268FE
:103C50000374054B1B6899689142FBD25A68036054
:103C600042601060586070475C5D002008B52023FA
:103C700083F31188037C032B05D0042B0DD02BB9C3
:103C800083F3118808BD436900221A604FF0FF33A7
:103C90004361FFF7DBFF0023F2E7D0E90032136056
:103CA0005A60F3E7002382680374054B1B68996828
:103CB0009142FBD85A6803604260106058607047B8
:103CC0005C5D0020054B1969087418680268536030
:103CD0001A60186101230374FCF702BD5C5D0020CB
:103CE0004B1C30B5044687B00A4D10D02B6901A893
:103CF000094A00F0FDF82046FFF7E4FF049B13B1EA
:103D000001A800F031F92B69586907B030BDFFF701
:103D1000D9FFF8E75C5D00206D3C000838B50C4D1C
:103D2000044641612B6981689A68914203D8BDE8D5
:103D30003840FFF78BBF1846FFF7B4FF01232C6113
:103D4000014623742046BDE83840FCF7C9BC00BFDB
:103D50005C5D0020044B1A681B6990689B68984260
:103D600094BF0020012070475C5D002010B5084C16
:103D7000236820691A6854602260012223611A7442
:103D8000FFF790FF01462069BDE81040FCF7A8BC92
:103D90005C5D002008B5FFF7DDFF18B1BDE8084005
:103DA000FFF7E4BF08BD0000FFF7E0BFFEE700003B
:103DB00010B50C4CFFF742FF00F08CF880220A4946
:103DC000204600F03DF8012344F8180C0374FFF777
:103DD000CDFE002383F3118862B60448BDE810408D
:103DE00000F04EB8845D0020C84F0008D84F00088E
:103DF00008B572B6034B586200F086FA00F054FB27
:103E0000FEE700BF5C5D002000F0E8B8EFF3118032
:103E100020B9EFF30583202282F311887047000058
:103E200010B530B9EFF30584C4F3080414B180F37E
:103E3000118810BDFFF7AEFF84F31188F9E7000089
:103E400082600222028270478368A3F17C0243F8F9
:103E50000C2C026943F83C2C426943F8382C074A81
:103E600043F81C2CC268A3F1180043F8102C02225E
:103E700003F8082C002203F8072C7047F906000805
:103E800010B5202383F31188FFF7DEFF00210446DD
:103E9000FFF744FF002383F31188204610BD000084
:103EA000024B1B6958610F20FFF70CBF5C5D0020BF
:103EB000202383F31188FFF7F3BF000008B5014604
:103EC000202383F311880820FFF70AFF002383F3E0
:103ED000118808BD054B4FF0FF3103F11402C3E90F
:103EE00005220022C3E90712704700BF5C5D002075
:103EF00070B51C4E05460C46C0E9032300F08CFB50
:103F0000334653F8142F9A420DD130620A2C2CBF3D
:103F100000190A302A60C5E90124C6E90555BDE843
:103F2000704000F063BB316A431AE31838BF1C4687
:103F30009368A34202D9081900F068FB73699A6874
:103F400094420CD85A68AC602B606A6015609A681D
:103F50005D60121B9A604FF0FF33F36170BDA41ACD
:103F60001B68ECE75C5D002038B51B4C6369984228
:103F70000DD08168D0E9003213605A600022C2601F
:103F80009A680A449A604FF0FF33E36138BD0368D2
:103F90002246002142F8143F93425A60C16003D187
:103FA000BDE8384000F02CBB9A688168256A0A4455
:103FB0009A6000F031FB6369411B9A688A42E5D937
:103FC000AB181D1A206A092D98BF01F10A02BDE83D
:103FD0003840104400F01ABB5C5D00202DE9F04130
:103FE000184C002704F11406656900F015FB236ADC
:103FF000AA68C11A8A4215D81344D5F80C802362E6
:10400000D5E9003213605A606369EF60B34201D1B1
:1040100000F0F6FA87F311882869C047202383F35C
:104020001188E1E76169B14209D013441B1ABDE868
:10403000F0410A2B2CBFC0180A3000F0E7BABDE8E7
:10404000F08100BF5C5D002000207047FEE70000AB
:10405000704700004FF0FF3070470000BFF34F8FF4
:10406000044B1A695107FCD1D3F810215207F8D13B
:10407000704700BF0020005208B50D4B1B78ABB94C
:10408000FFF7ECFF0B4BDA68D10704D50A4A5A60F8
:1040900002F188325A60D3F80C21D20706D5064ABD
:1040A000C3F8042102F18832C3F8042108BD00BF1F
:1040B000185F0020002000522301674508B5114B0E
:1040C0001B78F3B9104B1A69510703D5DA6842F02F
:1040D0004002DA60D3F81021520705D5D3F80C213D
:1040E00042F04002C3F80C21FFF7B8FF064BDA6834
:1040F00042F00102DA60D3F80C2142F00102C3F869
:104100000C2108BD185F0020002000520F289ABF24
:1041100000F5806040040020704700004FF400303C
:1041200070470000102070470F2808B50BD8FFF724
:10413000EDFF00F500330268013204D10430834200
:10414000F9D1012008BD0020FCE700000F2870B560
:10415000054645D8FFF75AFE224CFFF77FFF06467B
:10416000FFF78AFF4FF0FF33072D6361C4F8143166
:1041700020D82361FFF772FF2B0243F02403E36092
:10418000E36843F08003E36023695A07FCD42846C0
:10419000FFF764FF4FF40031FFF7B8FF00F060F95C
:1041A0003046FFF78BFFFFF73BFE2846BDE8704027
:1041B000FFF7BABFC4F81031FFF750FFA5F10803AD
:1041C0001B0243F02403C4F80C31D4F80C3143F043
:1041D0008003C4F80C31D4F810315B07FBD4D6E768
:1041E000002070BD002000522DE9F84F40EA020384
:1041F00005460C461746D80602D00020BDE8F88FC9
:1042000027F01F07DFF8D4B0FFF736FF2744BC4282
:1042100003D10120FFF752FFF0E720222946204674
:1042200000F096FD10B920352034F0E72B4605F15B
:1042300020021E68711CE0D104339A42F9D1FFF7C5
:10424000E5FD05F17843234AB3F5801F224B28BFD3
:104250009A4603F1040338BF9046A2F1080228BF32
:104260009846A3F108033ABF9146DA469946FFF70C
:10427000F5FEC8F80060A5EB040CD9F8002004F1A5
:104280001C0142F00202C9F80020221FDAF8006087
:1042900016F00506FAD152F8043F8A424CF8023073
:1042A000F4D1BFF34F8FFFF7D9FE4FF0FF32C8F8BC
:1042B0000020D9F8002022F00202C9F80020FFF700
:1042C000AFFD20222146284600F042FD0028AAD05A
:1042D00030469FE714200052102100521020005257
:1042E00010B5084C237828B11BB9FFF7C5FE012390
:1042F000237010BD002BFCD02070BDE81040FFF7EC
:10430000DDBE00BF185F002038B5054D0024033422
:10431000696855F80C0B00F0B5F8122CF7D138BDD0
:10432000F04F000870B5104E82B0FFF76FFD0546E4
:1043300000F072F9326803469042336037BF0B4A8F
:104340000A495168146836BF0131D1E90041516012
:104350000419284641F100010191FFF761FD204653
:10436000019902B070BD00BF1C5F0020205F0020DB
:1043700070B5124E82B0FFF749FD054600F04CF9CA
:10438000326803469042336037BF0D4A0C4951688A
:10439000146836BF0131D1E9004151600419284643
:1043A00041F100010191FFF73BFD4FF47A720023C8
:1043B00020460199FBF77CFF02B070BD1C5F002016
:1043C000205F00200244074BD2B210B5904200D1CA
:1043D00010BD441C00B253F8200041F8040BE0B2B9
:1043E000F4E700BF504000580E4B30B51C6F24045A
:1043F00005D41C6F1C671C6F44F400441C670A4CF6
:1044000002442368D2B243F480732360074B904286
:1044100000D130BD441C51F8045B00B243F8205079
:10442000E0B2F4E7004402580048025850400058F7
:1044300007B5012201A90020FFF7C4FF019803B0CE
:104440005DF804FB13B50446FFF7F2FFA04205D068
:10445000012201A900200194FFF7C6FF02B010BDA0
:104460000144BFF34F8F064B884204D3BFF34F8FF5
:10447000BFF36F8F7047C3F85C022030F4E700BFD2
:1044800000ED00E00144BFF34F8F064B884204D398
:10449000BFF34F8FBFF36F8F7047C3F870022030A8
:1044A000F4E700BF00ED00E0704700000020704717
:1044B000074B45F255521A6002225A6040F6FF72CD
:1044C0009A604CF6CC421A600122024B1A70704777
:1044D000004800582C5F0020034B1B781BB1034B96
:1044E0004AF6AA221A6070472C5F00200048005844
:1044F000034B1A681AB9034AD2F8D0241A607047DD
:10450000285F002000400258024B4FF48032C3F86D
:10451000D02470470040025808B5FFF7E9FF024B6E
:104520001868C0F3806008BD285F002070B5BFF335
:104530004F8FBFF36F8F1A4A0021C2F85012BFF39A
:104540004F8FBFF36F8F536943F400335361BFF351
:104550004F8FBFF36F8FC2F88410BFF34F8FD2F825
:10456000803043F6E074C3F3C900C3F34E335B01FC
:1045700003EA0406014646EA81750139C2F8605231
:10458000F9D2203B13F1200FF2D1BFF34F8F5369C3
:1045900043F480335361BFF34F8FBFF36F8F70BD10
:1045A00000ED00E0FEE700000A4B0B480B4A90428A
:1045B0000BD30B4BC11EDA1C121A22F003028B42E2
:1045C00038BF00220021FCF7EDBF53F8041B40F870
:1045D000041BECE7F8510008B85F0020B85F00202A
:1045E000B85F00207047000000F0D8B8034B0022ED
:1045F00058631A610222DA60704700BF000C004065
:10460000014B0022DA607047000C0040014B5863F8
:10461000704700BF000C0040014B586A704700BF54
:10462000000C00404B6843608B688360CB68C360BC
:104630000B6943614B6903628B6943620B680360DA
:104640007047000008B53C4B40F2FF713B48D3F87F
:1046500088200A43C3F88820D3F8882022F4FF6218
:1046600022F00702C3F88820D3F88820D3F8E0208E
:104670000A43C3F8E020D3F808210A43C3F808210D
:104680002F4AD3F808311146FFF7CCFF00F58060C0
:1046900002F11C01FFF7C6FF00F5806002F138014E
:1046A000FFF7C0FF00F5806002F15401FFF7BAFF89
:1046B00000F5806002F17001FFF7B4FF00F5806043
:1046C00002F18C01FFF7AEFF00F5806002F1A80156
:1046D000FFF7A8FF00F5806002F1C401FFF7A2FF19
:1046E00000F5806002F1E001FFF79CFF00F58060BB
:1046F00002F1FC01FFF796FF02F58C7100F5806076
:10470000FFF790FF00F0FEF80E4BD3F8902242F036
:104710000102C3F89022D3F8942242F00102C3F8B8
:1047200094220522C3F898204FF06052C3F89C20D1
:10473000054AC3F8A02008BD0044025800000258F2
:104740003850000800ED00E01F00080308B500F035
:10475000C7FAFFF72DFB0E4BD3F8DC2042F04002E6
:10476000C3F8DC20D3F8042122F04002C3F804216E
:10477000D3F80431074B1A6842F008021A601A682D
:1047800042F004021A60BDE80840FFF7B1BE00BF66
:10479000004402580018024870470000114BD3F83B
:1047A000E82042F00802C3F8E820D3F8102142F0D4
:1047B0000802C3F810210C4AD3F81031D36B43F030
:1047C0000803D363C722094B9A624FF0FF32DA62C3
:1047D00000229A615A63DA605A6001225A611A60B3
:1047E000704700BF004402580010005C000C0040FD
:1047F000094A08B51169D3680B40D9B29B076FEA23
:104800000101116107D5202383F31188FFF7FCFA1A
:10481000002383F3118808BD000C0040384B4FF093
:10482000FF31D3F88020C3F88010D3F88020002215
:10483000C3F88020D3F88000D3F88400C3F8841034
:10484000D3F88400C3F88420D3F88400D86F40F0F4
:10485000FF4040F4FF0040F43F5040F03F00D86775
:10486000D86F20F0FF4020F4FF0020F43F5020F0EC
:104870003F00D867D86FD3F888006FEA40506FEADE
:104880005050C3F88800D3F88800C0F30A00C3F87A
:104890008800D3F88800D3F89000C3F89010D3F8BC
:1048A0009000C3F89020D3F89000D3F89400C3F898
:1048B0009410D3F89400C3F89420D3F89400D3F85C
:1048C0009800C3F89810D3F89800C3F89820D3F84C
:1048D0009800D3F88C00C3F88C10D3F88C00C3F880
:1048E0008C20D3F88C00D3F89C00C3F89C10D3F82C
:1048F0009C10C3F89C20D3F89C3000F0C9B900BFCD
:1049000000440258614B0122C3F80821604BD3F8E0
:10491000F42042F00202C3F8F420D3F81C2142F044
:104920000202C3F81C210422D3F81C31594BDA606F
:104930005A689104FCD5584A1A6001229A60574A75
:10494000DA6000221A614FF440429A61514B9A6931
:104950009204FCD51A6842F480721A604C4B1A6FAC
:1049600012F4407F04D04FF480321A6700221A6795
:104970001A6842F001021A60454B1A685007FCD5CC
:1049800000221A611A6912F03802FBD10121196064
:104990004FF0804159605A67414ADA62414A1A61D0
:1049A0001A6842F480321A60394B1A689103FCD5B8
:1049B0001A6842F480521A601A689204FCD53A4A86
:1049C0003A499A6200225A6319633949DA63996352
:1049D0005A64384A1A64384ADA621A6842F0A852AD
:1049E0001A602B4B1A6802F02852B2F1285FF9D1F5
:1049F00048229A614FF48862DA6140221A622F4A93
:104A0000DA644FF080521A652D4A5A652D4A9A652C
:104A100032232D4A1360136803F00F03022BFAD1DF
:104A20001B4B1A6942F003021A611A6902F038023C
:104A3000182AFAD1D3F8DC2042F00052C3F8DC2067
:104A4000D3F8042142F00052C3F80421D3F8042122
:104A5000D3F8DC2042F08042C3F8DC20D3F80421F4
:104A600042F08042C3F80421D3F80421D3F8DC20BB
:104A700042F00042C3F8DC20D3F8042142F00042A7
:104A8000C3F80421D3F80431704700BF00800051FF
:104A9000004402580048025800C000F00400000121
:104AA0000000FF01008890083220600063020901C5
:104AB0001D02040047040508FD0BFF012000002033
:104AC0000010E00000010100002000524FF0B04251
:104AD00008B5D2F8883003F00103C2F8883023B15A
:104AE000044A13680BB150689847BDE80840FFF7C7
:104AF00065B800BF305F00204FF0B04208B5D2F873
:104B0000883003F00203C2F8883023B1044A936866
:104B10000BB1D0689847BDE80840FFF74FB800BF19
:104B2000305F00204FF0B04208B5D2F8883003F073
:104B30000403C2F8883023B1044A13690BB15069E9
:104B40009847BDE80840FFF739B800BF305F002044
:104B50004FF0B04208B5D2F8883003F00803C2F82D
:104B6000883023B1044A93690BB1D0699847BDE8F6
:104B70000840FFF723B800BF305F00204FF0B0427D
:104B800008B5D2F8883003F01003C2F8883023B19A
:104B9000044A136A0BB1506A9847BDE80840FFF712
:104BA0000DB800BF305F00204FF0B04310B5D3F810
:104BB000884004F47872C3F88820A30604D5124A0A
:104BC000936A0BB1D06A9847600604D50E4A136BFE
:104BD0000BB1506B9847210604D50B4A936B0BB170
:104BE000D06B9847E20504D5074A136C0BB1506CA3
:104BF0009847A30504D5044A936C0BB1D06C984731
:104C0000BDE81040FEF7DABF305F00204FF0B04340
:104C100010B5D3F8884004F47C42C3F888206205BC
:104C200004D5164A136D0BB1506D9847230504D572
:104C3000124A936D0BB1D06D9847E00404D50F4A2A
:104C4000136E0BB1506E9847A10404D50B4A936EB6
:104C50000BB1D06E9847620404D5084A136F0BB1AC
:104C6000506F9847230404D5044A936F0BB1D06F5B
:104C70009847BDE81040FEF7A1BF00BF305F00209D
:104C800008B5FFF7B5FDBDE80840FEF797BF000087
:104C9000062108B50846FEF7BBFF06210720FEF7F0
:104CA000B7FF06210820FEF7B3FF06210920FEF713
:104CB000AFFF06210A20FEF7ABFF06211720FEF703
:104CC000A7FF06212820FEF7A3FF09217A20FEF77F
:104CD0009FFF07213220BDE80840FEF799BF000082
:104CE00008B5FFF79BFD00F007F8FFF755FDBDE89D
:104CF0000840FFF779BC00000023054A194601333C
:104D0000102BC2E9001102F10802F8D1704700BF70
:104D1000305F00200B460146184600F003B8000043
:104D200000F00EB810B5054C13462CB10A460146EA
:104D30000220AFF3008010BD2046FCE70000000019
:104D4000024B0146186800F035B800BF1C22002055
:104D500010B501390244904201D1002005E00378EA
:104D600011F8014FA34201D0181B10BD0130F2E72A
:104D70002DE9F041A3B1C91A17780144044603F1A3
:104D8000FF3C8C42204601D9002009E00578BD4255
:104D900004F10104F5D10CEB0405D618A54201D1AC
:104DA000BDE8F08115F8018D16F801EDF045F5D05C
:104DB000E7E7000037B5002944D051F8043C0190E2
:104DC000002BA1F10404B8BFE41800F047F81E4A14
:104DD0000198136833B96360146003B0BDE83040D4
:104DE00000F042B8A34208D9256861198B4201BF7F
:104DF00019685B6849192160EDE71A465B680BB1D9
:104E0000A342FAD911685518A5420BD12468214450
:104E10005418A3421160E0D11C685B6853602144C0
:104E20001160DAE702D90C230360D6E7256861191F
:104E30008B4204BF19685B68636004BF4919216035
:104E40005460CAE703B030BDB05F0020034611F8DC
:104E5000012B03F8012B002AF9D17047014800F01B
:104E600009B800BFB45F0020014800F005B800BFDA
:104E7000B45F00207047000070470000636F6D2E24
:104E80006375626570696C6F742E68657265340055
:104E90004E6F20617070207369670A004261642060
:104EA0006677206C656E6774682025750A0042611C
:104EB0006420626F6172645F696420257520736885
:104EC0006F756C642062652025750A00426164205C
:104ED00066772064657363726970746F72206C65A5
:104EE0006E6774682025750A0042616420617070E5
:104EF00020435243203078253038783A30782530B6
:104F00003878203078253038783A3078253038783D
:104F10000A00476F6F64206669726D776172650A77
:104F20000040A2E4F16468910600000043414E464F
:104F30004449666163653A204D6573736167652016
:104F400052414D204F766572666C6F7721000000EC
:104F50004261642043414E496661636520696E6425
:104F600065782E00000100000001FF0000A0004055
:104F700000A400400000000000000000851D0008A3
:104F80005D160008C524000855160008CD16000857
:104F9000DD1A000845180008951600089916000843
:104FA00071160008591600089D1A00087D160008A1
:104FB000D125000889160008711A000841A3E5F2FE
:104FC00065699207000000006D61696E00000000D5
:104FD00069646C6500000000D04F0008A05D0020EF
:104FE000185F002001000000AD3D00080000000037
:104FF000000000200000020002000000000100305C
:105000000000000000000000000000240000080074
:10501000040000000004000000FC0000020000008A
:105020000000043000800000000000000000003894
:105030000000010001000000000000280000000046
:10504000AAAAAAAA00000024FFFF00000000000096
:10505000000000000000550A00000000AAAA9AAA59
:1050600000000000FFF200000000000000009900B6
:105070000000000000000000AAAAAAAA0000000088
:10508000FFFF000000000000000000005A000000C8
:10509000000000009AAAAAAA00000000F3FF000086
:1050A0009900000000000000000000000000000067
:1050B000AAAAAAAA00000000FFFF0000000000004A
:1050C000000000000000000000000000AAAAAAAA38
:1050D00000000000FFFF00000000000000000000D2
:1050E0000000000000000000AAAAAAAA0000000018
:1050F000FFFF0000000000000000000000000000B2
:1051000000000000AAAAAAAA00000000FFFF0000F9
:10511000000000000000000000000000000000008F
:10512000AAAAAAAA00000000FFFF000000000000D9
:10513000000000000000000000000000AAAAAAAAC7
:1051400000000000FFFF0000000000000000000061
:105150000000000000000000AAAAAAAA00000000A7
:10516000FFFF0000000000000000000074B1FF7F9E
:105170000100000000000000130400000000000017
:10518000000018000000000001000000FE2A0100DD
:10519000D2040000202200200000000000000000D7
:1051A00000000000000000000000000000000000FF
:1051B00000000000000000000000000000000000EF
:1051C00000000000000000000000000000000000DF
:1051D00000000000000000000000000000000000CF
:1051E00000000000000000000000000000000000BF
:1051F0000000000000000000FFFFFFFFFFFFFFFFB7
:10520000FFFFFFFFFFFFFFFFFFFFFFFFFFFFFFFFAE
:10521000FFFFFFFFFFFFFFFFFFFFFFFFFFFFFFFF9E
:10522000FFFFFFFFFFFFFFFFFFFFFFFFFFFFFFFF8E
:10523000FFFFFFFFFFFFFFFFFFFFFFFFFFFFFFFF7E
:020000040803EF
:020000040804EE
:1000000000070030610D04087D110608150304087F
:1000100005110608FD10060801110608630D040805
:10002000630D0408630D0408630D0408059B0708AD
:10003000630D0408630D0408630D0408630D0408D0
:10004000630D0408630D0408630D0408630D0408C0
:10005000630D0408630D0408C1D60708EDD6070830
:1000600019D7070845D7070871D7070889A00708D7
:10007000B1A00708DDA0070809A1070835A10708F6
:100080005DA1070889A10708630D0408A1E505081B
:10009000C9E50508B5E50508DDE505089DD70708AC
:1000A000630D0408630D0408630D0408630D040860
:1000B000630D0408630D0408EDD80708630D0408F8
:1000C000630D0408E1400408630D040861A70708F4
:1000D000630D040875D8070889D80708630D04085C
:1000E00001D80708630D0408630D0408630D0408B4
:1000F000630D0408630D0408630D0408B5A1070827
:10010000630D0408630D040801D9070875A70708E3
:100110009DD80708630D0408630D0408630D0408E7
:10012000E1A1070809A2070835A2070861A207088C
:100130008DA20708630D0408630D0408630D04080D
:10014000630D0408630D0408630D0408630D0408BF
:10015000B5A20708E1A207080DA30708B1D8070850
:10016000630D0408630D0408630D0408630D04089F
:10017000630D0408630D0408630D0408630D04088F
:10018000630D0408630D0408C5D80708D9D807080B
:10019000630D0408630D0408630D0408630D04086F
:1001A000630D0408630D0408630D0408630D04085F
:1001B000630D0408630D0408630D0408630D04084F
:1001C000630D0408630D0408630D0408630D04083F
:1001D000630D0408630D0408630D0408630D04082F
:1001E000630D0408630D0408630D0408630D04081F
:1001F000630D0408630D0408630D0408630D04080F
:10020000630D0408630D0408630D0408630D0408FE
:10021000630D0408630D0408630D0408630D0408EE
:10022000630D0408630D0408630D0408630D0408DE
:10023000630D0408630D0408630D0408630D0408CE
:10024000630D0408630D0408630D0408630D0408BE
:10025000630D0408630D0408630D0408630D0408AE
:10026000630D0408630D0408630D0408630D04089E
:10027000630D0408630D0408630D0408630D04088E
:10028000630D0408630D0408630D0408630D04087E
:10029000630D0408630D0408630D0408630D04086E
:1002A000A5200408F93D04081D61040865660408DA
:1002B00015ED0408A12B0508FD4F0508A5570508F5
:1002C000015B050819C00508F1E5050819EC0508EA
:1002D0006D0C060825F60608090F07082D2A0708E1
:1002E000B554070895590708CD70070800000000AD
:1002F00040A2E4F164689106BFD9DE0FADA7FA1DF4
:10030000ACD60600BF08A03D00001304FFFFFFFFAE
:10031000FFFFFFFFEFF30383EFF30982EFF30881A1
:10032000DFF814D02DE9FE4F684600F097FFBDE8D6
:10033000FE4F8D46704700008C2A0030F1EE101AF7
:10034000A0EC200A01607047A0EC108A704700BF43
:1003500081F0004102E000BF83F0004330B54FEA76
:1003600041044FEA430594EA050F08BF90EA020FE3
:100370001FBF54EA000C55EA020C7FEA645C7FEA76
:10038000655C00F0E2804FEA5454D4EB5555B8BF99
:100390006D420CDD2C4480EA020281EA030382EA0A
:1003A000000083EA010180EA020281EA0303362D9C
:1003B00088BF30BD11F0004F4FEA01314FF4801C6F
:1003C0004CEA113102D0404261EB410113F0004F81
:1003D0004FEA03334CEA133302D0524263EB430338
:1003E00094EA050F00F0A780A4F10104D5F1200ED6
:1003F0000DDB02FA0EFC22FA05F2801841F1000131
:1004000003FA0EF2801843FA05F359410EE0A5F104
:1004100020050EF1200E012A03FA0EFC28BF4CF035
:10042000020C43FA05F3C01851EBE37101F00045EB
:1004300007D54FF0000EDCF1000C7EEB00006EEBF8
:100440000101B1F5801F1BD3B1F5001F0CD3490882
:100450005FEA30004FEA3C0C04F101044FEA4452D9
:1004600012F5800F80F09A80BCF1004F08BF5FEA60
:10047000500C50F1000041EB045141EA050130BD40
:100480005FEA4C0C404141EB0101013C28BFB1F552
:10049000801FE9D291F0000F04BF01460020B1FA9D
:1004A00081F308BF2033A3F10B03B3F120020CDA70
:1004B0000C3208DD02F1140CC2F10C0201FA0CF04E
:1004C00021FA02F10CE002F11402D8BFC2F1200CB3
:1004D00001FA02F120FA0CFCDCBF41EA0C01904069
:1004E000E41AA2BF01EB0451294330BD6FEA0404B2
:1004F0001F3C1CDA0C340EDC04F11404C4F120029D
:1005000020FA04F001FA02F340EA030021FA04F3AE
:1005100045EA030130BDC4F10C04C4F1200220FA05
:1005200002F001FA04F340EA0300294630BD21FA43
:1005300004F0294630BD94F0000F83F4801306BF09
:1005400081F480110134013D4EE77FEA645C18BFFD
:100550007FEA655C29D094EA050F08BF90EA020F94
:1005600005D054EA000C04BF1946104630BD91EA8C
:10057000030F1EBF0021002030BD5FEA545C05D18F
:100580004000494128BF41F0004130BD14F58004CE
:100590003CBF01F5801130BD01F0004545F0FE4142
:1005A00041F470014FF0000030BD7FEA645C1ABF77
:1005B000194610467FEA655C1CBF0B46024650EAAE
:1005C000013406BF52EA033591EA030F41F40021DA
:1005D00030BD00BF90F0000F04BF0021704730B560
:1005E0004FF4806404F132044FF000054FF0000135
:1005F00050E700BF90F0000F04BF0021704730B5F6
:100600004FF4806404F1320410F0004548BF4042CA
:100610004FF000013EE700BF42004FEAE2014FEA1F
:1006200031014FEA02701FBF12F07F4393F07F4FFA
:1006300081F06051704732F07F4208BF704793F0FD
:100640007F4F04BF41F40021704730B54FF4607410
:1006500001F0004521F000411CE700BF50EA010213
:1006600008BF704730B54FF000050AE050EA0102BC
:1006700008BF704730B511F0004502D5404261EB2C
:1006800041014FF4806404F132045FEA915C3FF46D
:10069000D8AE4FF003025FEADC0C18BF03325FEA0A
:1006A000DC0C18BF033202EBDC02C2F1200300FABB
:1006B00003FC20FA02F001FA03FE40EA0E0021FAE0
:1006C00002F11444BDE600BF80F0004002E000BF2C
:1006D00081F0004142001FBF5FEA410392EA030F2D
:1006E0007FEA226C7FEA236C6AD04FEA1262D2EB77
:1006F0001363C1BFD218414048404140B8BF5B427C
:10070000192B88BF704710F0004F40F4000020F014
:100710007F4018BF404211F0004F41F4000121F02A
:100720007F4118BF494292EA030F3FD0A2F1010274
:1007300041FA03FC10EB0C00C3F1200301FA03F1B2
:1007400000F0004302D5494260EB4000B0F5000FD5
:1007500013D3B0F1807F06D340084FEA310102F194
:100760000102FE2A51D2B1F1004F40EBC25008BF46
:1007700020F0010040EA03007047490040EB000010
:10078000013A28BFB0F5000FEDD2B0FA80FCACF111
:10079000080CB2EB0C0200FA0CF0AABF00EBC2503E
:1007A00052421843BCBFD0401843704792F0000F2C
:1007B00081F4000106BF80F400000132013BB5E77F
:1007C0004FEA41037FEA226C18BF7FEA236C21D0F5
:1007D00092EA030F04D092F0000F08BF084670475A
:1007E00090EA010F1CBF0020704712F07F4F04D128
:1007F000400028BF40F00040704712F100723CBF3B
:1008000000F50000704700F0004343F0FE4040F464
:10081000000070477FEA226216BF08467FEA236322
:100820000146420206BF5FEA412390EA010F40F40D
:10083000800070474FF0000304E000BF10F0004359
:1008400048BF40425FEA000C08BF704743F0964340
:1008500001464FF000001CE050EA010208BF70475B
:100860004FF000030AE000BF50EA010208BF7047E2
:1008700011F0004302D5404261EB41015FEA010CF7
:1008800002BF84460146002043F0B64308BFA3F1EF
:100890008053A3F50003BCFA8CF2083AA3EBC253D1
:1008A00010DB01FA02FC634400FA02FCC2F12002F0
:1008B000BCF1004F20FA02F243EB020008BF20F027
:1008C0000100704702F1200201FA02FCC2F120028D
:1008D00050EA4C0021FA02F243EB020008BF20EA82
:1008E000DC7070477BB972B90029BEBF00204FF0A1
:1008F000004106E008BF00281CBF6FF000414FF028
:10090000FF3000F02BBAADF1080C6DE904CE0029E0
:1009100009DB002B1ADB00F0B9F8DDF804E0DDE9B3
:10092000022304B07047404261EB4101002B1BDB06
:1009300000F0ACF8DDF804E0DDE9022304B0404249
:1009400061EB4101524263EB43037047524263EB58
:10095000430300F09BF8DDF804E0DDE9022304B076
:10096000404261EB41017047524263EB430300F0A8
:100970008DF8DDF804E0DDE9022304B0524263EBB8
:100980004303704753B94AB9002908BF00281CBF68
:100990004FF0FF314FF0FF3000F0E0B9ADF1080C3F
:1009A0006DE904CE00F072F8DDF804E0DDE9022321
:1009B00004B07047430803F05533C01A830803F0AE
:1009C000333300F03330184400EB101000F00F30D8
:1009D00000EB002000EB0040000E704708B5024617
:1009E0000B4643EC172BB5EEC07BF1EE10FA03D4A7
:1009F000BDE8084000F02AB8B1EE477B51EC170B78
:100A000000F024F8404261EB410108BD9FED0B6B03
:100A100007EE900A9FED0B5BB7EEE77A27EE066BC9
:100A2000BCEEC66BB8EE464BA4EE457BFCEEC77B36
:100A300016EE101A17EE900A704700BF0000000073
:100A40000000F03D000000000000F0419FED0B6B46
:100A500041EC170B9FED0B5B27EE066BBCEEC66BF4
:100A6000B8EE464BA4EE457BFCEEC77B16EE101AA3
:100A700017EE900A704700BFAFF30080000000003F
:100A80000000F03D000000000000F0412DE9F047BB
:100A9000089D04468E46002B4DD18A42944669D962
:100AA000B2FA82F252B101FA02F3C2F1200120FA45
:100AB00001F10CFA02FC41EA030E94404FEA1C4893
:100AC000210CBEFBF8F61FFA8CF708FB16E341EA8F
:100AD000034306FB07F199420AD91CEB030306F115
:100AE000FF3080F01F81994240F21C81023E634436
:100AF0005B1AA4B2B3FBF8F008FB103344EA0344DA
:100B000000FB07F7A7420AD91CEB040400F1FF33EE
:100B100080F00A81A74240F207816444023840EA2B
:100B20000640E41B00261DB1D4400023C5E9004364
:100B30003146BDE8F0878B4209D9002D00F0EF80E7
:100B40000026C5E9000130463146BDE8F087B3FA1A
:100B500083F6002E4AD18B4202D3824200F2F98002
:100B6000841A61EB030301209E46002DE0D0C5E905
:100B7000004EDDE702B9FFDEB2FA82F2002A40F051
:100B80009280A1EB0C014FEA1C471FFA8CFE012654
:100B9000200CB1FBF7F307FB131140EA01410EFBF8
:100BA00003F0884208D91CEB010103F1FF3802D29F
:100BB000884200F2CB804346091AA4B2B1FBF7F099
:100BC00007FB101144EA01440EFB00FEA64508D9BC
:100BD0001CEB040400F1FF3102D2A64500F2BB80F9
:100BE0000846A4EB0E0440EA03409CE7C6F1200748
:100BF000B34022FA07FC4CEA030C20FA07F401FA8E
:100C000006F31C43F9404FEA1C4900FA06F3B1FB16
:100C1000F9F8200C1FFA8CFE09FB181140EA01417B
:100C200008FB0EF0884202FA06F20BD91CEB010118
:100C300008F1FF3A80F08880884240F28580A8F170
:100C400002086144091AA4B2B1FBF9F009FB1011C2
:100C500044EA014100FB0EFE8E4508D91CEB010160
:100C600000F1FF346CD28E456AD90238614440EA03
:100C70000840A0FB0294A1EB0E01A142C846A64683
:100C800056D353D05DB1B3EB080261EB0E0101FA0C
:100C900007F722FA06F3F1401F43C5E90071002669
:100CA0003146BDE8F087C2F12003D8400CFA02FCBF
:100CB00021FA03F3914001434FEA1C471FFA8CFECF
:100CC000B3FBF7F007FB10360B0C43EA064300FBBF
:100CD0000EF69E4204FA02F408D91CEB030300F15D
:100CE000FF382FD29E422DD9023863449B1B89B214
:100CF000B3FBF7F607FB163341EA034106FB0EF39D
:100D00008B4208D91CEB010106F1FF3816D28B4249
:100D100014D9023E6144C91A46EA004638E72E4615
:100D2000284605E70646E3E61846F8E64B45A9D20D
:100D3000B9EB020864EB0C0E0138A3E74646EAE77C
:100D4000204694E74046D1E7D0467BE7023B61442A
:100D500032E7304609E76444023842E7704700BF93
:100D600002E000F000F8FEE772B63A4880F3088827
:100D7000394880F3098839484EF60851CEF200010F
:100D8000086040F20000CCF200004EF63471CEF262
:100D900000010860BFF34F8FBFF36F8F40F2000078
:100DA000C0F2F0004EF68851CEF200010860BFF3A9
:100DB0004F8FBFF36F8F4FF00000E1EE100A4EF639
:100DC0003C71CEF200010860062080F31488BFF366
:100DD0006F8F3CF09FF93CF041F93CF025FA4FF061
:100DE00055301F491B4A91423CBF41F8040BFAE7BA
:100DF0001C49194A91423CBF41F8040BFAE71A49D1
:100E00001A4A1B4B9A423EBF51F8040B42F8040B9E
:100E1000F8E700201749184A91423CBF41F8040BFB
:100E2000FAE73CF059F93CF083FA144C144DAC420B
:100E300003DA54F8041B8847F9E701F023F9114C51
:100E4000114DAC4203DA54F8041B8847F9E73CF033
:100E500041B9000000070030002300300000040802
:100E6000000100300007003018D10A0800230030CC
:100E7000942800309828003000260130A002040891
:100E8000EC020408EC020408EC0204082DE9F04F1F
:100E90002DED108AC1F80CD0D0F80CD0BDEC108A22
:100EA000BDE8F08F002383F311882846A047002077
:100EB0003BF0FEF9FEE73BF0B5F800DFFEE700008F
:100EC00070B54FF0FF0C4CF4E06C1CEA11541DBFE0
:100ED0001CEA135594EA0C0F95EA0C0F00F0DEF8AB
:100EE0002C4481EA030621EA4C5123EA4C5350EA90
:100EF000013518BF52EA033541F4801143F48013E1
:100F000038D0A0FB02CE4FF00005E1FB02E506F071
:100F10000042E0FB03E54FF00006E1FB03569CF0C6
:100F2000000F18BF4EF0010EA4F1FF04B6F5007FCC
:100F300064F5407404D25FEA4E0E6D4146EB06063E
:100F400042EAC62141EA55514FEAC52040EA5E50C7
:100F50004FEACE2EB4F1FD0C88BFBCF5E06F1ED871
:100F6000BEF1004F08BF5FEA500E50F1000041EBA8
:100F7000045170BD06F0004646EA010140EA020055
:100F800081EA0301B4EB5C04C2BFD4EB0C0541EA77
:100F9000045170BD41F480114FF0000E013C00F38C
:100FA000AB8014F1360FDEBF002001F0004170BDB0
:100FB000C4F10004203C35DA0C341BDC04F11404C9
:100FC000C4F1200500FA05F320FA04F001FA05F255
:100FD00040EA020001F0004221F0004110EBD37022
:100FE00021FA04F642EB06015EEA430E08BF20EA4E
:100FF000D37070BDC4F10C04C4F1200500FA04F3F1
:1010000020FA05F001FA04F240EA020001F0004182
:1010100010EBD37041F100015EEA430E08BF20EAF5
:10102000D37070BDC4F1200500FA05F24EEA020E3D
:1010300020FA04F301FA05F243EA020321FA04F06C
:1010400001F0004121FA04F220EA020000EBD37023
:101050005EEA430E08BF20EAD37070BD94F0000F23
:101060000FD101F00046400041EB010111F4801F57
:1010700008BF013CF7D041EA060195F0000F18BF08
:10108000704703F00046520043EB030313F4801F44
:1010900008BF013DF7D043EA0603704794EA0C0FFE
:1010A0000CEA135518BF95EA0C0F0CD050EA410614
:1010B00018BF52EA4306D1D181EA030101F0004191
:1010C0004FF0000070BD50EA410606BF10461946B9
:1010D00052EA430619D094EA0C0F02D150EA0136C5
:1010E00013D195EA0C0F05D152EA03361CBF104606
:1010F00019460AD181EA030101F0004141F0FE41A5
:1011000041F470014FF0000070BD41F0FE4141F428
:10111000780170BD4FEA410212F5001215D211D5C7
:101120006FF47873B3EB625212D94FEAC12343F0E4
:10113000004343EA505311F0004F23FA02F018BF66
:10114000404270474FF00000704750EA013005D12F
:1011500011F0004008BF6FF0004070474FF00000F2
:10116000704700BF4FEA4102B2F1E04324BFB3F53C
:10117000001CDCF1FE5C0DD901F0004C4FEAC0020E
:101180004CEA5070B2F1004F40EB830008BF20F0F2
:101190000100704711F0804F21D113F13872BCBFAC
:1011A00001F00040704741F480114FEA5252C2F101
:1011B0001802C2F1200C10FA0CF320FA02F018BF4A
:1011C00040F001004FEAC1234FEAD32303FA0CFC9D
:1011D00040EA0C0023FA02F34FEA4303CCE77FEA2C
:1011E000625307D150EA01331EBF4FF0FE4040F476
:1011F0004000704701F0004040F0FE4040F4000025
:10120000704700BF10F8012B11F8013B012A28BFDD
:101210009A42F7D0D01A7047034613F8012B002AE0
:10122000FBD1181A0138704710B5044620461CB18E
:1012300054F80C3B013300D110BD0822012100F00D
:1012400069FB54F80C0C54F8082C14F8041C121AFE
:10125000B2FBF1F200F05EFBE8E70000C26AD0E901
:10126000003112F0040F2DE9F04118BF0B46A6B073
:101270000021594C042601270291CDE90003D00634
:101280004CBF03F1200203F168020392DA6903996B
:10129000D2099B6902F004021B880A4303F47F43CE
:1012A00003924FF0E022A3F53E41D2F8882D02F4DC
:1012B000A002B2F5A00F04BF012202924B424B41A3
:1012C0000493464D03A82C6000F022FA0422012169
:1012D000434800F01FFB0422012102A800F01AFB82
:1012E00010220121019800F015FB00982022012115
:1012F0000C3000F00FFB019804220121103000F0A7
:1013000009FB0422012103A800F004FB01980C2230
:101310000121143000F0FEFA0C220121009800F0A7
:10132000F9FA029BDA071FD5009BDB6ADB064ED475
:1013300015A8FFF709F8DDF804C00DF1140E0CF143
:1013400020030CF160081868083353F8041C724637
:10135000434503C29646F6D1DCF8603025938422DB
:10136000012105A800F0D6FA00F0C0F8FFF75CFFF5
:101370004FF0E023D3F8003D03F47023B3F5402F82
:101380000ED0184B05A88DF81C60059314338DF80A
:10139000287006934FF0FF33CDE90833FFF744FF81
:1013A0002B68A34206D0104B0422012105A8059307
:1013B00000F0B0FA00F022FA002882D0049B1BB1A2
:1013C000019A93690233936126B0BDE8F08105A8C4
:1013D000FEF7B4FFC3E700BFED55CEAC9828003050
:1013E0005838080828ED00E0ACCE55ED08B52520AA
:1013F00039F0B0FF144BD3F8982042F01002C3F834
:101400009820D3F8982022F01002C3F89820D3F83F
:101410009820D3F8F02042F01002C3F8F020D3F85F
:10142000182142F01002C3F818216D22D3F81831A8
:10143000064BDA604FF0FF321A620D221A60012269
:10144000034B1A7008BD00BF004402580010014051
:10145000C42A003037B50E4D2A78202A15D10D4CFC
:101460000D4823680D49184401923BF075F9236833
:101470000021019A20330948297023603EF06EFF55
:1014800003B0BDE830403BF0B3BD03B030BD00BF9A
:101490008C2A0030B42A0030C0D60A088E2A0030C8
:1014A000014B1868704700BFFCFF1708014B02484A
:1014B000C01A7047C0D60A080000180800487047D4
:1014C000C0D60A0807490022074B5B1A9A4201D38B
:1014D0000120704751F8040B013001D10432F5E7C7
:1014E00000207047C0D60A08000018085A4B2DE9A2
:1014F000F74F1F680224594B07F56A57DFF88091B0
:101500001B781837DFF87C81554D1F44DFF878A130
:101510003AF07AFCA9EB080B06460EB13A2C41D9F9
:10152000A9EB0803B3EB070C24D4DFF860E1661CD9
:101530004C4A0C21F6B2AEEB0200614360456FDD10
:10154000681801276A50624407721F464260DB1B1D
:1015500077D445490234454FE4B2CA1B9A424FF052
:101560000C0206FB02F266DDA91801203B44AF50D5
:1015700008724B603B2C66D80C2301225C432B196C
:101580001A724FF0FF322A515A60394B1B782BB137
:10159000384B1B682B60384B1B686B60304803B0BE
:1015A000BDE8F08FF369B06953450ABF334BF31AB6
:1015B000A3EB0A0380B101933BF0A0FA019B58B161
:1015C00022460C2101344A430121E4B2A8180172D9
:1015D000B169A9500D3141600C2001211F4400FB6D
:1015E00004FC5F4505EB0C0245F80C6006F1380C75
:1015F0001172C2F804C004EB010204F10204D2B279
:10160000E4B200FB02F205EB02000172F169A9509D
:1016100019444160AED230463AF006FC06467CE7FB
:1016200005EB010C4FF0010807446A508CF8088064
:10163000CCF804E08BE7AB180120AF50187259606A
:1016400098E7344696E7012385F8CC324FF0FF3314
:10165000C5E9B13399E700BFB42A00308C2A0030C5
:1016600004230030982800300000043000260130A8
:1016700000230030B82A0030B02A003000230030A8
:1016800000001808C0D60A08000700300026013004
:101690000C4B1B7810B50BB9FFF7A8FE00230A49C5
:1016A0000A48CA699206FCD54A6A1C5CD2B29442C6
:1016B00005D10133DBB20E2BF3D1002010BD002386
:1016C000EFE700BFC42A0030001001405C38080872
:1016D00038B5084B04461B780BB9FFF787FEE4B218
:1016E000054DAC62EB695B0600D538BD3BF080FC74
:1016F000F8E700BFC42A00300010014010B5441EB6
:1017000014F8010F00B910BDFFF7E2FFF8E7000081
:1017100070B502680446EFF30581D9205369C9B258
:101720001FF0F2FC294B1B78A3B1294B94E803006E
:1017300083E803002748FFF7E1FF6368B3B1264859
:10174000FFF7DCFF2548FFF7D9FFFFF7A1FF24488B
:10175000FFF7D4FF234D2B783BB124681CB1204602
:101760003BF0CCF920B900232B7070BD1E48E7E791
:1017700020461E4E3BF0D6F900F2145084421FD290
:1017800020463BF0CFF930602046194E3BF0DEF9A1
:1017900004F5E053834217D920463BF0D7F9306077
:1017A0000023144A1360144A1370FFF78BFE0028BD
:1017B000D9D03BF01DFC0120BDE870403BF048B89B
:1017C000A4F214533360DFE73360E9E78D2A003079
:1017D000BC2A00306C3808087138080882380808BC
:1017E000149B0808002300307C380808B82A003011
:1017F000B02A0030B42A00308C2A0030284B1A78E6
:1018000070B542B12748FFF779FF274B5868003879
:1018100018BF012070BD254A107800283CD0244E06
:10182000244C33682448254D1A1D21782D1A0A446A
:10183000AA4205D3224A4FF0FF31D1612022227003
:101840002278D2B103F120018D4205D81F2A9FBF13
:101850001B4AD361202222702022194918443AF0F1
:101860007BFF326823780021154813442022217021
:1018700033603EF073FD3BF0BBFB33689D4207D9FC
:101880000F4920220F48CB613AF066FF3BF0B0FBD6
:1018900000203AF0DDFFB8E701221A70BAE700BF76
:1018A0008D2A0030C8380808BC2A003000230030D8
:1018B000B42A00308C2A0030C0D60A08000018086C
:1018C0008E2A0030E0FF17082DE9F84307460E4640
:1018D0000024DFF83890DFF83880B44201D1BDE849
:1018E000F88324B1230702D14846FFF707FF3D5D87
:1018F00001342B0905F00F0518F80300FFF7E8FE87
:1019000018F80500FFF7E4FEE7E700BF149B08089E
:10191000D8380808474B1B782DE9F74F07460E4685
:1019200090465BB1022925D0042938D0012902D183
:101930001146FFF7C9FF4048FFF7E0FE3F4B1B7819
:10194000002B4ED03E4A00253E4BA2EB030938E067
:1019500037F81430ADF8043024B1620702D12846BC
:10196000FFF7CCFE0134022101A8FFF7ADFFA0452F
:10197000EED1E0E70024304DF9E757F82430019329
:1019800024B1A30702D12846FFF7B8FE0421013491
:101990000DEB0100FFF798FFA045EED1CBE7002447
:1019A000254DF9E7FFF756FD022E1DD0042E2CD051
:1019B000012E06D12378795D5A1C2270224AD15417
:1019C0000135A8450DD0214B214C1B6822780433EA
:1019D00013444B45E6D31C4B4FF0FF32DA61202312
:1019E000237003B0BDE8F08F2378DFF85CA05A1CA9
:1019F00022703A780AF80320FFF72CFD23785A1C4E
:101A0000227000220AF80320DAE74FF0000ADFF81C
:101A100038B022783B78511C23FA0AF30AF1080AFD
:101A200021700BF80230FFF715FDBAF1200FF0D14D
:101A3000C6E700BF8D2A0030149B08080023003041
:101A400000001808C0D60A088E2A0030B42A0030D8
:101A50008C2A0030054B10B50446C0F87C35D0F810
:101A6000200708B104F06CFB204610BD1C9D0A083D
:101A700070B504462C3011F039FF04F1500004F227
:101A80009C5505F017FFFF2304F5E67004F5C066CA
:101A900084F8C83104F056FB04F5397003F054FCA7
:101AA00004F582601AF0DEF904F264400DF04AF9A0
:101AB00004F598630120002143E90201002304F1A9
:101AC000180104F59A6084F8C8340AF0D5F82D4B53
:101AD000C4F87C352846143515F0CEFCB542F9D152
:101AE0001E2340F2CC60C4F824370023A4F8283722
:101AF00004F024FBC4F8200704F22C701CF0FEFD57
:101B000004F5EE601CF0FAFD1F4B1A6812B904F2DE
:101B10007C521A601D4B04F28C701D491826C4F8C3
:101B20007C351C4B196000239DB201332A46724359
:101B30008A5C002AF8D1184B1D80184B1A6812B124
:101B400017481FF01FFB186004F5F960154BC4F827
:101B5000BC371CF0D3FD144B64224FF4FA71C4F867
:101B6000E03704F2E47304F5FE60C4F8E43711F0E2
:101B700009FE0E4B1A680AB10D48E2E720461C60C8
:101B800070BD00BF1C9D0A0800510030486C080859
:101B9000906E08080C4900300A490030C4480030F3
:101BA000EC3808083CA10A0898A40A08C82A0030A2
:101BB00007390808082906D1084B09211B68586C09
:101BC00003681B6918470A2906D1044B07211B68C3
:101BD000586C03681B69F5E7704700BFF02A0030B6
:101BE000FFF7E8BF2DE9F0415F4D88B004463BF0B8
:101BF000EBF93BF0FDF9032128681AF0A3FD036817
:101C000080224FF4E131DE6A4FF48073B047204602
:101C100000F03EFC04F12C063BF0EAF9204601F00E
:101C200013FD3BF0E5F917F075FF12F0B7F93046F8
:101C300011F08CFF17F06EFF15F052FC17F06AFFE1
:101C400015F060FC17F066FF484A062112F0DAF939
:101C50003BF0CEF99B22464904F59A600AF09CFCC1
:101C6000444945484B6902930B6901934B7E0093AD
:101C70000B7ED1E902121CF0B7FD2B68586D03688A
:101C80005B68984710B13D481CF0AEFD94F95030A8
:101C900093B394F928307BBB0423314604F1500000
:101CA000E36705F053FE04F2BC7604F5FC613046B0
:101CB0001AF0A4FC012130461AF07AFC204602F00A
:101CC000A3F804F5E67004F093FB04F5397003F013
:101CD00099FE2B68D86C03681B6898472B68D86CF2
:101CE00003681B6D984704F264400DF05BF908B07F
:101CF000BDE8F0411FF082BA2B6800220821204F76
:101D0000586C032603685B6A98472B6801220721F9
:101D1000586C03685B6A98472B6800220A21586C4C
:101D200003685B6A98472B6801220921586C036895
:101D30005B6A98472B6822460821586C0494036814
:101D40000597D3F82C803B460096C0472B680A21A4
:101D5000586C0368D3F82C8008AB0096CDE9064791
:101D600013E90C00C0479EE7F02A00302839080824
:101D7000745D0808F0020408433908086A39080845
:101D8000E11B04080148FFF72DBF00BFF82A00300F
:101D9000F0B52DED028B90F8C8348BB0002B54D1E8
:101DA0002C4E1FF02BFA02463368C31A632B4CD912
:101DB000294B04AD03F118071868083353F8041CC5
:101DC0002C46BB4203C42546F6D10024234D9FED8B
:101DD000248A32602B780AAA2344013403F00703D3
:101DE00003EB4303134413F8162C07EE902A13F861
:101DF000172C13F8183CF8EEE77A67EE887AFCEEB9
:101E0000E77ACDED017A07EE902A9DF80420F8EEEE
:101E1000E77A67EE887AFCEEE77ACDED027A07EE94
:101E2000903A9DF808100023F8EEE77A67EE887A7A
:101E3000FCEEE77ACDED037A9DF80C000DF0F8F892
:101E4000042CC7D12B7801332B700BB0BDEC028B67
:101E5000F0BD00BFCC2A0030D8360808D02A0030A8
:101E60009A99993E2DE9F341144C154E2046DFF81E
:101E700060803AF0CDFF134A01461348121B134FFE
:101E800001F07AFD39F0C0FF0446A4B1E069A16910
:101E9000B042019114BF251AA8EB06053AF0B8FF2D
:101EA000019902462B46384601F066FD204639F07E
:101EB000BBFF0446E9E702B0BDE8F0810001003055
:101EC00000070030000700308839080892390808F8
:101ED0000023003008B590F8603463B1002380F827
:101EE000603419F0E3FF1AF059F819F007FEBDE865
:101EF00008401AF05BB808BD10B5094C0FF058FD4A
:101F0000002105222368186D0368DB699847236860
:101F10002821186D0368BDE810405B68184700BFB2
:101F2000F02A003073B504461FF068F94B4A0546A5
:101F30001368C31AB3F57A7F0CD9106019F0BCFE90
:101F400017F0E8FD002118F059FD17F0E3FD04211A
:101F500018F054FD09F06CFC414A41F288311368D5
:101F6000EB1A8B4206D9016821B1156002893D4800
:101F700001F002FD94F91130012B0AD13A4A41F2E5
:101F800088311368EB1A8B4203D920461560FFF79E
:101F900069FF364A1368EB1A132B0CD904F264401C
:101FA00015600DF013F817F0B5FD17F069FA17F08A
:101FB000B1FD19F053FB04F59A602D4D09F0CEFFE9
:101FC000204601F017FD94F8B8371BB32B7843B9BE
:101FD00094F928303BBB204602B0BDE87040FFF7C3
:101FE000D7BE244E64213368186D03681B69984777
:101FF00001230DF1070104F128008DF8073010F0DE
:1020000041FE2046FFF778FF33680021186D036812
:102010009B6B98472B78002BDAD094F92830002B53
:10202000D9D002B070BD134E002564213368186DFD
:1020300003681B6998470DF1070104F128008DF82A
:10204000075010F01FFE2046FFF756FF3368294661
:10205000186D03689B6B9847DFE700BFD42A0030F8
:10206000DC2A0030A4390808D82A0030E02A0030E1
:10207000D4250030F02A00300148FFF753BF00BFDD
:10208000F82A003038B5054B0A4601461C6823681B
:1020900020461D68024BA847002038BDF02A0030BA
:1020A000E42A003010B50A4C2046FFF7E1FC094A4B
:1020B000094920463BF082FC1CF09EFD074B084A74
:1020C000186008490848BDE810401AF033BB00BF4B
:1020D000F82A0030B8E10030551A0408F02A003020
:1020E00079200408851D0408E42A00300020704788
:1020F0007047000070470000704700007047000004
:102100000020704700207047002070470120704772
:102110007047000000207047002070470020704783
:102120000020704700207047002070470020704753
:102130007047000000207047C8207047012070479A
:102140000020704700207047704700000120704752
:102150000020704701207047704700000120704741
:102160000220704700207047002070477047000031
:10217000704700000020704703207047014B187F14
:10218000704700BFF82A00307047000013B54FF4C5
:102190003E70CDE9002103F0C7FF044660B1DDE9E0
:1021A000002118F093F8064B23604FF0FF33C4F87A
:1021B000F031002384F8F032204602B010BD00BF99
:1021C000886C080810B5044603F0B4FF204610BD23
:1021D00008B590F884308B4208D209F029FB5C22C4
:1021E0004FF4802109F010FB002008BD223150F887
:1021F0002100FAE708B590F884308B4208D209F044
:1022000017FB55224FF4802109F0FEFA002008BD8B
:10221000223150F82100FAE7F0B5CA78C5B004467B
:102220000026062A01F10C0102A8029628BF062208
:10223000ADF80C603EF06AF8029DD4F8E8319D429A
:1022400007D91F4801F098FB012384F8F03245B00C
:10225000F0BDD4F8F031002BF9DB04F5FA7704F087
:10226000FDF933462A46D4F8F01104F06DF904F074
:10227000F5F9FC233A46D4F8F01104F045F9ADF82D
:102280000E61FC2639460DF112003246B5FBF6F51B
:10229000ADF810503EF03AF8FF23DF22207C832176
:1022A000CDE9003204AA12F05FFDD4F8E821BDF8B0
:1022B00010100448B2FBF6F201F05EFBC7E700BF66
:1022C000646B0808806B08082DE9F043CA7897B062
:1022D00000230646092A884603A801F10C0128BFFD
:1022E00009228DF81430CDE903333EF00FF89DF844
:1022F0001030222B40F0828096F8F042002C7DD1E5
:10230000D6F8F031013363D104F0A8F92346224610
:102310003C4904F0C1F800280446C6F8F0013BDB54
:1023200006F5FA7904F09AF9FC234A46D6F8F0113A
:1023300004F0EAF8B0F1000C38DD334D06ACD6F805
:10234000EC710FCD0FC40FCD0FC40FCD0FC495E8A6
:102350000F0084E80F00FB434C4609EB0C0014F817
:10236000012B16AD82EA0301A04201F00F0105EB3B
:10237000810151F8401C81EA131383EA121202F022
:102380000F0205EB820252F8402C82EA1313E6D1C9
:10239000DB43C6F8EC31C5E73DF0D0FE21460268CC
:1023A0001A4817B0BDE8F04301F0E6BA04F056F958
:1023B0000023D6F8F0111A4604F0C6F804F04EF9DE
:1023C00002230022D6F8F01104F0BEF8C6F8E801A6
:1023D00098F8072098F808308DF82020F0228DF822
:1023E00021300A23D6E97A01CDE90032CDE9060190
:1023F00006AA4CF25431307C12F0B6FC17B0BDE89E
:10240000F08300BFA46B0808F0360808BA6B080810
:1024100030B5CD788FB00C463322332D4FF000010C
:1024200001A828BF33253DF099FF04F10C0101A854
:102430002A463DF06BFF01A9024801F0CFF80FB02A
:1024400030BD00BFF82A003038B58A7A05464B7A8D
:102450000C4643EA0223CA7A43EA024343F2762255
:10246000934210D04CF25532934208D00BB9FFF78B
:102470002BFF21462846BDE8384018F045BDBDE891
:102480003840FFF7C9BEBDE83840FFF7C1BF0000C4
:1024900013B504460FF0ECFE0EF0DAFF20460FF005
:1024A00061FE18B1B4F90030022B0BD019F0C0FD59
:1024B0000EF07EFC02230DF106012046ADF8063039
:1024C00010F00EFC02B0BDE8104010F015BB00008B
:1024D000BFF34F8F0549064BCA6802F4E06213430D
:1024E000CB60BFF34F8F00BFFDE700BF00ED00E002
:1024F0000400FA05102213B5002104468DF80720C8
:102500003DF02CFF054B0DF1070221461B68586D6D
:1025100003685B6B984702B010BD00BFF02A003023
:102520002DE9F041ADF54A7D0D46002140F27512CE
:1025300068AC06460AA809913DF010FF4FF4C4723A
:10254000002120463DF00AFFDFF808811EF056FE0C
:102550004FF47A72384B09AFB0FBF2F0186093E891
:10256000070084E8070003F03DFB037C237403F0BD
:1025700039FB437C0DF5E17063740323A3742F4B87
:102580005A6962619A68DB68A261E361FFF7B2FF92
:1025900041F20433D8F814202384002A284B186809
:1025A000284B3CDD0DF2D321CDE90032264B5022E1
:1025B000406D1AF0B7F950210DF2D3203EF06CFABD
:1025C00098F91E20394684F83201013A204618BF96
:1025D000012202F091FB98F91E3080B2E97E5A1E6A
:1025E0005342534107930723069300230393AB7E83
:1025F000029305F1190301930123CDE904700093BF
:1026000030460BA3D3E9002336F0E0FD011E02DCC7
:102610000E481CF0E9F80DF54A7DBDE8F081009305
:1026200050220B4B0DF2D321406D1AF07BF9C2E71B
:102630009E6AC421818A46EE0C330030F002040801
:10264000F02A00301F710808187108083371080853
:1026500085800808F82A00302DE9F04F334E97B0F6
:10266000DFF8D490304636F0FDFD0446002855D002
:102670000021402205A82E4F04914FF00108ADF82B
:1026800054103DF06BFE94F8440019F0FBFD211D41
:102690008DF8540005A894F844203DF037FE2368D7
:1026A000244D43F0004305F1100A049394F8473099
:1026B0008DF855301EF0A4FDC71941F1000368687C
:1026C000C0B12A7894F846101141C90712D54A447E
:1026D00092F80C24012A0DD1026800210393009185
:1026E00004A9D2F810B03A46D8470028039BD8BFB7
:1026F0004FF0000808355545E1D1B8F1000F06D07C
:10270000304636F0B3FD002386F8D13FAAE796F8AD
:10271000D13F072B05D8013386F8D13F17B0BDE86C
:10272000F08F024836F0A2FDF8E700BF1833003002
:1027300040420F00EC420030F82A00302DE9F04111
:10274000DC220C46CAB00546002144483DF006FE96
:102750004FF04053424A1A60A38A013B9BB2C92BF7
:1027600075D8404B002608222046009300231946C6
:1027700036F0C0FD721CF3B2D1001646A28A013AAF
:10278000934209DA03F1405308222046163300939E
:10279000002336F0AFFDEDE74FF040531A7D0AB944
:1027A000E27E1A752846002636F0B4FC4FF04053FE
:1027B00031467D22587509A8DFF8B08008AF089629
:1027C0003DF0CCFD3146812229A83DF0C7FD98F9A6
:1027D0001E20394629A8013A18BF012202F0E6FB63
:1027E00098F91E3080B203965A1E1F4E5342534131
:1027F00007930723CDE9047006932846A37E02932E
:1028000004F11903019328230093E17E332411A3DB
:10281000D3E9002336F0DAFC013C14F0FF0408D0C1
:10282000FFF71AFF33680121186D03685B6898474A
:10283000F2E70E48FFF760FB284636F06BFC40F0ED
:10284000304040F400203AF06FFAFFF741FE4AB002
:10285000BDE8F08126417272DF25D7B70400003051
:102860009AAD44C514000030F02A0030F82A003038
:102870002DE9F0410D46ADF5876D06463AF0B8FBFF
:102880000AA9284602F0ECFB0446002840F0AA8082
:102890004FF4D0720146A6A83DF060FD9DF8C0201F
:1028A000102A71D8531E0F2B1FD80DF1C1010DF244
:1028B000D9303DF02BFD22460DF127010DF2D93024
:1028C0000EF0ACFF0446002C5ED09DF8C0304BB338
:1028D0009DF8303033B39DF82720013A032A00F2E7
:1028E0008180DFE802F01628323B49AA0DF127016A
:1028F000BDF8280049940FF063FF0446002843D038
:1029000001230DF2D93249A9009311230EF0C6FE1E
:10291000D9E7012B66D10E9B49A920468DF82431B9
:1029200010F0CAF99DF82730013B032B5AD8DFE895
:1029300003F01C5D6368012B54D10E9B49A920460E
:10294000ADF8243110F0E6F9ECE7012B4AD10E9BEB
:1029500049A92046499310F02DFAE3E7022B41D113
:102960000EA9204610F070F9DCE701238DF89832AB
:1029700094F90030DA17CDE9A8325C210DF2D93094
:102980003EF08AF88DF8D8030024DFF88C8040F2FE
:102990006F124AA8214649943DF0E0FC98F91E20A8
:1029A00049AFA6A8013A394618BF012202F062FCDD
:1029B00098F91E3080B2E97E5A1E03945342534167
:1029C000079307230693AB7E029305F11903019346
:1029D0000B23CDE90470009330460DA3D3E9002307
:1029E00036F0F4FB0DF5876DBDE8F08101238DF81D
:1029F0009832B4F90030BDE701238DF8983223688E
:102A0000B8E702238DF898322368A893B5E700BF92
:102A1000D5A4D139F922B6A7F82A003007B508495C
:102A2000684637F039F8BDF8040064235843BDF810
:102A30000030B0FBF3F080B203B05DF804FB00BFE0
:102A40001833003070B50E4614461D4636F062FB52
:102A500050B9022D07D1012C05D144A3D3E900239D
:102A60000120C6E9002370BD40F239439C4261D089
:102A700034D80B2C28D854B90020F4E7A4F59C4096
:102A80003F38032862D8DFE800F05D69656D601E9D
:102A90000A28F1D801A353F820F000BF052B040841
:102AA000792A0408792A04083D2B0408152B040808
:102AB000792A0408792A0408792A0408792A04085A
:102AC000252B04081D2B0408282C1FD040F2264378
:102AD0009C42D1D127A3D3E90023C1E744F6426346
:102AE0009C42C9D844F63D639C42C7D840F24C434F
:102AF0009C421BD044F627639C42BDD11FA3D3E95F
:102B00000023ADE71FA3D3E90023A9E71FA3D3E95F
:102B10000023A5E71FA3D3E90023A1E71FA3D3E95F
:102B200000239DE71FA3D3E9002399E71FA3D3E95F
:102B3000002395E71FA3D3E9002391E71FA3D3E95F
:102B400000238DE71FA3D3E9002389E71FA3D3E95F
:102B5000002385E71FA3D3E9002381E71FA3D3E95F
:102B600000237DE71FA3D3E9002379E7401DA120BF
:102B700026812A0B011517CB0E03561FECFD5116AB
:102B80009C2A1F639E6AC421818A46EE2641727286
:102B9000DF25D7B7F017304A39059E56D5A4D1396D
:102BA000F922B6A7CDD269EBC51A133B03806A554B
:102BB00075F30087C41EDD8B3CD93120DBC293A79F
:102BC00016112720AA4CB1BCC5A2A3EA33C54F8E6B
:102BD0004A621C5B3724F39BF472C89A85A1064CA9
:102BE000DC81BE5935F93AF0C77F1E582DE9F04710
:102BF000DFF898A088B005460F465046164698461E
:102C000036F088FA28B3DAF8C84F45EA064934BBEB
:102C10000C21012039F0FAFECAF8C80FC8B184604F
:102C2000041DC0F80090184B184893F91E30009608
:102C30005A1E534253412A46069307230593BDF873
:102C40004030CDE903831823CDE901433B4636F0FC
:102C500063FA08B0BDE8F087A246A46824B12368EF
:102C60009945F9D10434DEE70C21012039F0CEFE7C
:102C7000CAF808000028ECD0C0F80090DAF8083054
:102C80009C60DAF80840EDE7F82A0030183300308D
:102C900000B5C5B0694601F0A3FAF0B9BDF800303F
:102CA000B3F5007F0E4B0FD1BDF802209FED0D7ADA
:102CB00007EE902AF8EE677A67EE877A9FED0A7A38
:102CC00067EE877AC3ED007ADDE9420143E902014C
:102CD0001EF08AFA054BC3F8C40445B05DF804FB46
:102CE000B82F00300AD7233C35FA8E3CF82A003042
:102CF0002DE9F0432DED028BBDB005460C4636F0B4
:102D000009FA8046002854D1237E022B1CD1E38A85
:102D1000012B19D11EF072FA07460AF001F803469A
:102D20004FF4C87007F51677A14EB3FBF0F202FB23
:102D3000103317FA83F3C6F8CC3FE77E4FB99D48AE
:102D40001BF052FD86F8D07F3DB0BDEC028BBDE894
:102D5000F0831AA9204602F0EDF80AA8FFF7CAFB93
:102D60009DF86A400AA90DF16B0022463DF0BEFABB
:102D700028B191481BF038FD86F8D08FE4E70F2C7E
:102D80000CD8D6F8CC2F21468C48A2F5167286F8BE
:102D9000D04FC6F8CC2F1BF027FDD5E79DF8681063
:102DA000284636F0AFF99DF8682096F8D21F84487F
:102DB000F1E7E38A40F23942934200F0158140D8AE
:102DC0000B2B29D8002BBFD0013B0A2BBCD801A26A
:102DD00052F823F0792E0408492D0408492D0408DF
:102DE000C73004089D2E0408492D0408492D040805
:102DF000492D0408492D0408CD2E0408BB2E0408D3
:102E0000A3F59C433F3B032B00F2C481DFE813F0A2
:102E10007C011A02E8013E02282B36D040F22642FD
:102E2000934291D11AA9204601F0B8FE014600282C
:102E30008AD19DF869300DF16A02624805F090F878
:102E400082E744F6426293423FF67EAF44F63D622B
:102E50009342D5D840F24C42934200F08E8044F623
:102E6000276293427FF470AF20463DB0BDEC028BE9
:102E7000BDE8F043FFF70CBF214628463DB0BDEC4E
:102E8000028BBDE8F043FFF74BBB214628463DB01F
:102E9000BDEC028BBDE8F043FFF750BC4A481BF085
:102EA000A3FC4A4B0A211B68186D03685B689847AE
:102EB0004748FFF721F8FFF70BFB214628463DB0B6
:102EC000BDEC028BBDE8F043FFF7D2BC0AA9204657
:102ED00002F098F800287FF437AF9DF82830012BD6
:102EE00013D119F0A5F80DF063FF0FF005FE0FF0F8
:102EF000BFF9384933480FF0E9F9374937480FF03F
:102F0000E5F9374937480FF0E1F9DFF8C4801022BE
:102F100000211AA83DF022FA012398F91E2008AFDB
:102F200000261AA8D21A39468DF8703018BF01222F
:102F30000896ADF824608DF8266002F07BF898F9C9
:102F40001E3080B2039603F1FF3CDCF1000343EB3B
:102F50000C0307930723CDE9047006932846A37E4C
:102F6000029304F1190301930A230093E17E0EA357
:102F7000D3E9002336F02AF9E6E61AA9204601F043
:102F8000ADFE00287FF4E0AE104B9DF868101B6882
:102F9000A1F1FF04586D6142036861411B689847C5
:102FA000D2E600BFAFF30080CDD269EBC51A133B68
:102FB000183300305C71080887710808A871080888
:102FC000DF710808482B0030FB710808F02A003038
:102FD000F82A00306C7A080804760808C42C0030FF
:102FE0002C740808DC2D0030DFF8EC8201231AA9CC
:102FF000204688F8C83401F035FE00287FF4A4AEDE
:10300000074608F26449DFEDB38A9DF86820FBB2F9
:103010009A427FF699AE3CAA484602EB830313F826
:10302000864C13F8855C13F8846CE400AD00F60060
:103030000CF04AF86428E4B205F0F805F6B237D08F
:10304000002835DB07EE900AFF220021B8EEE78A60
:1030500007EE904AF8EEE77A28EE288A67EE887A3B
:10306000FDEEE77A17EE903A18B209F051FE07EE3E
:10307000905AFF220021F8EEE77AC4B267EE887A10
:10308000FDEEE77A17EE903A18B209F041FE07EE2E
:10309000906AC5B2FF22F8EEE77A002127EE888A0F
:1030A000BDEEC88A18EE103A18B209F031FEC6B269
:1030B00000233246294620460BF0BAFF01231F4465
:1030C00088F86034A1E71AA9204601F0B9FE00286B
:1030D0007FF43AAE804DD5F8A02705F5F466736805
:1030E00052EA03010BD0DDE91A01CDE9000105F533
:1030F000FE6010F04BFB05F5F66343E90201D4E9ED
:103100000023C6E900231FE61AA9204601F02EF984
:103110003C2200210AA83DF021F914220DF1690199
:1031200012A802F04DFD9DF87D30FE210AAA8DF80F
:103130005C30BDF87E30ADF84030BDF88030ADF881
:103140004230BDF88230ADF84430219B0A93229B77
:103150000B93239B0C93249B0D939DF894308DF837
:103160005D30269B0E93BDF89C30ADF85E30BDF807
:103170009E30ADF86030289B0F939DF8A4308DF8F9
:1031800062303B23CDE9003143F26521022011F08A
:10319000EBFDD9E50AA9204601F086F82C23002191
:1031A0001AA81A463DF0DAF814220DF129010DF1A2
:1031B0006A0002F005FD9DF83D2010A920A88DF8B9
:1031C0007E209DF83E208DF87F20142202F0F8FC2E
:1031D00072222C2343F26421CDE900321AAAD5E7EA
:1031E0000AA9204601F03CFA382200211AA83DF035
:1031F000B5F814220DF129010DF1860002F0E0FC72
:103200009DF83D304D2243F268218DF89A309DF8AB
:103210003E308DF89B30109B1A93119B1B93129B91
:103220002093139B1C93149B1D93BDF85430ADF851
:103230009C30169B1E93179B1F933623CDE90032BB
:103240001AAAA3E70AA9204601F0B0F92E2300210B
:103250001AA81A463DF082F814220DF129010DF149
:103260006A0002F0ADFC9DF83D200DF13F010DF12B
:103270007F008DF87E20172202F0A2FCF9222E2377
:1032800043F26721CDE900321AAA7FE70AA9204656
:1032900001F032F92B2300211AA81A463DF05EF8FE
:1032A00014220DF129010DF16A0002F089FC9DF84C
:1032B0003D200DF13F010DF17F008DF87E2014229D
:1032C00002F07EFC31222B2343F26921CDE900324A
:1032D0001AAA5BE70AD7233CF82A0030F0B500F1C0
:1032E00050050446ADF5277D284605F071FA94F89F
:1032F0006061D4F8942704EB0613D3F89C309A420B
:1033000000F03481C4F894374FF4D07200213EA805
:103310003DF024F894F8C23133B9B02303FB0643DF
:1033200093F8A930012B0CD894F8E8774FB91DF029
:1033300063FF00220023CDE93E01CDE940230023B5
:1033400013E001233146284684F8E83704F062FB95
:10335000CDE93E0194F86011284604F0B7FB50EA2D
:103360000103CDE94001EAD002238DF80831B023F2
:103370000A2203FB064103FB0656D1F8C0008C3637
:1033800080FB0207CDE94407D1F8BC0080FB0207AF
:10339000CDE94607D1F8B8004243CDE94822D1F83B
:1033A000DC2094F860114A92726803FB01434B924F
:1033B000B2684C9293F8DA208DF8342193F8A92062
:1033C00094F8C23153B9062A0DD8DFE812F007008D
:1033D0000700D200D600D800DE00E30000238DF8FD
:1033E0003531ADF83631062303AA28468DF8383139
:1033F00004F0FCFA38B1DDED037A67EEA77ACDED83
:10340000507ACDED4F7A04AA94F86011284604F062
:10341000F7FA28B1DDED047A67EEA77ACDED517A9F
:1034200005AA94F86011284604F0D6FA48B1DDEDFB
:10343000057A67EEA77ACDED547ACDED537ACDEDCE
:10344000527A00265D4FDA2207A8314606963CF0F4
:1034500085FF97F91E2006A93EA8013A18BF012250
:1034600001F092FA06AB80B240F2274200904DA1E3
:10347000D1E90001FFF7BAFB202231463EA83CF01B
:103480006DFF94F86031B022DFED4D6A06A93EA8C9
:1034900002FB0343B3F8D620B3F8D83007EE102A66
:1034A00097F91E2007EE903AB8EEC77A013AF8EE87
:1034B000E77A18BF012227EE267A67EEA67A8DED0D
:1034C000407ACDED417ACDE90666CDE9086601F096
:1034D000E5F906AB80B240F22542009033A1D1E974
:1034E0000001FFF783FB94F8601128464096CDE970
:1034F0003E6604F047FE94F95E308DF8FC003BB167
:10350000284604F04FFE18B9409B43F00103409356
:103510009DF8FC3043B104A9284604F00DFD18B90C
:10352000409B43F00203409305AA94F8601128469B
:1035300004F048FE08B1059B3E9397F91E20002336
:1035400006A93EA8013A0693ADF81C3018BF012227
:103550008DF81E3000F028FE06AB80B244F62362E0
:10356000009014A1D1E90001FFF740FB0DF5277D84
:10357000F0BD02228DF8352133E70322FAE7032359
:103580008DF8353140F201132BE703238DF83531E7
:10359000022326E703238DF835314FF4817320E7AA
:1035A000AFF300805F43370F00E741CAD2BFDBC3F0
:1035B000C4BDE89B697F00BBABB43CBAF82A0030BD
:1035C0000AD7233C10B590F81411044602F008FE07
:1035D0006423C0B203FB0044A06F10BD10B59CB0C3
:1035E0000C463422002102A83CF0B8FE3222611CB5
:1035F0000DF10A0002F0E4FA32210DF10A003DF06B
:103600004BFA23780FA98DF809008DF8083002A82D
:103610000C4B93F91E20013A18BF012200F018FE4E
:103620000FAB80B244F64362009004A1D1E90001DF
:10363000FFF7DCFA1CB010BDAFF30080DD3B6FF08C
:10364000CC72DFFEF82A00302DE9F04F4FF4807382
:103650004E4D87B00446AB801DF0D0FD4FF47A7319
:1036600005A9B0FBF3F0286000256388B4F90220B7
:103670007F2B47488DF814509CBF464B1A700FF0B3
:103680001BFB94F90C30012B04D16568424BEB1AFB
:103690005D425D4194F90D3004F10C07261D012BAC
:1036A00003D1A2683C4B9A420DD065B9012305A90C
:1036B00038468DF814300FF0E5FA374B05A930463F
:1036C00005930FF05FFB94F929304FF0000ADFF803
:1036D000E490DA4303F00103DFF8DC8002F001023A
:1036E000DB0043EAC2432D4A93612D4B039301E073
:1036F0004FF0010A43F2B0705FFA8AFB02F014FD4A
:10370000054608B11AF090FA039BC9F8045043F833
:10371000045B89F800B0039317F8013B87F8FF3387
:1037200088F80430C8F8005055B194F91E302A6862
:10373000012B316821D1D2F800B02846F269D84770
:10374000043609F1080908F10808BAF1000FCFD0D2
:10375000002314494FF47A620193A1F12800124B1F
:103760000093124B35F0A8FC0A4B197851B1104860
:1037700007B0BDE8F04F35F0C5BC536828460122BC
:103780009847DDE707B0BDE8F08F00BF0C3300308D
:10379000072B00300833003040420F00000C025865
:1037A000FC42003040330030452A0408F12C040864
:1037B00018330030EC4200301C43003070B590F9F3
:1037C000E13196B00446002B5CD090F8DF32002B3C
:1037D00058D000F5E675284602F014FDD4F890673D
:1037E0002846FFF7EFFE86424CD094F8E0122846B8
:1037F00002F0F6FC6426C0B206FB004090F8FD31F2
:10380000002B3FD02846FFF7DDFE94F8E012C4F805
:103810009007284602F0E4FC2822C5B200210CA83B
:103820003CF09CFD06FB05439FED1A7A0021D3ED89
:103830008E7A152203A8029167EE877ACDED097A78
:10384000D3ED8F7A67EE877ACDED0A7AD3ED907A51
:1038500067EE877ACDED0B7A3CF080FD0E4B02A926
:1038600009A893F91E20013A18BF012200F094FF25
:1038700002AB80B240F2E932009004A1D1E900012C
:10388000FFF7B4F916B070BDAFF30080F2C20B467B
:10389000A9D4A7E26F12833AF82A003090F9503089
:1038A0000BB1FFF71BBD704730B5314D044695F99C
:1038B0000E302DED028B87B0002B4CD000F5397007
:1038C00001F0E6FE242294F8F532D4F8981702FBB2
:1038D0000343D3F8002391423DD0C4F8982793F8CE
:1038E0001D23002A37D0D3F80823002402A904A8F6
:1038F000049295F91E2093EDC38A013A059402942F
:1039000018BF0122ADF80C4000F08AFF02AB80B274
:1039100040F20442009012A1D1E90001FFF766F9DC
:1039200095F91E20DFED137A02A9013A04A878EE7A
:10393000277A059418BF01220294CDED047A00F095
:103940008BFF80B202AB40F20542009006A1D1E9A4
:103950000001FFF74BF907B0BDEC028B30BD00BF93
:103960009AC8BD1234C4C7CD7162D977642A274979
:10397000F82A0030339388430FB430B5C3B07C22AB
:10398000002146AC23A854F8045B3CF0E7FC00217E
:10399000772205A804913CF0E1FC23462A465A21EF
:1039A0000DF1AE0003941AF0D5FE114B5A2804A96C
:1039B00093F91E2028BF5A20013A8DF8AD0023A8A4
:1039C00018BF012201F072FA04AB80B243F6FF7215
:1039D000009005A1D1E90001FFF708F943B0BDE867
:1039E000304004B0704700BF759D040C8EA454D6BF
:1039F000F82A00302DE9F04F2DED028BB3B00446CC
:103A00001DF0FCFB834A07461368C31A322B09D901
:103A1000814B1B7833B1814910600B78013303F07F
:103A20001F030B707E4E1DF0DFFBD6F8CC3F984293
:103A300009D93046DFF8E08135F06CFB002861D011
:103A4000002388F80030774A1368FB1AB3F57A7FB1
:103A5000C0F0158117601DF0D3FB02460B4670487D
:103A600035F00EFCFEF7DAFF462804D96E4B6F489E
:103A700019781AF0B9FEFEF7D1FF462804D96A4B2F
:103A80006A48197A1AF0B0FE1DF0AEFB4FF47A7353
:103A9000674EDFF8C481B0FBF3F0664B30601F68FF
:103AA000786D03685B6E984798F91E2020A93081D5
:103AB000013A304618BF012201F0D0F920AB80B2A4
:103AC00040F2551200904FA1D1E90001FFF78EF8A6
:103AD00098F90F50002D00F0C7800023EDB220A907
:103AE00008F10F008DF880300FF0E6F82A2D6BD129
:103AF000514C2046FFF740FF386D642103685B6836
:103B00009847F6E71DF07AFB98F8003005462BB190
:103B1000FEF784FF014649481AF066FE09F000F9F5
:103B20004FF4C873B0FBF3F202FB130305F51670F4
:103B300096F8D02F10FA83F0414B1B78C6F8CC0FC3
:103B40005B00DBB28DF8383052B943F001038DF8D9
:103B5000383096F8D23F013303F0010386F8D23FA4
:103B600020A8FEF7C7FC96F8D01F20AB0DF1390056
:103B7000C1F110051944EDB2062D28BF06252A46CD
:103B80003CF0C4FB002301222548069396F8D23F5F
:103B9000154402FA03F3EDB2DBB2049505930EABC4
:103BA000039318230293274BCDE9002317A3D3E9EE
:103BB000002335F0B1FA011E02DA23481AF014FE90
:103BC000002386F8D03F3EE72B2D04D11F48FFF796
:103BD000D3FE1F4B98474FF4FA6120A818F0E8FD78
:103BE000386D4FF47A7103685B689847786D0368A5
:103BF000DB6A984790B3012800F0C68015482EE094
:103C0000AFF30080F1C6A7C1D068080F401DA12006
:103C100026812A0B0C430030D4250030104300309D
:103C20001833003008430030EC4200306E72080850
:103C30000C330030F02A0030987208080872080827
:103C400008330030044300303D720808A9720808A8
:103C500038ED00E0E4720808F82A00305F48FFF70A
:103C60008BFE20A818F0B0FD002373711DF0C6FA7A
:103C700047F23053984202D9594839F055F894F92F
:103C80002830002B40F082802046FFF707FE2046B8
:103C9000DFF85C81FFF792FD2046FFF705FE204626
:103CA000FEF718F91DF094FA09909FED4A8B1DF06C
:103CB0008FFA099BC01AB0F57A7F80F08380D8F81C
:103CC00000304021474C0226186DDFF82091036830
:103CD000DFF820A19B689847FEF7BEFC0021402238
:103CE0000FA80E91ADF87C103CF038FB54F8043C62
:103CF000002B60D014F8083C4B4493F80C74012F4F
:103D000059D154F8040C4FF0000B8DF82C700BA90E
:103D10008DF82DB002688DED008B93680DF12D02AA
:103D20001D465B46A8479DF82C20002A43D05946E3
:103D3000482220A83CF012FB54F8040C0CAA0EA94F
:103D40000368D3F814B00DF12E03D847002832DDF4
:103D50009DF87C0018F0B2FA9DF87D3002460FA95C
:103D60008DF8C40021A88DF8C7303CF0CFFA0E9B27
:103D700020A95046209314F8083C8DF8C530DDE9A1
:103D80000C2335F043FCBCE7174868E794F8B437D8
:103D9000002B3FF47CAF002394F8B22794F8B117BE
:103DA00084F8B43794F8B0070BF042F90F4B0122B6
:103DB00083F860246BE7012E04F108043FF477AF29
:103DC000012693E733B0BDEC028BBDE8F08F00BF56
:103DD000AFF300800000000000000000B972080886
:103DE000263A09B0F4420030CE720808F82A0030B2
:103DF000F02A003018330030024B012283F8D22F12
:103E0000704700BF1833003037B5054640F2062230
:103E10003948012136F06AFB40F206220221364879
:103E200036F064FB354B364C0321D3F8E8202120D3
:103E300042F48002C3F8E820D3F8102122F4800273
:103E4000C3F81021D3F81021D3F8902042F4800257
:103E5000C3F89020D3F8902022F48002C3F8902079
:103E6000D3F89030236823F001032360236823F400
:103E700080532360236823F470632360214B236104
:103E8000236823F400332360636823F400636360D2
:103E90004023A360A36843F40043A360AA23E36024
:103EA000E36843F40043E36037F03EFA23681649C1
:103EB00043F002032360236843F004032360236874
:103EC00043F008032360236843F020032360236842
:103ED00043F0010323600D4B00951B68186B0368CA
:103EE000DC680B4BA446019302AB13E90C0003B052
:103EF000BDE83040604700BF00140258004402583B
:103F000000580040380F300000730808F02A0030D5
:103F10008940040890F9283010B513B9012380F8BE
:103F2000B83711B153B2002B04DA02F07F0380F8E6
:103F3000B33710BD90F8B347022C10D0032C15D026
:103F4000012C05D103F00F0141EA021380F8B237CA
:103F50000134012380F8B34780F8B437E9E703F070
:103F60000F0141EA021380F8B137F1E703F00F01C6
:103F700041EA021380F8B037EAE70000092B2DE987
:103F8000FF410C46054611461E465BD81A4601A85D
:103F90003CF0BCF9242C3AD1092E38D19DF80530DB
:103FA0009DF804201B029DF8081043EA02439DF887
:103FB0000620090213435B421A0C8DF806308DF877
:103FC00004201A0A9DF807308DF8052041EA0341C4
:103FD0009DF80930194349420B0C8DF809108DF8F2
:103FE00007300B0A9DF80B108DF8083009029DF878
:103FF0000A3041EA03419DF80C30194349420B0C49
:104000008DF80C108DF80A300B0A8DF80B30D5F8AE
:10401000CC7467B1013E01AD4FF00108731C11D0A3
:104020003B79A3421CD03B6813B31F46F8E7082036
:1040300002F07AF89DF80430C5F8CC0443710123EE
:104040000471837104B0BDE8F081047101342B78F0
:10405000E4B280F806804371013E01350746DDE792
:104060002B780134384687F80680E4B27B71F3E799
:10407000082002F059F838600028E6D101481DF008
:1040800081F800BF0873080810B49DF8044001943B
:104090005DF8044BFFF772BF3629D0F8CC0410D07E
:1040A000E0B103798B4213D00068F9E70379242B40
:1040B00009D000680028F9D170470023837180205F
:1040C0007047222070478379002BF6D1184670473D
:1040D0003429EED000238371407970477047000087
:1040E0002F4B10B59C69200715D52E4AC4F34641C5
:1040F000002082F8B617C4F3004182F8B50782F8B1
:10410000B71719B19A6942F001029A61244AD3693A
:1041100043F00803D361610718D5214B21485A6A3F
:1041200090F8B637D2B290F8B517232B05D81F2BCD
:1041300007D931B980F8C92403E0552B01D1FFF725
:10414000E9FE90F8B537013380F8B537A2071CD5E2
:10415000144A92F8B637232B0DD81F2B10D992F89A
:10416000B537104692F8C9141944C9B2FFF794FF45
:104170000B4B986204E0552B02D1094B0021996248
:1041800092F8B537013382F8B537A30604D5044A4F
:10419000D36943F02003D361BDE8104035F0EABC99
:1041A00000580040F82A003013B5044608460021A4
:1041B0002022234601900160C0F8031035F0DEF99B
:1041C000231D01980122202135F0D8F9019804F12E
:1041D00008031722212135F0D1F9072002B010BDC4
:1041E000002308222DE9F3410C46009119460546AB
:1041F00035F080F8631C0822002604F102080093C1
:1042000011460023284635F075F86378F7009E4282
:1042100007F1100111D304F58474002340222846CD
:104220000094573735F066F8AB8AB3EBD70F14BF5D
:104230000120002002B0BDE8F08108EB060308224F
:10424000284601360093002335F054F8DDE70000DE
:10425000F8B50E46054614460021342230463CF09F
:104260007DF82B4608220021304635F087F97CB9CD
:104270000E246B1C06220821304635F07FF90123FD
:104280005F1C6A78013B934204D3E01DC008F8BD6F
:104290000824F4E7EB1921460822304635F06EF980
:1042A00008343B46ECE7000000232DE9F7430527DF
:1042B000002690F81C800C46009105221946054600
:1042C00035F018F8237807F108099E4230D304F13D
:1042D00015030822394628460093002335F00AF8D2
:1042E00004F116030822494600932846002307F1EB
:1042F000100634F0FFFFB8F1000F24D104F11703CA
:10430000314607F11506052200932846434634F04E
:10431000F1FF2746E27D3B1B9A421AD80736AB8A4B
:10432000B3EBD60F14BF0120002003B0BDE8F0832B
:104330000136394608222846A3194F460093002328
:1043400034F0D8FFBEE7AB8AC6EBC303DB08E375E6
:10435000DFE707F1180331460822284600930023BF
:104360000836013734F0C6FFD4E7000000230522E9
:104370002DE9F3410525002700910C461946064614
:1043800034F0B8FF237805F108089F42C0F0A880F8
:1043900004F115032946082230460093002334F027
:1043A000A9FF04F116034146102200933046002372
:1043B00034F0A0FF04F1180305F118011022009356
:1043C0003046002334F096FF04F11A0305F128016A
:1043D000102200933046012334F08CFF04F11C03BB
:1043E00005F13801202200933046012334F082FF8A
:1043F00004F1200305F158012022009330460123E7
:1044000034F078FF04F1240305F1780120220093B1
:104410003046012334F06EFF04F1280305F19801C2
:10442000202200933046012334F064FF04F12C0372
:1044300005F1B801082200933046002334F05AFFFA
:1044400004F1300305F1C00120220093304601231E
:1044500034F050FF04F1340305F1E0010822009329
:104460003046002334F046FF04F1350305F1E8013E
:10447000082200933046002334F03CFF04F1360359
:1044800005F1F001082200933046002334F032FF9A
:1044900004F1370305F1F8010822009330460023A8
:1044A00034F028FF04F138033C3405F580710093A3
:1044B00020220123304634F01DFF05F590710023C2
:1044C00008223046009434F015FF05F22F11B38A0C
:1044D000B3EBD10F14BF0120002002B0BDE8F08182
:1044E0000137294608223046E31945460093002348
:1044F00034F000FF46E7000000232DE9F7430527CD
:104500004FF0000890F81C900C46009105221946C7
:10451000064634F0EFFE237807F10805984525D3C9
:1045200004F115030822394630460093002334F085
:10453000E1FEB9F1000F26D104F11603294607F177
:104540000D050522009330464B4634F0D3FE274636
:10455000A27D3B1B9A421CD80735B38AB3EBD50F1B
:1045600014BF0120002003B0BDE8F08308F101086A
:1045700039460822304604EB08032F4600930023F7
:1045800034F0B8FEC7E7B38AC5EBC303DB08A375F5
:10459000DDE707F117032946082230460093002380
:1045A0000835013734F0A6FED2E7000000232DE9DC
:1045B000F74305274FF0000890F81C900C46009137
:1045C00005221946064634F095FE237807F10805C2
:1045D000984525D304F11503082239463046009347
:1045E000002334F087FEB9F1000F26D104F1160341
:1045F000294607F10D050522009330464B4634F05D
:1046000079FE2746A27D3B1B9A421CD80735B38A08
:10461000B3EBD50F14BF0120002003B0BDE8F08339
:1046200008F1010839460822304604EB08032F46FA
:104630000093002334F05EFEC7E7B38AC5EBC303E3
:10464000DB08A375DDE707F117032946082230468A
:10465000009300230835013734F04CFED2E7000008
:10466000002305222DE9F3410525002700910C4682
:104670001946064634F03EFE237805F108089F42AD
:104680007FD304F115032946082230460093002306
:1046900034F030FE04F11603414608220093304600
:1046A000002334F027FE04F1180305F11001202245
:1046B00000933046012334F01DFE04F11C0305F184
:1046C0003001202200933046012334F013FE04F120
:1046D000200305F15001102200933046002334F0EE
:1046E00009FE04F1220305F1600110220093304617
:1046F000002334F0FFFD04F1240305F170012022B2
:1047000000933046012334F0F5FD04F1280305F150
:104710009001202200933046012334F0EBFD04F198
:104720002C0305F1B001082200933046002334F039
:10473000E1FD04F12D0305F1B80108220093304694
:10474000002334F0D7FD04F13003343405F1C00107
:10475000009320220123304634F0CCFD05F1E00126
:10476000002320223046009434F0C4FD05F20711E6
:10477000B38AB3EBD10F14BF0120002002B0BDE813
:10478000F0810137294608223046E3194546009357
:10479000002334F0AFFD6FE72DE9F74305460E46E1
:1047A00000241746A8461922002130463BF0D6FDCA
:1047B000B8EC010A35F078F921461034ADF806005E
:1047C0000DF106031022304634F0D8FE302CEFD124
:1047D0003FB92146342405F10C030422304634F05D
:1047E000CDFE05F110094FF000082B7B04EB0817F4
:1047F000984504D3F81DC00803B0BDE8F083B9ECB8
:10480000010A08F1010835F04FF90DF10603ADF882
:10481000060010223946304634F0B0FEE5E70000CD
:1048200037B50C4600210546034621602022A180B1
:10483000204634F0A3FE95ED010A35F035F90DF16F
:104840000603ADF8060010222046202134F096FE23
:10485000062003B030BD000073B500260C460546A7
:104860000E6090ED000A35F01FF90DF10603314698
:104870001022ADF80600204634F080FE95ED010AC6
:1048800035F012F91022ADF806000DF106032046AE
:10489000114634F073FE042002B070BD73B50C46AF
:1048A000102605460021324620463BF057FD95ED87
:1048B000000A35F0F9F80DF1060332460021ADF893
:1048C0000600204634F05AFE95ED010A35F0ECF86A
:1048D0000DF1060332463146ADF80600204634F0AD
:1048E0004DFE95ED020A35F0DFF80DF10603324674
:1048F0002021ADF80600204634F040FE95ED030A75
:1049000035F0D2F80DF1060332463021ADF806003D
:10491000204634F033FE95ED040A35F0C5F80DF16C
:10492000060332464021ADF80600204634F026FE4C
:1049300095ED050A35F0B8F80DF106033246502121
:10494000ADF80600204634F019FE95ED060A35F064
:10495000ABF80DF106033246ADF8060060212046A3
:1049600034F00CFE05F11C0320460722702134F0C0
:1049700005FE204605F11D030622772134F0FEFDD9
:10498000304602B070BD00002DE9F04F0C460546E0
:1049900085B0002191462046DE2205F1440A3BF015
:1049A000DDFC2B46382200212046002734F0E6FDAE
:1049B000382205F108032046114634F0DFFD05F1E9
:1049C000100303227021204634F0D8FD05F11103B5
:1049D00008228021204634F0D1FD05F1180325225C
:1049E0008821204634F0CAFD05F120032522AD219F
:1049F000204634F0C3FD05F128031B22D2212046B6
:104A000034F0BCFD05F12C031B22ED21204634F0CF
:104A1000B5FD05F1300320224FF48471204634F0B7
:104A2000ADFD05F1340320224FF49471204634F09B
:104A3000A5FD05F1380320224FF4A471204634F07F
:104A40009DFD05F13C0306224FF4B471204634F07D
:104A500095FD05F13D0302224FF4B771204634F075
:104A60008DFD05F13E0304224FF4B871204634F069
:104A700085FD05F13F0306224FF4BA71204634F05C
:104A80007DFD05F1400306224FF4BD71204634F050
:104A900075FD4FEA071895F8403008F5C0719F4240
:104AA00008F5C876019125D395ED350A34F0FCFF61
:104AB0000DF10E03ADF80E0010220199204634F0DE
:104AC0005DFDB9F1000F08D1314608F2911605F1EC
:104AD000D8030122204634F051FD05F586774FF0CA
:104AE000000A95F8D8309A4513D3F01DC00805B0D8
:104AF000BDE8F08FBAEC010A013734F0D5FF0DF1B3
:104B00000E03ADF80E0010220199204634F036FD58
:104B1000BFE7A7F12C0B06F16008B146494609F141
:104B200020095B46202220460BF1040B34F026FDC1
:104B3000C845F3D1A7F11C0906F1CC0B414608F199
:104B400024084B462422204609F1080934F016FDBA
:104B5000C345F3D106F1D201B946D8364FF000086B
:104B60003B1F0622204634F009FD17F8043C984507
:104B700003D30AF1010AC037B3E7B9EC010A08F11F
:104B8000010834F091FF3146ADF80E000DF10E032F
:104B900010222046103634F0F1FCE6E70023F7B58A
:104BA000047F0E46009108221946054634F0A2FB08
:104BB000BCB9731C082228460093234610241146D2
:104BC00034F098FB01235F1C7278013B9A420FD8A6
:104BD0000734AB8AB3EBD40F14BF0120002003B01D
:104BE000F0BDAB8A0824DB00083BDB087370E9E703
:104BF000F3192146082228460093002334F07AFB5B
:104C000008343B46DFE70000F7B50C461546009236
:104C1000002308220968064634F06CFB21686F1CEB
:104C200000230522083100973046AF1C2160033570
:104C300034F060FB216800230622053130460097DE
:104C4000216034F057FB21680023052206313046ED
:104C50000095216034F04EFB23680533236003B0D8
:104C6000F0BD0000F0B5002385B0057F06460C4678
:104C7000039375BB2B4600910522294634F03AFB7D
:104C8000039B671C0533039323789D4217D23A4652
:104C900003A9304601350437FFF7B6FFF4E7227861
:104CA00003A9304617FB02522244FFF7ADFF2378D9
:104CB00001332370B28A039BB3EBC20FEFD1039B86
:104CC000B28A0733B2EBD30F14BF0120002005B026
:104CD000F0BD042701250B70ECE70000002308223B
:104CE00013B504460091194634F004FBA08A01383C
:104CF00018BF012002B010BD2DE9F0470D46044653
:104D000000219046284640F279123BF027FB2346CB
:104D100020220021284604F1220734F02FFC231D15
:104D2000022220212846C02634F028FC631D0322DD
:104D30002221284634F022FCA31D032225212846E7
:104D400034F01CFC04F1080310222821284634F01A
:104D500015FC04F1100308223821284634F00EFC1B
:104D600004F1110308224021284634F007FC04F125
:104D7000120308224821284634F000FC04F11403F1
:104D800020225021284634F0F9FB04F11803402278
:104D90007021284634F0F2FB04F120030822B021F0
:104DA000284634F0EBFB04F121030822B821284601
:104DB00034F0E4FB314608363B46082228460137EA
:104DC00034F0DCFBB6F5A07FF4D1002704F1330A00
:104DD00004F1320308223146284634F0CFFB94F820
:104DE00032304FEAC7099F4209F5A47615D3B8F1CE
:104DF000000F08D1314609F24F1604F599730722C6
:104E0000284634F0BBFB27463B1B94F832219342E3
:104E10000CD3F01DC008BDE8F0870AEB0703082299
:104E200031462846013734F0A9FBD8E707F233139F
:104E30003146082228460836013734F09FFBE3E765
:104E40000023382213B504460091194634F052FA73
:104E5000A08A073818BF012002B010BD13B5044660
:104E6000084600212022234601900160C0F803106B
:104E700034F084FB231D01980222202134F07EFBB4
:104E8000631D01980322222134F078FBA31D0198B1
:104E90000322252134F072FB019804F1080310224B
:104EA000282134F06BFB072002B010BD2DE9F04142
:104EB0000E4605460021174630467B223BF04EFA4F
:104EC0002B4603220021304634F058FB6B1C052290
:104ED0000321304634F052FB0123DC0003F10108CA
:104EE0006A78013B9A4212D83FB92146073405F14E
:104EF00021030722304634F041FB2F467B1B95F8F7
:104F0000212093420CD3E01DC008BDE8F08105EBE1
:104F1000080308222146304634F030FB4346DCE7E4
:104F200007F122032146082230460834013734F0C5
:104F300025FBE3E70023F7B50C46067F0722009127
:104F40001946054634F0D6F9631C01220721009367
:104F50002846002334F0CEF9B6B9A31C0522082157
:104F60002846009333460D2634F0C4F92746A2782C
:104F70003B1B9A420FD80736AB8AB3EBD60F14BF50
:104F80000120002003B0F0BDAB8A0826DB00083BFF
:104F9000DB08A370EAE7FB1C314608222846009391
:104FA00000230836013734F0A5F9E0E7F8B50E46DE
:104FB000054614460021812230463BF0CFF92B46AE
:104FC00008220021304634F0D9FA7CB90F246B1C3A
:104FD00007220821304634F0D1FA01235F1C6A7899
:104FE000013B934204D3E01DC008F8BD0824F4E758
:104FF000EB1921460822304634F0C0FA08343B460B
:10500000ECE7000037B50C46002305460091083454
:105010001946082234F06EF901233022082128466F
:10502000009434F067F9A88A073818BF012003B04C
:1050300030BD000038B50C4600210546034621600E
:105040002046C4F80310302234F098FA204605F1C7
:1050500008030122302134F091FA072038BD000006
:105060002DE9F043002385B00D4690F81C800D22F9
:1050700000911946064634F03DF90DF10F03032265
:105080000D2100933046002334F034F99DF80F30A1
:105090002B72013B032B5DD8DFE803F00229343F7C
:1050A00005F11003502440221021009330460123C3
:1050B00034F020F9B8F1000F4ED105F198032146E4
:1050C0000734072200933046434634F013F92F4645
:1050D00095F898207B1B9A4245D80734B38AB3EBE6
:1050E000D40F14BF0120002005B0BDE8F08305F106
:1050F000100320221021304600930123302434F085
:10510000F9F8D7E705F11003082210213046009383
:105110000023182434F0EEF8CCE705F11003002743
:1051200005F111090822009310210023304634F0C4
:10513000E1F82B7CFC009F4204F11804BAD209EB81
:10514000070308222146304600930023013734F03C
:10515000D1F8EEE71024ADE7B38AC4EBC303DB0854
:1051600085F89830B3E707F19903214608223046C5
:10517000009300230834013734F0BCF8A8E700009E
:10518000F7B513780C46154609688DF807300322E9
:105190000DF10703064634F0F1F92168033121606F
:1051A0002B78013B032B0CD8DFE803F0020D161F10
:1051B00005F108034022304634F0E0F9236840331B
:1051C000236003B0F0BD05F108032022304634F01F
:1051D000D5F923682033F3E705F1080308223046A8
:1051E00034F0CCF923680833EAE705F10803082214
:1051F00030462F4634F0C2F92368083323602A7AF8
:105200007B1B9A42DDD907F1090308222168304649
:1052100034F0B4F92368013708332360EFE7000066
:1052200073B513780C46154609688DF807300222CD
:105230000DF10703064634F0A1F92168023121601F
:105240002B78012B03D0022B0BD002B070BD05F1DF
:1052500008034022304634F091F92368403323603C
:10526000F3E705F108032022304634F087F923687C
:105270002033F4E7F7B50D4604461646002140F208
:10528000731228463BF06AF80523224601A92846F6
:105290000193FFF775FF019B04F1900201A905330B
:1052A00028460193FFF76CFF019B04F5907201A95A
:1052B000284606330193FFF7B3FF019B04F598726C
:1052C00001A9284606330193FFF7AAFF4EB904F55A
:1052D000A07307220199284634F050F9019B073347
:1052E0000193002604F2411794F8403101999E423F
:1052F00003D30731C80803B0F0BDBB190822284604
:10530000013634F03BF9019B08330193ECE70000D0
:10531000002343608360C360036143618361C361B1
:10532000002380F82030704790F82020531C00EBB9
:105330008202DBB2062B80F8203082ED010A84BFA6
:10534000002380F8203070474FF0FF3310B54361E1
:1053500004460D4BB0300360002380F82030FFF787
:10536000D7FF0A4B04F58870C4F8B03019F0C6F9BD
:10537000074B204607491C600CF0A8FFD4F890307A
:105380002046C4F8943010BDB8730808C8730808E4
:10539000144300302C740808B03008B50EF036FD08
:1053A000DFED027A20EE270A08BD00BF00007A4434
:1053B00090ED3E0ADFED057AB0EEC07AB4EEE77A02
:1053C000F1EE10FA48BF90ED3F0A7047000000343C
:1053D000F0EE406A10B52DED028BFFF7E9FFB0EE5D
:1053E000408A80EEA60A044638F054FEDFED0C7ABF
:1053F00020EE270A38F0D4FDDFED0A7A38EE278A4E
:10540000DFED097A28EE278AF7EE007A77EEC07A88
:1054100094ED250A98EE270ABDEC028B10BD00BF63
:1054200041D3423E33938843A1D8194308B52DEDAB
:10543000028BB0EE408AFFF7BBFFD0ED257A9FEDDF
:105440000D7ADFED0D0A67EE877A9FED0C7A30EE6C
:10545000070A87EE807A9FED0A0A30EE470A38F095
:10546000C9FEDFED087A28EE278A28EE000ABDEC97
:10547000028B08BD00409C451931A8C03393884376
:10548000F0CC3B49C762DA7210B52422B3EE097A38
:105490000446DFED276A2DED028B437CD0ED287AA0
:1054A00002FB030292ED0B8A78EE677AF0EEE77A60
:1054B000F4EEC77AF1EE10FA08D590ED290AF0EE75
:1054C000C07AF4EEE67AF1EE10FA2BD5242202FB34
:1054D000034393ED096AF0EEC67AF4EEE67AF1EE54
:1054E00010FA22D42046FFF763FFDFED127A9FED1A
:1054F000127A30EE270ADFED117AA8EE670ADFEDA7
:10550000107A20EE270AC6EE007A87EE270AB4EE5C
:10551000E60AF1EE10FA08DB39F0C0F984ED288ACA
:1055200084ED290ABDEC028B10BDB7EE000AF9E745
:105530000000003433938843CDCC9C3FF4FDD43B32
:1055400048A18F4338B5D0F8AC3004460D465BB166
:105550001BF04AFED4F8AC30C01A42F20F739842E6
:1055600002D894ED2A0A38BD2421DFED077A01FB29
:10557000054494ED0A0AB4EEE70AF1EE10FA58BFBA
:10558000B0EE670AEFE700BF00000C422DE9F047DC
:1055900004461BF029FE42F210734FF00008D4F8C5
:1055A00000614FF0240942F2107A861B9E4288BFA8
:1055B000C4F80001237C5FFA88F5AB4219D909FBD6
:1055C000054797F8393053B197ED0D0A2046D7EDCE
:1055D000097A30EE270AFFF729FF87ED0C0A5645B6
:1055E00004D909FB054030300CF0ECFE08F101084D
:1055F000E0E7617C2046FFF7A5FF002384ED3F0A2A
:10560000C4F8A430BDE8F08708B561B10378022B77
:1056100002D906481BF0B6FD5A1C027000EB83004D
:105620004160012008BD0846FCE700BF7873080808
:105630002DE9F84305460E469146002400F13C084A
:105640002B78A34211DD00234A463146012016F093
:105650008BFF242307460021634358F8030016F00C
:1056600093FF874204D00134EAE70020BDE8F883C5
:105670000120FBE7054B1B682BB141694A1C02D096
:10568000184607F043B80020704700BF4448003078
:10569000F0B52DED048B85B0044640F2853200F55F
:1056A000887103A8002517F09DF8D4ED227AD4ED77
:1056B000236A24229FED746A37EEE67A637C02FB4C
:1056C0000343B0EEC77AB4EEC67AF1EE10FAC1BF6A
:1056D0009FED6E7A67EE877A9FED6D7AE6EE877AB8
:1056E000C4ED237A93F83960E9B223788B4206D966
:1056F00004EB8103013558681EF00CFCF4E7002729
:10570000DFED648A9FED648A9FED649A237CFDB28D
:105710002422AB425FD902FB054393F83920002ACB
:1057200057D0D3ED0C7AF4EEE87AF1EE10FA0BDBF9
:10573000F4EE677AF1EE10FA06D6F0EEE77AF4EEC0
:10574000487AF1EE10FA04DD242303FB05435A6A7C
:105750001A63242303FB0543D3ED090AD3ED0D7A25
:1057600093F8382070EEA70A82B993ED0C0A204610
:10577000FFF72EFEB4EE400AF1EE10FA16D72423FE
:1057800003FB0545002385F83A3022E0012A09BFD2
:10579000D3ED0C7A93ED0B0A77EEE00AD4ED3D7A67
:1057A00004BF80EE897A87EE270AE3E7F0EEC07A3D
:1057B000242303FB0545F4EE487AF1EE10FAE1DC10
:1057C000012385F83A30D4ED237A37EE800A85ED4F
:1057D0000B0A01379AE7637C02FB034393F83920F5
:1057E00032B1D96904F1B00093ED0B0A0EF0F0FA72
:1057F00094F99C30217C002B07DB8B4205DA2422B4
:1058000002FB034292F839207AB9002304F115050E
:1058100024276374DAB2914208D9013307FB03F0FD
:10582000285C0028F6D0627400E063742046FFF71D
:1058300021FF10B120461FF061FB637C242505FB8E
:10584000034393F83930B34216D006F07BFF4FF68E
:10585000FF7106F05BFF78B1607C05FB004494F8B3
:105860003930002B14BF00220422019206F06AFF97
:10587000019A122106F0E8FE03A816F0D5FF05B044
:10588000BDEC048BF0BD00BF0AD7233CCDCC4C3D12
:105890003333733F00000034FFFF7F7F0020194641
:1058A00008B5037C022B02D903481BF06BFC5A1C81
:1058B0000274184608BD00BF9473080810B5002292
:1058C000017C00F115032424D0B2814206D90132B3
:1058D00004FB02F0185C0028F6D110BD081E18BFAA
:1058E0000120FAE7014B1868704700BF14430030ED
:1058F00010B50446006810B103685B6898472046FD
:1059000010BD000010B50446006810B103685B6864
:105910009847204610BD00002DE9F04F8FB0D0F819
:1059200008310446344D0893344B05F1C00A1B6816
:10593000D86A05930368DB68984794F99D30069010
:10594000002BA2BF012606FA03F306932B68089AE0
:105950001A420BD000274FF0010BB9460BFA07F3A0
:10596000069A134206D10137202FF7D10C35554541
:10597000ECD12DE0F9B26B682A7A204609910793A1
:10598000FFF756FE0999804628B3CDE90A990B9B8B
:105990000DA920460D93079BCDE90B999847014629
:1059A0002046FFF731FE0DA8FFF7ACFF0CA8FFF76C
:1059B000A9FF0BA8FFF79CFFB8F1000F02D00AA8BF
:1059C000FFF796FF2378032B02D0237C032BCAD149
:1059D0000FB0BDE8F08F059B0422D86A0368CDE9BB
:1059E0000182074A00920A461B6801460BA81E4620
:1059F0002B7AB047CBE700BFF4740808F02A0030D8
:105A0000801A060070B5D0ED247A01239FED487A04
:105A10008AB0F0EEE77A04460376F4EEC77AF1EE48
:105A200010FA09D49030002309A9059009930DF0CC
:105A3000F3F805980CF0C6FC3E4B00253E4A07A83B
:105A40001E68E5632566C4F88450316B0B681B68DB
:105A50009847079B2A4609A920460993CDE907558F
:105A60001FF080FF01462046FFF7CEFD09A8FFF793
:105A700049FF08A8FFF746FF079810B103685B6865
:105A800098472378032B42D0237C032B3FD094F9F3
:105A90009D10002911DA20463A34FFF73DFF14F833
:105AA0002A1C00230122D8B2243481422FD9013389
:105AB00004F8232C04F8242CF5E77722C9B22046F9
:105AC000FFF7B6FD054620B30023CDE90633079B5B
:105AD000002209A920460993CDE907221FF042FFC1
:105AE00001462046FFF790FD09A8FFF70BFF08A825
:105AF000FFF708FF07A8FFF7FBFE15B106A8FFF7A1
:105B0000F7FE2378032B02D0237C032BC3D10AB0EA
:105B100070BDF16A04220B68CDE90102074A07A8AB
:105B200000921E68772394F89D20B047CFE700BF0E
:105B300000000034F02A0030A8730808801A06001C
:105B4000002213B50B680A6001A901931EF02EFD17
:105B5000044601A8FFF7D6FE204602B010BD0000A3
:105B6000002213B50B680A60022201A901931FF0FD
:105B7000F9FE044601A8FFF7C5FE204602B010BD9D
:105B8000002213B50B680A60012201A901931FF0DE
:105B9000E9FE044601A8FFF7B5FE204602B010BD9D
:105BA000002213B50B680A6001A901931FF0DAFE09
:105BB000044601A8FFF7A6FE204602B010BD000073
:105BC00070B50C4615460646114620463AF064FF6D
:105BD000854202462146304688BF0132BDE870400A
:105BE0003AF094BB004870473C73080810220449FF
:105BF00008B53AF07BFBB0FA80F0400908BD00BF61
:105C00002C430030102200213AF0A8BB10B5044606
:105C1000FFF7F8FF204610BD0378022A416023F009
:105C20000D03037008D0032A0AD0012A03D1DBB286
:105C300043F0010303707047037843F00803F9E76A
:105C4000037823F0050343F00503F3E773B5044637
:105C50000E4615460193FFF7D5FF2046069A019997
:105C6000C4E90265FFF7D8FF02B070BD00784207B3
:105C700004D4030704D400F00100704703207047E8
:105C800002207047F0B585B005461646FFF7EEFFD7
:105C900088420F4605D16B6833600124204605B069
:105CA000F0BD032801D10024F8E70329FBD0012827
:105CB0000BD0022816D018BB6D68012F22D0022FFE
:105CC0002ED0002FEFD13560E7E71CF0B7FB90F83E
:105CD0003C34DB07E7D56D681CF0B0FBD0F83034FE
:105CE0001D44EAE76846FFF78DFF1CF0A7FB6946F5
:105CF0001CF0FCF904460028D0D06D68019BEFE74A
:105D00000025DAE71CF09AFB90F83C4414F00104FB
:105D1000C9D01CF093FBD0F83034ED1A3560BDE7E4
:105D20006846FFF76FFF1CF089FB69461CF0DEF93F
:105D300004460028B2D0019BEFE7000007EE900A6E
:105D40009FED0C0AF8EEE77A08B527EE800A37F0E7
:105D50003BFEDFED097AB4EEE70AF1EE10FA02DD60
:105D6000B7EEC00A08BD9FED010BFBE70000004045
:105D7000E17A843F50E0EF300AD7233C10B5044667
:105D8000806807F0AFF820B1E068BDE8104007F088
:105D9000BDB810BD0D4B83424FF000038B4106DAB6
:105DA00000F1255000F5311000F5E0507047084B28
:105DB00098424FF0FF3371EB0303BEBF00F1564032
:105DC00000F5130000F52440704700BF00D2496B76
:105DD000002EB69490EA010F01D4401A7047C31701
:105DE000401A63EBE1710D4B83424FF000038B418E
:105DF00006DA00F1255000F5311000F5E05070474B
:105E0000074B98424FF0FF3371EB0303BEBF00F125
:105E1000564000F5130000F52440704700D2496B4E
:105E2000002EB69470B52DED028B84B004460D465D
:105E30006846FFF7E7FE1CF001FB69461CF056F9C7
:105E4000064628B3A368029ADFED148A9B1A0399C9
:105E500007EE903AF8EEE77A67EEA87AC5ED007A99
:105E6000E068FFF7B7FF08EE100AA068B8EEC88A2E
:105E7000024428EE288A02EBD2725010B7EEC88A8C
:105E8000FFF75CFF28EE000BB7EEC00B85ED010AB3
:105E9000304604B0BDEC028B70BD00BFF67C8E3F77
:105EA00037B505460C46FFF7BDFF10B9002003B01B
:105EB00030BD002301AA022128460193FFF7E2FE2C
:105EC0000028F3D0DDED017AF8EEE77AC4ED027A2E
:105ED000EDE7000038B50C4602462DED028BC16897
:105EE000E068FFF777FF9568A46808EE100A60196C
:105EF000641B00EBD0704010FFF720FF07EE904AC4
:105F0000B8EEC81BB8EEE77B87EE006BBDEEC60BA4
:105F100010EE103A5B4200EE103AB8EEC00B38F0CB
:105F200003FC9FED087B30EE070BB5EEC00BF1EEE6
:105F300010FA03D59FED057B30EE070BBDEC028B0D
:105F400038BD00BF00000060FB21F93F0000006089
:105F5000FB211940F0B50D4606462DED028B8C68ED
:105F600089B0D0E90271E868FFF734FF08EE100A43
:105F7000E019E41B00EBD0704010FFF7DFFEB8EE35
:105F8000C86ADFED0F4A736826EE246A6A689FEDDF
:105F90000D1A9B1AB7EEC66A07EE903A26EE006B12
:105FA000B8EEE75A07EE904AF8EEE75AF7EEC60B5E
:105FB00025EE011A25EEA40A09B0BDEC028BF0BD56
:105FC0008262363C0AD7233C0B4630B52DED028B5E
:105FD0008C6889B0D0E90251D868FFF7FBFE08EE63
:105FE000100A6019641B00EBD0704010FFF7A6FE8A
:105FF00007EE904AB0EE401BB8EEE76BB8EEC87BF8
:106000009FED050B27EE007B26EE000B27EE011B14
:1060100009B0BDEC028B30BD0000004050CC863F83
:1060200084B004B0FFF7D0BF10B52DED048B8468A9
:106030000B468A68111B224409EE101AC168D86801
:1060400002EBD272FFF7C6FE08EE100A5010B8EE4F
:10605000C99BB8EEC88BFFF771FE28EE000B20EE4F
:10606000000BA9EE090B38F08FFB9FED037BBDEC15
:10607000048B20EE070B10BD0000004050CC863F83
:10608000094B984206DDC0F1D64000F5930000F5BB
:10609000A4407047054B9842BEBFC0F1144000F5C4
:1060A000360000F53850704700E9A43500175BCA88
:1060B000F8B52DED048B9FED149BB0EE418B076876
:1060C00006460D4620EE090B28EE098BFDEEC07B3F
:1060D00017EE904A04EBD47007EB6000FFF72EFE3A
:1060E00088EE007B3819FFF7CBFF306051EC170BBF
:1060F000FAF774FC2B68C01841EBE371FFF74AFE16
:106100002860BDEC048BF8BD00000040407556408F
:1061100000F10C010830FFF7CBBF00000148FFF78A
:1061200071BD00BF2C4300300121884238BF0846B2
:1061300036F06CBC08B136F06DBC7047FFF7F4BFA9
:10614000FFF7F8BF00214FF0FF33002210B5436284
:10615000044600F1300301600171F83040F8F31C8F
:1061600000F8EF1C00F8DF1CD970643343F85C2C96
:1061700043F8582C43F8542C43F8402C43F83C2C5B
:1061800043F8382C43F8342C43F8302C43F82C2CAB
:1061900043F8282C43F8242C43F8202C43F8102CE7
:1061A00043F80C2C43F8082C9842DDD1044B1A68B4
:1061B00022B9044920461C600CF088F8204610BD26
:1061C0003C4300300476080890F8321029B90123C6
:1061D0004386117083751846704700207047000091
:1061E0004FF000007047000049B1037D012B06D03D
:1061F0005A1C0433027540F8231001207047002018
:106200007047000073B590F915500446002D49D031
:1062100090F81351002D45D090F831600025227D73
:10622000EBB29A4207D90433013554F823000368CE
:106230009B689847F3E71AF0D7FFA36FC01AB0F531
:10624000FA7F2CBF00230123B0F5FA7F84F83130A8
:106250000CD2636A013309D006F074FA616A06F061
:1062600055FA18B106F06EFA05F0EAFC94F9F83028
:1062700013B1002384F8143194F83150AE4211D098
:1062800006F060FA4FF6FF7106F040FA50B1002DAB
:1062900014BF00220422019206F054FA019A03214D
:1062A00006F0D2F9284602B070BD000010B50446D1
:1062B000002138300BF01CFB04F14C0104F14800C4
:1062C000BDE810400CF05EBD30B403460D4600F151
:1062D000380407CA84E807002946184630BCFFF78F
:1062E000E5BF0000024690F9150058B192F813017D
:1062F00040B1114491F9F80020B192F91800033827
:1063000018BF01207047000090F831201AB190F8B2
:106310001411FFF7E7BF104670470000024690F9DE
:106320001500B0B192F8130198B1D2ED117A9FED3A
:10633000097AF4EEC77AF1EE10FA09D4B7EE087ACA
:10634000F4EEC77AF1EE10FAD4BF012000207047B6
:1063500000207047ABAA2A3F836C1BB10021483054
:106360000BF0C6BA70470000014B1868704700BFB9
:106370003C43003030B5D0F8045185B0044615F4E4
:1063800080351FD1174B01A8174A1B68196B0B6882
:106390001B689847019B0422294603A80393CDE973
:1063A000015521F0C1F901462046FFF71DFF03A862
:1063B000FFF7A8FA02A8FFF7A5FA019810B1036841
:1063C0005B689847237D0BB1A37D4BB9054B07490B
:1063D0001B68186C03681B6805B0BDE8304018479F
:1063E00005B030BDF02A003000730808B475080805
:1063F00010B590F915300446A3B1836C0365837D15
:106400008BB10C4B64211B68186D03685B6898475F
:106410002046FFF7F7FE94F8323003B9A364012356
:1064200084F8133110BDFFF7A5FFA37D002BF2D038
:10643000E7E700BFF02A00302DE9F3410F460E6870
:1064400001250D4C54F8351008460191FAF7E4FE89
:1064500001995FFA80F8304642463AF0F5FA30B9D1
:10646000464404EBC5003E6002B0BDE8F081013552
:10647000052DE7D10048F7E7107708080B680548B5
:10648000B3F5A06F3FBF1A0ADBB200EBC2000B608E
:10649000704700BF1077080830B585B0CDE90221FC
:1064A00003A90193FFF7C8FF044640680168DDE9CE
:1064B00001320D680399A847011E09DBFF290ADD97
:1064C000606803685B68984739F038FE22230360F0
:1064D0004FF0FF3005E00448201AC0F3C70001EB7D
:1064E000002005B030BD00BF1077080807B5019146
:1064F00001A9FFF7C3FF4068019903685B689847EB
:1065000003B05DF804FB00001FB5CDE9022103A92B
:106510000193FFF7B3FF40680168DDE901328C6841
:106520000399A04704B010BD1FB5CDE9022103A90E
:106530000193FFF7A3FF40680168DDE90132CC68F1
:106540000399A04704B010BD1FB5CDE9022103A9EE
:106550000193FFF793FF40680168DDE901324C6960
:106560000399A04704B010BD07B5CDE9002101A9EA
:10657000FFF762FF40680368DDE900219B699847E7
:1065800003B05DF804FB000007B5019101A9FFF716
:1065900053FF406801990368DB69984703B05DF8D1
:1065A00004FB000007B5019101A9FFF745FF406812
:1065B000019903681B6A984703B05DF804FB00006B
:1065C00073B5019101A9FFF737FF05460820FFF7D2
:1065D000ABFD044658B16868019903685B6A984747
:1065E0000646606030B920463446FFF7A3FD2046DA
:1065F00002B070BD02482D1AED102570F7E700BFFC
:106600001077080841B10A78044B496803EBC203CC
:10661000586803689B6A184708467047107708084F
:1066200038B50C4671B10A78084B496803EBC203D0
:1066300058680368DB6A984705462046FFF77AFDED
:10664000284638BD4FF0FF35FAE700BF107708083D
:1066500001207047704700000020704700487047D5
:1066600040430030044B054A1A60054B054A1A6046
:10667000054B064A1A607047DC430030B4770808BF
:10668000784300305C77080844430030C478080839
:10669000002070474FF0FF30704700004FF0FF3090
:1066A0007047000000207047002070474FF0FF3017
:1066B00070470000002000217047000000200021EA
:1066C00070470000002070470120704770470000AD
:1066D000002070470329F7B506460D4617461C46AD
:1066E00004D8182303FB01031A793AB939F026FDBF
:1066F000092303604FF0FF3003B0F0BDD3F818C09A
:10670000BCF1000FF2D046F21B72D968ADF8002040
:10671000C1B1182202FB0562D368906923448268E4
:10672000934227D818232246394603FB0565AB69F7
:106730001868EB68184439F0E9FDEB6820462344FB
:10674000EB60D9E7052CE4D93868B7F804E000908D
:1067500080B2DCF808309042ADF804E0D9D1BDF841
:1067600004209A42D5D9D21A604620F0AFFC002806
:10677000CFD1BFE79A1A002120F0A8FC0028D1D180
:10678000B8E70000032938B504D8182404FB010435
:10679000257935B939F0D2FC092303604FF0FF3079
:1067A00038BD012B08D0022B09D003B9E2601823B1
:1067B00003FB0100C068F3E7E3681A44F6E739F029
:1067C000BDFC1623E9E700002DE9F04F1F4600232A
:1067D0008A4615462DED028B8FB054688DF8343003
:1067E000ACB914870DF11B0107AA28460BF0AAFFCC
:1067F000BAF80420A3B280469A4212D9013400B3F9
:1068000007AA0DF11B0128460BF0C2FFF0E7138F1A
:106810000DF11B0128460133138707AA0BF0B8FFBF
:106820008046BAF80630B8F1000F0AD0ABB12A8F13
:106830009A4212D3002630460FB0BDEC028BBDE861
:10684000F08FBAF80660002EF4D12C8F0CF00AF805
:106850008442EFD00BF0E4FDEDE7012309AA4046A6
:106860002946009310230AF019FF05F10803E81DDB
:10687000002208EE103A09ABD1B29B4613F9014B46
:10688000059110F9011FA14202D101320029F3D173
:106890005846FAF7C1FC10F0FF03049307D1059B9B
:1068A0000BF1FF3B013BDBB20593012304939AF804
:1068B0000130039363B19DF81B1040460BF0BCFA06
:1068C000DDED070A06F05EF980F00100C3B2039324
:1068D0009DF81B000AF042FD049B044603F10209E7
:1068E000039B002B50FA89F214BF064600260128AC
:1068F0001644F6B215D96D68BAF80220063535444B
:10690000B5FBF2F102FB11555DB1854209D2451B81
:1069100038460021EDB22E442F442A46F6B239F013
:106920001DFD039B59469DF81B50B81C45EA0312F8
:10693000049B3A705A1E059B43EA02127A70049A2D
:1069400039F0E4FC2246414607EB090039F0DEFC51
:10695000039BB3B1013D042D13D8DFE805F0180304
:10696000181F1F00DDED077AFDEEE77A17EE903A6B
:10697000ADF8203004EB0900224608A9384439F06C
:10698000C5FC09A918EE100A3AF034F853E7DDED1A
:10699000077AFDEEE77ACDED087AEBE704EB090024
:1069A000224607A9EAE700002DE9F04F064689B024
:1069B0000F461C46154642B93C222946184639F076
:1069C000CDFC012009B0BDE8F08F5B68934204D98B
:1069D0003C220021204639F0C1FC94F81990B9F10D
:1069E000000F1AD0D4F804A0A5EB0A08C84528BFA8
:1069F000C8465FFA88FBD94508D008F11A01A9EB0F
:106A0000080204F11A00214439F08EFCA9EB0B09AD
:106A100008EB0A0384F81990636004F11A086368AC
:106A2000AB421BD0A5EB030A22466B4639463046E3
:106A3000FFF7CAFE90B18245D14628BF8146824504
:106A400008D2A0EB0A030DEB09014046DAB26276E8
:106A500039F05CFC63684B446360E0E76068431BAB
:106A600058425841AEE7000003292DE9F04F804617
:106A7000894692461D462DED028B8BB004D8182313
:106A80004B43C61832795AB939F058FB09234FF0F5
:106A9000FF34036020460BB0BDEC028BBDE8F08FE5
:106AA0000433C31808EE103AB3691BB139F046FB42
:106AB0001623ECE7F3880BB905B1F580F3880BB129
:106AC000AB42F3D1182202FB098213693BB1D268B1
:106AD0009342C0F0AA809B1A9D4228BF1D461823EE
:106AE00003FB0983DB68052B00F2A18046F21B73D0
:106AF000ADF808300BF0B6FE3389ADF80C009842C3
:106B0000D4D9C01A738980B2ADF80A001BB198427B
:106B100088BFADF80A30182303FB0983D96873795D
:106B2000C1F10604AC4228BF2C461BB146F21C73CF
:106B3000ADF80830E4B202AB50462246194439F0B1
:106B4000E5FB18232D1B03FB0983DA682244DA6076
:106B5000A0D0A2441823012703FB0983DA685E69E9
:106B60000023063A7068022F06D0316C914203D39D
:106B700081424FF002075CD3C3EB031306EB83069D
:106B80007368934208D0334618EE101A4046FFF758
:106B90000BFF00283FF47EAF002D3FF47BAF777EE4
:106BA00027B3AF42504628BF2F46FBB23A46ED1BF3
:106BB000BA44009306F11A031946019339F0A6FB73
:106BC00096F819B0009B9B4508D007F11A01019B6C
:106BD000ABEB07023144184639F0A6FB009BABEB48
:106BE000030B73683B4486F819B0736006F11A030F
:106BF00008EE903A7DB102AB324618EE101A4046CC
:106C0000FFF7E2FDE8B9182303FB0983DA68196985
:106C10003A4489B91A6118213C4401FB0988D8F823
:106C20000C303B44C8F80C3034E7002557E700240B
:106C300090E70846012396E78A4294BF1A611961DA
:106C4000E9E7A842834628BFAB46A84208D9401BC3
:106C500002ABC2B2591918EE900A727639F056FB9F
:106C60005A46504602A9A5EB0B0539F04FFB726856
:106C7000DA445F4402EB0B037360BBE710B50C46CC
:106C800009220849204639F0DFFE38B994F9090095
:106C900030B1A0F13F035842584110BD0020FCE73D
:106CA0000120FAE79BB30A082DE9F84F0746894609
:106CB0001446FFF7E3FF40B939F040FA02234FF0E2
:106CC000FF3603603046BDE8F88F04F003044FF050
:106CD000000818233A1D03FB08F54646515D0029BC
:106CE00000F08680032E08F10108F4D139F026FA6D
:106CF0001723E4E718234FF0000A012203FB08736F
:106D0000C3F80CA0C5E9012AC3F810A0C3F818A065
:106D10009CB11020FFF708FA044618B11022514622
:106D200039F01CFB182303FB08739C612CB93B68EA
:106D3000414638465B68984765E03F21484639F050
:106D40004BFEDFF8D0A00446DFF8CCB0002CB9D061
:106D500094F90030002BB5D004F101092C4906222A
:106D6000484639F071FE014680B907340A222046B0
:106D70003AF050FD4FF6FE7398422CD82881262118
:106D8000204639F029FE81464C46DFE7514606226F
:106D9000484639F059FE014650B907340A222046C8
:106DA0003AF038FD4FF6FE73984214D86881E6E752
:106DB00059460D22484639F047FE01460028E3D1E6
:106DC0000E340A2220463AF025FD012803D800F0AF
:106DD00001006871D3E7182000FB0877786908B1D3
:106DE000FFF7AEF900232B7139F0A8F9162366E7F7
:106DF0003D44002C7FF47EAF7820FFF79FF9686157
:106E000000287FF477AF39F099F90C2357E700BFDA
:106E1000387708083F7708084677080810B5144601
:106E2000FFF72CFF30B939F089F9022303604FF0E6
:106E3000FF3010BD58220021204639F08FFA0BF0A8
:106E400011FD0C23584320610020F2E72DE9F04F9B
:106E50000025934691B015704A699368052B40F25E
:106E6000B98014682068A288049080B2ADF814201C
:106E700046F21B72904240F0AD80BDF814209A4259
:106E800040F0A8800D22294607A80634069539F05F
:106E900065FABDF81220ABB29A4240F29F80277883
:106EA00007F00F063F0940F0958094F8018008F044
:106EB0000F0A4FEA181808F101030AEB03090193BE
:106EC000B9F1100F00F38680524606A90BA808F10D
:106ED000030839F01BFA019BA11C44441A460BAB72
:106EE00003EB0A0039F012FA10AB0DF12C0E0DF184
:106EF000180C994409F8147CBEE80F00ACE80F00A8
:106F0000DEF800300DF10E020DF10D010BA88CF82A
:106F100000308DF80D700AF081FC48B9012E02D1C5
:106F200001340135B5E7022E0CBF02340434F8E712
:106F3000BDF80E309DF80D1013F004031ED001298A
:106F400004D190F90070B7FA87F77F098E4217D104
:106F5000032E15D154F8043B0360002211460BF0B8
:106F600067FA002FDDD0012364218BF800301C4B21
:106F70001B68186D03685B689847D2E71F46E5E712
:106F8000012E0FD1237817B11F1E18BF01275BB246
:106F90000134019000EE103AB8EEC00A0AF0C0FFCA
:106FA0000198DAE7022E09D134F9023B00EE103ADB
:106FB000B8EEC00A01900AF0B3FFF1E7032E02D148
:106FC00054F8043BF2E7042EC7D154F8043B00EE1A
:106FD000103AEFE7002011B0BDE8F08F0120FAE78A
:106FE000F02A003073B505460E460524013C14F026
:106FF000FF040CD00DF1070231462846FFF726FFAB
:1070000018B19DF80730002BF0D102B070BD0120FF
:10701000FBE700000329F8B504460D4604D8182103
:107020006943461833793BB939F088F84FF0FF3798
:10703000092303603846F8BDB369DBB90027002394
:107040003371182606FB0543586908B1FFF778F835
:1070500006FB054600237361B6692EB1304620F069
:1070600057F83046FFF766F81821002301FB054466
:10707000A361DFE704310144FFF7B4FF0028DDD14D
:1070800039F05CF816234FF0FF370360D7E70000B4
:10709000002070470020002170470000002070474A
:1070A00008B539F04BF81E2303604FF0FF3008BDE0
:1070B000032938B504D80C2404FB0104656835B9EC
:1070C00039F03CF8092303604FF0FF3038BD012B45
:1070D00008D0022B12D063B9002A05DA39F02EF855
:1070E0001623F0E7E3681A44A3689A4294BFE2606B
:1070F000E3600C2303FB0100C068E7E7A368E360DB
:10710000F7E7000008B539F019F81E2303604FF0C7
:10711000FF3008BD48680BF0CDBE00000329F8B56C
:107120000646104604D80C2202FB0166776837B980
:1071300039F004F8092303604FF0FF30F8BDD6E9B9
:1071400002516C1A9C4228BF1C4634B12246394475
:1071500039F0DCF8F3682344F3602046EEE70000E2
:1071600000F134032DE9F341CE1A1D4B8046F71090
:10717000B6F5467F03FB07F705D938F0DFFF092393
:107180000360002426E04FF4847306F1380103FB0A
:1071900007070144786B0BF08FFE0446D0B1796B82
:1071A00008460191FAF738F801990546024620464B
:1071B00039F04AFC0028E4D163572F2B0ED101355A
:1071C00087F83901FF22611906F13A044444204648
:1071D00039F04EFC204602B0BDE8F0810446F9E7E4
:1071E000E1830F3E70B506460C200D46FEF79CFF6E
:1071F000044670B10146866028460BF00BFE05463A
:10720000606030B9204600F003FB20462C46FEF7B4
:1072100091FF204670BD000012F00302F8B504464D
:10722000084606D038F08AFF1E234FF0FF35036072
:107230000FE00C23211D03FB02F615468F5957B1B1
:10724000032D02F10102F6D138F078FF1723ECE7A5
:10725000E7602846F8BD06F10801214434440BF0EC
:10726000D9FD60600028F3D138F068FF0223DCE725
:1072700000F13403C91A0D4B10B5B1F5467F4FEA42
:10728000E10403FB04F406D938F058FF0923036036
:107290004FF0FF3010BD4FF4847303FB0404606BA8
:1072A00035F0B8FB00206063F4E700BFE1830F3ED8
:1072B00013B5084601A914460BF0ACFD38B938F0F7
:1072C0003DFF022303604FF0FF3002B010BD0BF012
:1072D000F1FD58220021204639F040F8019B0020A2
:1072E0002361F2E770B50546002308464FF4847128
:1072F00005F1340601FB03F4325942B10133042B8A
:10730000F8D138F01BFF17230360002007E02E1987
:10731000328735F0DFFB706308B13434281970BD53
:10732000032910B504D80C2404FB0104606830B9AB
:1073300038F004FF092303604FF0FF3010BD0BF05D
:10734000B9FD00206060F9E74FF0FF3070470000A2
:10735000032910B504D80C2404FB0101087930B9C5
:1073600038F0ECFE092303604FF0FF3010BD012B15
:107370000AD0022B11D02BB9CB689B689342D4BFA3
:107380008B608A608868F1E78B681A44CB689B68D9
:107390009A4294BF8A608B60F4E738F0CFFE1623E0
:1073A000E1E7000091F9003010B533B138F0C6FEC6
:1073B000002402230360204610BD4FF48270FEF7C4
:1073C000B3FE04460028F6D138F0B8FE0C23036063
:1073D000F1E70000032970B50646104604D80C22D8
:1073E00002FB0166327932B938F0A8FE0923036046
:1073F0004FF0FF3070BDD6E9021295686C1A9C42BE
:1074000028BF1C4613682246194438F07FFFB36832
:1074100020462344B360EDE713B50B680C4600200B
:107420000B2B0DD881F80301081D0649FF2201909E
:1074300051F82310FEF7C4FB236801980133236041
:1074400002B010BD8C780808032970B504460D46BB
:1074500004D80C2303FB01031A7932B938F06EFE0D
:10746000092303604FF0FF3070BD0022DE681A71FF
:107470002EB130461FF04CFE3046FEF75BFE0C216D
:10748000002001FB0544E060EEE70000084608B577
:1074900031B938F053FE162303604FF0FF3008BDBA
:1074A000FEF748FE0020FAE770B50D46074E0024AF
:1074B00056F8041B2846F9F7A5FE08B960B270BD5E
:1074C00001340C2CF4D14FF0FF30F8E78C78080829
:1074D0002DE9F04F12F0030485B005460E4604D0A6
:1074E00038F02CFE1E23036009E14FF00C0A031D47
:1074F0000AFB04F9274613F809B0BBF1000F00F0AE
:10750000F080032F04F10104F2D138F017FE1723A5
:10751000E9E731462846FFF7C7FF00280BDA404667
:107520001FF0F6FD4046FEF705FEC9F80CB038F036
:1075300005FE0223D7E773493046F9F763FE30B9F9
:10754000714B41461B68586D0368DB6E98476F4965
:107550003046F9F757FE48B96B4B1B68586D0C2342
:10756000026803FB0453126FD9689047684930469C
:10757000F9F748FE48B9644B1B68586D0C23026844
:1075800003FB0453526FD968904762493046F9F7BC
:1075900039FE48B95C4B1B68586D0C23026803FB2D
:1075A0000453D26FD96890475B493046F9F72AFEF9
:1075B00050B9554B1B68586D0C23026803FB0453EC
:1075C000D2F88020D968904754493046F9F71AFE1E
:1075D00028B153493046F9F715FE68B901204A4BE6
:1075E0001B6803EB8000406E30B10C23026803FB84
:1075F0000453526AD96890474A493046F9F702FE67
:1076000048B9414B1B68586D0C23026803FB0453B7
:10761000926FD968904744493046F9F7F3FD08BBAB
:107620000C2303FB0453D3F80C80374BD3F800A092
:10763000DAF854000368D3F8943098470190DAF8E8
:1076400054000368D3F8903098470090DAF854005B
:107650000368D3F890A0D04703464046DDE90021F7
:107660001FF060FD31493046F9F7CCFD98B9264B43
:1076700003AA02A91B68CDE90200D86B03689B69C5
:10768000984740B10C20039B029900FB04501A4616
:10769000C0681FF047FD0C2606FB0456F3689A6885
:1076A000AAB91B7B002B14BF0C27022738F046FD1C
:1076B0000760F6682EB130461FF02AFD3046FEF70F
:1076C00039FD0C20002300FB0454E36017E0002385
:1076D000C9F80830012389F80430384605B0BDE800
:1076E000F08FA9441020FEF71FFD8046C9F80C005A
:1076F00000287FF40EAF38F021FDC0F800A04FF055
:10770000FF37EAE704780808F02A00301078080804
:1077100018780808237808082D78080838780808A9
:107720004778080856780808A58408086678080885
:1077300070B5044616460D4619B112B191F90030E4
:107740003BB938F0FBFC16234FF0FF3403602046B2
:1077500070BD58220021304638F000FE2846F9F767
:107760005BFD012895F9003003D12F2B04D10024B3
:10777000EDE72F2B08BF013529462046FFF794FE81
:10778000002803DA38F0DAFC0223DDE70D49284649
:10779000F9F738FD044618B94FF400433361D6E7D2
:1077A00009492846F9F72EFD044640B9074B1B68E6
:1077B000586D0368D3F8903098473061C7E7044BA1
:1077C0003361D4E766780808A5840808F02A0030F9
:1077D000A08601004FF0FF30704700004FF0FF30EF
:1077E000704700004FF0FF30704700004FF0FF304F
:1077F000704700004FF0FF3070470000486810B538
:107800000C4618B135F006F90023636010BD000086
:1078100010B50446806818B103682146DB6C9847B0
:10782000204610BD2DE9F04399B00368054688460F
:107830009B6902AA9847074620B10024204619B048
:10784000BDE8F0830C20FEF76FFC04460028F4D05E
:107850008560069835F09AF8064630B92046FFF75D
:10786000D7FF2046FEF766FCE7E72B6841463A461D
:107870002846D3F800903B46C847431C014603D135
:10788000304635F0C7F8E9E72B68324601902846C4
:10789000D3F80880069BC047069B019998422B6845
:1078A00028465B6801D09847EAE79847069BC4E9F9
:1078B0000036C3E738B500254FF0FF3304463030BB
:1078C00040F8043C40F81C5C40F8185C40F8145C3C
:1078D00016F014FF04F16400FEF798F90C492046F5
:1078E000C4F88C50C4F89050C4F89450C4F858515F
:1078F000C4F85C51C4F860510AF0E8FC054B1A6802
:1079000012B1054819F03EFC20461C6038BD00BF8E
:107910006C7A0808304800306C790808084699B13C
:10792000C81FC3B2102B0ED810280CD8DFE800F007
:10793000090B090B0B0B0B090B0B0B0B090B0909A3
:10794000090000207047012070470000F7B590F94A
:10795000023004460E46032B15D100F12A073846A3
:107960000AF0BEF8054670B901230DF1070138464B
:107970008DF807300BF086F90DF10701A01C8DF88A
:1079800007500BF07FF921782046FFF7C7FF30B191
:107990000022052130460CF08DF8C4F80C010025BA
:1079A000B3EE0E1AF1EE040A4FF4E37094ED090AF7
:1079B000A56005F079F9B7EE007A238A84F858506B
:1079C000C7EE007A013B9BB2C72B84BFC82323823A
:1079D000C4ED5B7A03B0F0BDB02303FB010191F865
:1079E000A90010B1D1F8983013607047B02303FBA1
:1079F000010191F8AA0010B1D1F89C3013607047D2
:107A0000B02303FB010191F8AB0010B1D1F8A03015
:107A1000136070472DE9F843B02384460F4603FBFB
:107A20000103D3F8B82022B9D3E9300150EA0103A9
:107A30002CD0B02606FB07C6B6F8600000283FD061
:107A4000204DDFF88490A0FB0545D6E93023134391
:107A50001ED042375CF8270003F094FD074619F06A
:107A6000CBFB14EB090245F14904D3194FF47A75A5
:107A700044F10004A3FB053205FB0422D6E930459E
:107A8000001B61EB0501181842EB0101BDE8F8830A
:107A9000F06D492310EB090043F10003071945EB92
:107AA000030419F0A1FBD6F8B8104FF47A73401A0A
:107AB000C01944F10004A0FB030103FB0411E5E736
:107AC0000146E3E700840C24B0F5F790B02303FBF4
:107AD000010310B5B3F86040ACB1423150F8210059
:107AE00003F050FD094B4FF47A72A4FB0313084CCA
:107AF000091943F14903081843F10003A0FB0201EF
:107B000002FB031110BD20462146FBE700840C2434
:107B1000B0F5F79000EBC101C1F84C21A1F850314C
:107B200070470000435609B2022B0BD1038D5B074F
:107B300015D50C4B00EBC100C0F84C312E23A0F83A
:107B4000503170470B2B08DC092B08DD00231A4647
:107B500000EBC100C0F84C21F1E70F2BF6D02E232B
:107B6000014AF5E7AC7B08083C7A080838B500EB19
:107B70008105D5F80C31FBB100EBC104B4F85021FC
:107B8000D2B11A681846126A9047D5F80C31B4F889
:107B9000502119688242CD6828BF0246D4F84C11A2
:107BA0001846A847D4F84C310344C4F84C31B4F813
:107BB0005031181AA4F8500138BD00002DE9F043E7
:107BC000425C85B004460E46172A04D80123934030
:107BD000834A134204D104EB8607D7F80C310BB962
:107BE000002552E03825012305FB064585F81931AB
:107BF00019F0FAFAD5F814318046C31AB3F5966F26
:107C000025D995F81831774A0133DBB2082B08BF24
:107C1000002385F818313825D7F80C0105FB0645F7
:107C2000036895F818115B6A52F821109847D7F845
:107C30000C0100210368DB6D9847C5F8148194F9A5
:107C40001330002B0BDD31462046FFF76BFF94F914
:107C50001330002B03DD31462046FFF787FFA35783
:107C60000B2B16D00F2B25D00A2B34D14FF4CC7010
:107C7000FEF75AFA054640B1B022D7F80C3121463A
:107C800002FB0642583201F041FB284605B0BDE830
:107C9000F0834FF4BC70FEF747FA05460028F4D095
:107CA000B022D7F80C31214602FB0642583200F0D0
:107CB00015FEEAE74FF4C870FEF736FA05460028CD
:107CC000E3D0B022D7F80C31214602FB06425832ED
:107CD00001F068F8D9E704EBC603B3F85031002B84
:107CE0007FF47EAFD7F80C014FF03808036808FB2B
:107CF000064908FB06481B6909F58D799847B0F5D8
:107D0000005F28BF4FF4005085B2002D3FF468AFEC
:107D1000D7F80C0103685B699847A35DC1B2013BCA
:107D2000012B0AD898F818212E4B53F8223094F9D9
:107D300013208ABBB3F5164F37D2238D13F0010FF2
:107D4000A35DA3F1110314BF4FF461324FF4E1229C
:107D5000012B1ED898F81801224B53F8203093427B
:107D600017D1484602F010FB98B1A3574FF49D601D
:107D7000112B0CBF4FF001084FF00208FEF7D4F9A9
:107D80000546002881D0B022CDF8008002FB0642D3
:107D90001FE0013DADB2B8E7B3F5E13FCDD3228D91
:107DA000500702D4B3F5613FC7D14846039102F0B2
:107DB000EBFA03990028C0D04FF49D60FEF7B4F9A8
:107DC000054600283FF461AFB022002302FB0642C3
:107DD0000093D7F80C315832214603F007FA54E7E4
:107DE0000042C0001C7A0808F8B504460D46B026CB
:107DF00019F0FAF90023074606FB054629462046F6
:107E000086F859304FF6FF73A6F88630A6F888300A
:107E1000FFF7D4FE90B1012204EB051386F8592038
:107E200005F14202194644F82200DF644FF47A63F8
:107E3000A1F85030BDE8F84003F048BCF8BD0000A0
:107E4000054B1B682BB1C16A4A1C02D0184604F0CE
:107E50005DBC0020704700BF4448003031B990F845
:107E6000123122B143F0010380F81231704723F040
:107E70000103F9E710B40C4611461A463CB9D0F894
:107E8000080120B103685DF8044B5B6918475DF891
:107E9000044B704770B490F90660044613467F2E79
:107EA0000DD00A46F1B270BCFFF7E4BF172B0AD021
:107EB000D4F8080138B1036870BC5B69184790F9C1
:107EC0000030122BF2D170BC7047000070B5CE7834
:107ED0009EB00C467122712E4FF00001054601A89C
:107EE00028BF712638F03AFA04F10C0101A8324695
:107EF00038F00CFA9DF806206E2A04D80DF107011F
:107F00002846FFF7C7FF1EB070BD000013B504463A
:107F100001917AB9D0F8080160B103689B6998476C
:107F200040B1D4F8080101990368DB6902B0BDE8EB
:107F30001040184702B010BD10B590F900300C4643
:107F40000BB9002010BDD0F8080118B9002301209A
:107F50002370F7E703681B6998470028F1D1F5E71C
:107F60002DE9F0479146CA0704460F461E4605D440
:107F700049461A46BDE8F047FFF78CBFD0F85431A8
:107F8000002B44D0C7F34105D4F854A14FF0B408F6
:107F9000FF089AF8003008FB05A808F10608002B36
:107FA00040D1D4F8543140465F700123D4F85411C5
:107FB00003FA05F20B78134332460B70494638F04A
:107FC000A5F9B32ED4F8543141D86A1C05EB450508
:107FD000C5EB05159A70D4F8543106EB85059D80E4
:107FE000D4F854118A78DAB1012308789340013B20
:107FF000984215D18A8820460631FFF74BFFD4F806
:10800000542100239370D4F85421137008E040F2F7
:10801000D621012034F0FAFCC4F854010028B1D173
:10802000BDE8F0879AF80120BA4209D1EB40DB079E
:10803000B7D532464946404638F058F90028EFD0C7
:1080400000238AF80230D4F854211370A9E71A7873
:108050000F2AC5D104229A704FF43472D4F85431E7
:108060009A80BDE770B5CE78AEB00C46B622B62E7B
:108070004FF000010546684628BFB62638F06EF975
:1080800004F10C016846324638F040F99DF80130A1
:10809000B42B06D80DF102029DF800102846FFF718
:1080A0005FFF2EB070BD000070B58A7A05464B7A2E
:1080B0000C4643EA0223CA7A43EA02437B2B05D0EB
:1080C000E92B07D1BDE87040FFF7CCBFBDE8704099
:1080D000FFF7FCBE002695F81121F3B29A420CD9A5
:1080E00003F1420255F8220028B1EB561BB1036898
:1080F00021465B6A98470136EDE770BD174B10B417
:10810000136049BBB0F92030002B0DDD07EE903A2B
:108110009FED137AF8EEE77A67EE877AC2ED007A80
:1081200001205DF8044B7047D0F8083113B190F886
:10813000591049B990F9000010B900231360EFE716
:10814000431E58425841ECE7196818468C6A11469C
:1081500023465DF8044B18470020E2E7CDCCCC3D28
:108160006F12833A90F811318B4209D9083130F9F6
:108170001100002804DDC828A8BFC82080B27047BD
:10818000C820704759B990F92A3043B990F90030A6
:108190002BB1D0F8080110B10368DB6A1847002042
:1081A0007047000008B5034690F90E0040B1D3F8BF
:1081B000080128B103681B6B984780F00100C0B22A
:1081C00008BD000031B9D0F8080118B103681146A4
:1081D0009B6C184700207047B02301FB030191F806
:1081E000B40010B1D1F8B030136070472DE9F743F7
:1081F000984690F8733104460E46DDF8289073BB1C
:10820000B02505FB010595F8AC7017B3EB6F136053
:1082100001AAD5F88030C9F80030FFF76FFF70B1C0
:10822000DDED017A9FED0F7AD9F8003067EE877A9D
:10823000FCEEE77A17EE902A9B1AC9F80030B021BD
:1082400001FB064494F8AD303BB1D4F8A430C8F833
:108250000030384603B0BDE8F083034BF7E7002752
:10826000F7E700BF00007A44000020417FB5B0234B
:1082700003FB010393F88430EBB105AB03AA009331
:1082800004ABFFF7B3FF80B1DFED0C7A9DED030A7D
:1082900020EE270A04F0C2FCFDEEC07A17EE900A29
:1082A00030B180B207B05DF804FB4FF6FF70F9E71C
:1082B00048F6A040F6E71846F4E700BF0000C842C1
:1082C0002DE9F04F2DED068B90F8B43095B088462F
:1082D000856E9FED56AA002B00F09B800A23D0EDFF
:1082E0002C7A6B4308EE103AB8EEC88AA7EECA8A19
:1082F000BDEEC88A90F8AA30002B00F08D80D0ED3A
:10830000279A90F8AB30002B00F0898090ED289AE6
:1083100090F8A930002B00F08580D0ED268A866C7D
:108320004FF47A7790F87231A6FB077690F859905F
:1083300023B1B9F1010F28BF4FF00109DFED3C6A0D
:10834000002190ED1D7AD0ED1E7A27EE267A036F7C
:1083500067EEA67AC26E0493BCEEC77AB0F886B018
:10836000FCEEE77AB0F888A0059217EE103A9CB2BE
:1083700017EE903A9BB2029390F88A300393FFF77E
:1083800075FF049B69EE8A9A29EE0A9A059A0A9368
:108390000A23FCEEE99A18215D43029B68EE8A8A63
:1083A0000992ADF83630BCEEC99A039B07AAFCEEE1
:1083B000E88AADF84E008DF8393018EE103A404694
:1083C0000B95CDF83A3019EE903AADF830B0CDF8C3
:1083D0003E3019EE103AADF832A0CDF8423018EE2A
:1083E000903AADF83440CDF8463000238DF83890FF
:1083F000ADF84A30ADF84C303423CDE900311E23BE
:10840000CDE907760CF0B0FC15B0BDEC068BBDE8ED
:10841000F08F08EE103A6DE7DFED069A71E79FEDF9
:10842000059A75E7DFED038A79E700BF00007A441B
:108430000000C842000000002DE9F043A1B004464E
:108440000D4618F0D9FE05AB0027814688460093FB
:1084500003AA04AB2946204603970497FFF7C6FEFC
:10846000A323CDF84F90CDF853808DF84C30952351
:108470008DF857508DF84D3058238DF84E3094F8C4
:1084800072313BB1B02303FB054393F85930012B04
:1084900000F2BD80B02303FB054393F85930B026AA
:1084A0008DF8583006FB0546F36DCDF85930B6F817
:1084B0006030ADF85D3096F88A308DF85F30B6F8F0
:1084C0008630ADF86030F36ECDF86230336FCDF8A2
:1084D0006630B36ECDF86A30736FCDF86E30B36F1F
:1084E000CDF87230D6F89430CDF87630039BCDF8C5
:1084F0007A30484B1B6893F810315A1B5342534152
:108500008DF87E3004F01EF913A9332203F020FC0D
:1085100006AA294620460697079708970997FFF766
:1085200065FA07AA294620469FED3B6AFFF768FADD
:1085300008AA29462046FFF74FFA09AA29462046ED
:10854000FFF74AFE9DED067ADFED346AA32327EE9E
:10855000067ADDED087A8DF82830952367EE867A65
:10856000CDF82B90B4EEE67A8DF829305923CDF86A
:108570002F808DF83350F1EE10FA8DF82A30B6F8CE
:10858000883058BFB0EE667AADF83430BCEEC77AAA
:1085900017EE103A9DED077A27EE067AADF83630E1
:1085A000B4EEE67AF1EE10FAF4EEE67A58BFB0EEE9
:1085B000667AF1EE10FABCEEC77A58BFF0EE667A32
:1085C00017EE103AFCEEE77AADF8383017EE903A35
:1085D000ADF83A30049B0F9396F8A8308DF84030F0
:1085E00004EB051304EB0514DB6CCDF84130B4F853
:1085F0005030ADF84530099BCDF8473004F0A2F873
:1086000023220AA903F0A4FB21B0BDE8F0830123D3
:1086100045E700BF304800300000C84200FF7F47F8
:108620002DE9F84F435604460D46072B0BD063B98E
:10863000B02101FB050484F859304FF6FF73A4F80C
:108640008630A4F88830BDE8F88F90F81231CB401E
:10865000DA07F8D400EB81090FB2D9F808311BB959
:10866000BDE8F84FFFF7C0BB90F91330002B01DDD8
:10867000FFF77CFAD9F808014FEA051803689B68F0
:108680009847834618F0B0FD0646BBF1000F6DD148
:10869000A044D8F84C30C31AB3F57A6FD3D94FF051
:1086A000B00A59460AFB05405246583037F056FE8C
:1086B0000AFB05424FF6FF734FF47A6182F8585077
:1086C000A2F88630A2F88830C8F84C60A8F850109C
:1086D000615D172903D83B4BCB40DB070CD4D9F89D
:1086E000080100283ED1B023002203FB0543C9F84E
:1086F000082183F8592002E0012382F8593004EB65
:108700000712B2F85030F52B58D992F85210B3F541
:10871000FA6F01F1010182F8521017D292ED157A29
:1087200007EE903AB5EEC07AF1EE10FA85BFF8EE9A
:10873000E77ADFED256AF8EE677A67EEA67A84BFFE
:10874000DFED226AE7EE267AC2ED157A2046FFF7C2
:1087500077FB00283FF477AF29462046BDE8F84F65
:10876000FFF76ABE03685B689847BCE74FF0B00943
:1087700009FB054999F8C83053B100234FF47A72C8
:10878000D9E93001F8F7FEF80023064689F8C83029
:1087900004EB080304EB0512D96C711AA2F850100F
:1087A000B022DE6402FB054292F85920012AA6D9C4
:1087B00094F87221002AA2D19E64A0E7002182F8D9
:1087C0005210ABE70042C0000AD7A33C48E17A3F11
:1087D00013B5044600F130014FF4856201A814F08E
:1087E00001F800212046FFF71BFFD4F8083113B130
:1087F000012384F8113101A814F016F802B010BD5D
:10880000014B1868704700BF3048003001207047A6
:10881000002070477047000070470000014B0120A6
:108820000B607047CDCC4C3E012070470120704753
:1088300001207047002070477047000000207047FB
:10884000704700000620704700487047DC7B08082E
:108850007047000010B50446FDF76CFC204610BDC3
:1088600070B586B004460E46122201AD002128469E
:1088700037F074FD0221642303228DF804108DF873
:1088800006300D238DF80F1004218DF807300123D9
:108890008DF80B208DF8101007218DF8162094F814
:1088A00066218DF812108DF80820D11800228DF85D
:1088B0000D308DF8116084F86611E95C01330A44CB
:1088C000122BD2B2F9D1606829468DF815201322F7
:1088D0000368DB68984706B070BD000010B5044619
:1088E00002F034FE0F4B0021204623600E4B84F82B
:1088F00066111A681B79C4F86D2184F87131C4F8C7
:10890000681184F86C1184F85A10FFF7A9FF03214D
:108910002046FFF7A5FF18F067FC6E30C4F8680129
:10892000204610BDEC7B08083037080870B586B0CB
:1089300004460D46164600211422684637F00EFD07
:108940000223072103228DF8003064238DF80B10D9
:1089500006218DF802300F238DF807208DF80330A3
:1089600001238DF80C100A218DF8142094F866214B
:108970008DF80D108DF80420D11800228DF80930E3
:108980008DF80F308DF80E6084F866118DF8115057
:108990001DF8031001330A44142BD2B2F8D16068D9
:1089A00069468DF8132015220368DB68984706B0E6
:1089B00070BD00008B18002030B5DD790C46002119
:1089C00065F307009D7965F30F205D7965F3174026
:1089D0001D7965F31F60DD7865F307019D785B788D
:1089E00065F30F2163F31741A35C63F31F6141EC4F
:1089F000100B30BD881800238A5C10B5C47864F36E
:108A000007038478407864F30F2360F3174362F31D
:108A10001F6300EE103A10BD8B18002010B5DC78F3
:108A200064F307009C785B7864F30F2063F31740CE
:108A30008B5C63F31F6010BD8B184FF000005B78F8
:108A400063F307008B5C63F30F2080B27047000074
:108A50002DE9F04F2DED068B90F85D3083B0044684
:108A6000402B40F0F080032500269FED7B8B9FED8F
:108A70007C9B9FED7DAB94F85E30AB4240F2DD8095
:108A800004EB050A05F102089AF85F709AF8609005
:108A9000012F33D1D4F80CB0424604F15F012046D7
:108AA000FFF7BAFFCBF80400D4F80CB0AA1D20469B
:108AB000FFF7C2FFABF80800E3689AF8672083F875
:108AC00032209AF86830E26813F0010F14D09AF857
:108AD00069300321DD0751700AD5E2680421980747
:108AE000517005D55907E2684CBF06230523537022
:108AF000013609EB0805BEE75770F9E7022F30D1C0
:108B000004F15F01424620460191FFF753FF20EE3A
:108B1000080BE36805F10A020199204620EE090BD3
:108B2000BDEEC00B83ED050AFFF744FF20EE080BF6
:108B3000E36805F112020199204620EE090BBDEE13
:108B4000C00B83ED060AFFF735FF20EE0A0BE36842
:108B5000BDEEC00B83ED040AE56818F045FB2866FE
:108B6000C6E7082F2DD104EB080393F85F30DB072D
:108B7000BED504F15F01E768EA1C2046DFED3C7AD0
:108B80000191FFF737FFEA1D204687ED070AFFF73F
:108B900031FF20EE270AE368204683ED080A02F041
:108BA00005FD05F10B0201992046FFF723FFB1EE09
:108BB000400AE368012283ED0F0AE36883F850203E
:108BC00096E7092F10D1DFED2B7AAA1D04F15F0182
:108BD0002046FFF70FFF20EE270AE368BCEEC00A2D
:108BE00010EE102ADA8583E70C2F82D104F15F01A1
:108BF000AA1D2046FFF7FEFEF0EE407A05F10A02BC
:108C00002046FFF7F7FEE36837EE800A05F112020F
:108C1000F6EE007A204620EE270A83ED110AE76877
:108C2000FFF7E8FE012387ED120AE2681E4482F88E
:108C30005230E26882F853305BE7052E4FF00100B6
:108C400002D0E3685870002003B0BDEC068BBDE88D
:108C5000F08F00BFAFF30080F8C1631ADCA54C4071
:108C600000000000D01263410000000000005940E5
:108C7000E02E65420000C84290F85A30013B052BB7
:108C800004D8DFE803F0101B1F233944022908D160
:108C900040F20123A0F85A300023A0F8623180F896
:108CA000643100207047022380F85C1080F85A304D
:108CB00090F86431194480F86411F2E7032380F8D6
:108CC0005D10F3E7042380F85E10EFE7B0F862313F
:108CD000C218013382F85F109BB290F86421A0F8AB
:108CE0006231114490F85E209A4280F86411D8D81D
:108CF000052380F85A30D4E7062380F85F1180F806
:108D00005A3090F864318B42CBD1FFF7A1BE0023DB
:108D100080F86011EDE7000038B5044618F064FAF9
:108D2000054694F86C31042B1BD8D4F86821824294
:108D300017D22344002220466E3593F86D11FFF7B9
:108D4000F5FD94F86C3103222046234493F86D110D
:108D5000FFF7ECFD94F86C31C4F86851013384F8E6
:108D60006C310025606803681B69984750B16068E2
:108D700003685B699847C1B22046FFF77DFF28432F
:108D8000C5B2EFE7284638BD062070470048704757
:108D90003C7C08087047000010B50446FDF7CAF98E
:108DA000204610BD10B5044602F0D0FB104B2360E6
:108DB000002384F8603084F86C30C4E91933AA23A6
:108DC00084F8713141F24423A4F87231A36893F915
:108DD00013305BB160680E2206490368DB68984770
:108DE0006068222204490368DB689847204610BD6A
:108DF000D87C0808447C0808537C080870B5B0F893
:108E00007921044690F87431B0F875511A44D0F8BD
:108E1000811102F06FFC2A2D40F0B480E36804F168
:108E20006D06B4F87F211A81E368D4F881215A6075
:108E3000E56818F0D9F99FED817B28660125D4F803
:108E40007520D4F87930E16843EC162B26EE076BD9
:108E5000BDEEC66B81ED056AD4F87D20D4F8813073
:108E6000E16843EC162B26EE077BBDEEC77B81ED58
:108E7000067AD4F88520D4F88930E1689FED717BBB
:108E800043EC162B26EE077BBDEEC77B81ED047A03
:108E9000E36883F85C50E368D4F88D209A65E36852
:108EA00094F8AE2083F83220D4F8953007EE903A4B
:108EB000D4F8993000EE103A20EE000AA7EEA70A87
:108EC000B7EEC00A35F060FCB7EEC00BE3689FED6B
:108ED0005F7A83ED110AE268316B9164E26882F88F
:108EE0005250E26882F85350B36BE26807EE903A52
:108EF00067EE877AFCEEE77AC2ED207AE36894F8B1
:108F0000AE2083F88420D4F86D30E268C3BBD4F877
:108F10007130222B0FD81F2B30D8102B16D00F2BCF
:108F200007D9122B03D8102B03D004230FE0142BE6
:108F3000FBD001230BE0322B02D003D8302BF8D129
:108F4000062304E0443B012BEFD9F2E703235370DF
:108F500094F85A3043F0010384F85A3094F85A30A8
:108F60009A07C3F3400065D5E268E16D526891420B
:108F700026D123F0030384F85A305BE00523E6E7AB
:108F80005570E5E7632D1DD0AE2D4ED1D4F8752078
:108F9000DFED2F6A07EE102AE36827EE267ABCEE93
:108FA000C77A17EE102ADA85D4F87920E36807EE3D
:108FB000902A67EEA67AFCEEE77A17EE902A1A86D8
:108FC000002037E0D4F87D2004F16D05D4F881301D
:108FD0002046E16843EC172BF7EEC77BC1ED077A1B
:108FE000D4F88520D4F88930E16843EC172BF7EEEC
:108FF000C77BC1ED087A02F0D9FA2A6A6B6AE06889
:1090000043EC172BF7EEC77B0122F1EE677AC0ED38
:109010000F7AE36883F85020D4F88131E36594F83F
:109020005A3043F0020384F85A3094F85A0010F092
:10903000010093D170BD00BFAFF3008000000000BD
:10904000D0126341000000000000594000007A4443
:109050000000C8420823054A01F00100490800B198
:109060005140013BF8D10846704700BF2083B8ED5E
:10907000F8B5054614465618A6420AD014F8010B56
:109080001F0A5840C1B22846FFF7E4FF87EA0003F1
:10909000F2E71846F8BD000038B590F86C30044689
:1090A000013B082B06D8DFE803F010191D26374CCA
:1090B00050586000AA2904BF012380F86C300023B7
:1090C00080F88D3184F88E3104E0442904D10223E4
:1090D00084F86C30002038BD0023F9E71229FBD159
:1090E0000323F5E7042380F8741180F86C3080F8CE
:1090F0008D310023E6E7B0F88D311B2BECD8C21878
:10910000013382F871119AB2A0F88D3190F8743160
:109110009342DFD80523DBE7B0F88D31FF2BDBD896
:1091200090F874011A1A0133224482F86D109AB231
:10913000A4F88D31B4F8793103449A42CADB06238E
:10914000C6E70723C0F86D11C2E7D0F86D3103EB15
:1091500001210823C0F86D11BAE7D0F86D3103EB97
:1091600001410923C0F86D11B2E7D0F86D51002319
:1091700000F2711205EB016580F86C3090F8741103
:10918000C0F86D51FFF774FF04F16D020346B4F8A7
:1091900079112046FFF76CFF854204D12046BDE8D7
:1091A0003840FFF72BBEA36E0133A36692E70000A1
:1091B00073B58368044693F91330F3B118F014F8CB
:1091C00094F860300546032B17D8626E824214D2A1
:1091D000144AC835666852F8231008460191F8F71A
:1091E0001BF8336802460199DB683046984794F8CB
:1091F00060306566013384F860300025606803687C
:109200001B69984750B1606803685B699847C1B2B1
:109210002046FFF741FF2843C5B2EFE7284602B0DA
:1092200070BD00BFC07C080806207047004870472A
:10923000287D080801207047014B01200B60704712
:109240000AD7A33D836F01200B607047836893F9B1
:10925000133023B1006E031F58425841704701205C
:1092600070470000836F13F4746F0CBF012000205F
:109270007047000010B50446406E33F0CBFB20462B
:1092800010BD000010B50446FFF7F4FF2046FCF7C0
:1092900051FF204610BD00008268436F92F90E20F6
:1092A00003F42073022A04D0A3F5207358425841D6
:1092B0007047B3F5207F08D0064B1B685B6D93F8B1
:1092C0009C3023B990F87C00704701207047002043
:1092D000704700BFF02A003007B5836893F9133058
:1092E0007BB1026E042A0CD0C3684FF0030C1978CE
:1092F00004230131CDE9003C90F85A300248FAF7D6
:109300003BFB03B05DF804FB2C7D080810B5044658
:1093100002F01CF90B4B23600B4BE3660023236721
:1093200084F87E3017F060FFE2680123A0662046D3
:1093300082F88530A268128D920744BFE26882F8F5
:109340002C3010BDF07F0808607D080838B5B0F8F3
:10935000843040F6AE720446C3F30C03934200F02F
:109360002F810AD840F6A172934200F01A8140F68C
:10937000A77293423AD0002000E140F6BC729342BB
:1093800000F0418141F214729342F4D1B0F886208A
:10939000D0F8881002F0AEF9D4F8903007EE903A89
:1093A000D4F8943007EE103AD4F8983000EE103A22
:1093B000E368B4EE407AF1EE10FA37FE000AF4EEFC
:1093C000407AF1EE10FA37FE800ADFEDA27AB4EEB1
:1093D000E70AF1EE10FAC0F21281012283F851205F
:1093E000E46835F05BFA84ED100AC4E7B0F88C301D
:1093F0004FF6FF7299B2914205D0C2681381C368DB
:10940000D0F888205A60B4F886202046D4F8881016
:1094100002F070F9E56817F0E7FEDFED8F7A286655
:10942000D4F8AC3007EE103AB4EEE77AF1EE10FA69
:109430003BDDE268012520465363E368D4F8B020A1
:109440009A63D4F8B430E26807EE903AF1EE677AA6
:10945000C2ED0F7AE36883F85050E16802F0D2F869
:10946000B4F8CE300A21E268DFED7C6A4B43C2F8E3
:109470008030B4F8DA20E36807EE102AB8EE477AB5
:1094800027EE267A83ED117AB4F8DC20E36807EE44
:10949000902AF8EE677A67EEA67AC3ED127AE3684F
:1094A00083F85250E36883F85350D4F89020D4F8EE
:1094B00094309FED627B43EC162BB4EEC76BF1EE5C
:1094C00010FA3CDDE1689FED5F5B43EC172B9FEDED
:1094D0005F6B27EE057B27EE067BBDEEC77B81ED3C
:1094E000057AD4F89820D4F89C30E16843EC172B27
:1094F00027EE057B27EE067BBDEEC77B81ED067A66
:10950000D4F8A020D4F8A430E16843EC172BD4F8A9
:10951000A830B7EEC77B012207EE903A77EE677A64
:109520009FED4F7A67EE877AFDEEE77AC1ED047A18
:10953000E36883F85C20E368D4F8A8209A6594F87F
:10954000CA30FF2B1CBFE26882F8323094F88E30AC
:1095500003F00F03082B09D8DFE803F005111411FD
:10956000171A14171A00E36801225A7094F88E3003
:10957000012013F0400F0ED0E368587038BDE36847
:109580000322F2E7E3680422EFE7E3680622ECE750
:10959000E3680522E9E71B06F0D5E36802225A706A
:1095A000ECE7B0F88620D0F8881002F0A3F8E36862
:1095B000B4F89420DA85E368B4F896201A86DAE6DF
:1095C000B0F88620D0F8881002F094F8D4F89430DF
:1095D000A26F6367D4F8983082EA030111F4746FC4
:1095E00009D0E16803F4746302F474621D480978D9
:1095F0000131FAF7C1F9D4F89830A367BBE600202F
:1096000083F85100BAE7B0F88620D0F8881002F04D
:1096100071F894F88E00E36830BB83F88400E36847
:10962000C3F88000E368C3F88C00E368C3F88800DF
:10963000E368C3F89000A1E7AFF3008000000000EA
:10964000006A08C1F8C1631ADCA54C4000000000A4
:10965000D012634100000034005043C80AD7A33B36
:109660000000C842707D080894F8902083F8842098
:109670004FF6FF72B4F8BD30934216BF0A220023A2
:109680005343E2689FED2F7BC2F88030D4F89420DA
:10969000D4F89830E56843EC162BB4EE476BF1EE46
:1096A00010FA42D0D4F89C00D4F8A01041EC160B6C
:1096B000B4EE476BF1EE10FA37D0D4F8A400D4F82A
:1096C000A81041EC160BB4EE476BF1EE10FA2CD05B
:1096D000B4F8B8004FF6FF71884226D09FED1B6B9F
:1096E00043EC172B27EE067BBDEEC77B85ED237A77
:1096F000D4F89C20D4F8A030E16843EC172B27EE77
:10970000067BBDEEC77B81ED227AD4F8A420D4F885
:10971000A830E1689FED0F7B43EC162B26EE077B0C
:10972000BDEEC77B81ED247A25E60020C5F88C00CC
:10973000E368C3F88800E368C3F89000E36883F83F
:1097400054001BE7BBBDD7D9DF7CEBBD0000000098
:1097500000408F400000000000408FC02DE9F84F0E
:1097600090F87E3004460D46013B082B06D8DFE812
:1097700003F0404B4F575B63677DB200242908D14B
:10978000012380F87E300023A0F888310020BDE856
:10979000F88F90F88F314FB2DFF8F0914FF0060854
:1097A0005E1C00F5C57B0344F6B2032EB24680F87A
:1097B0008F61A8BF4FF0030A83F88A715246594659
:1097C00059F8040B37F040F978B9042E06D1303F30
:1097D000092FDBD9002384F88F31D7E7D6D93E2D66
:1097E000F8D1012384F89031F4E7B8F10108E5D10C
:1097F000F0E7402903D1022384F87E30C6E75229DE
:1098000040F09A800923F7E70323A0F88210F3E7DA
:10981000B0F88210042301EB0525A0F88250EBE795
:109820000523A0F88410E7E7B0F88410062301EBC5
:109830000525A0F88450DFE70723A0F88610DBE7B2
:10984000B0F8861001EB0525ADB2AB07A0F8865045
:109850000CBF08230023072D80F87E3096D8002304
:1098600080F87E30236F013323678FE7B0F88831AB
:10987000FF2B98BFC21803F1010398BF82F888102C
:109880009BB2B0F88620A0F88831083A9342FFF6E0
:109890007DAFB3F5807F4FD800220221843003F0E2
:1098A000DDFA0221024604F1860003F0D7FAB4F88B
:1098B0008610024604F18800083903F0CFFA00232D
:1098C00084F87E30B4F882308342CBD12046BDE8A4
:1098D000F84FFFF73BBDB0F88821FE2A2CD883183B
:1098E00001320A2992B283F88810A0F888217FF407
:1098F0004DAF8318002183F8881090F888303A2BF8
:109900001AD1466EC6B100F18A01053A304637F0E9
:109910009BF8054680B9304633F07CF8236E6566C7
:10992000042B06D8DFE803F0030A0C1A28000123F1
:10993000236617F059FCA06600235DE70223F7E7D2
:1099400094F85A300133DBB2032B84F85A30F0D943
:1099500003232366002384F85A30EAE794F85A3048
:10996000A2680133DBB284F85A3092F90C200AB1B4
:10997000022BDED90423DBE701F05AFF40F261122B
:109980004FF4801101F040FFD3E700BFC07F08080B
:109990004068112201490368DB6818479C7D08086C
:1099A00038B58368054693F90E303BB3406F10F429
:1099B000007412D1EB68124819780131F9F7DCFF15
:1099C000EB68104819780131F9F7D6FF2846FFF700
:1099D000DFFF85F87C40002038BDC30506D5EB6865
:1099E000094819780131F9F7C7FFF4E710F080044E
:1099F00004D1EB68054819780131F4E70120EBE761
:109A0000B07D0808D07D0808F17D08080A7E0808A6
:109A100010B504460548F9F7AFFF13226068044902
:109A20000368BDE81040DB68184700BF307E0808B7
:109A3000447E0808F0B504464068002585B00368F8
:109A40002E461B6998470746BD420BD0606801351A
:109A500003685B699847C1B22046FFF77FFE064363
:109A6000F6B2F1E7A36893F91320FAB1226E042A43
:109A700000F0938017F0B8FBE36D0546834215D2E2
:109A8000A36E03F5FA63834213D2E06EF7F7C4FBCB
:109A90000746606803681B6A9847B84206D3606847
:109AA0003A46E16E0368DB689847A566304605B024
:109AB000F0BD94F89031002BF8D0636E2BBB236E71
:109AC000042B22D8DFE803F00337444A6100D4E9CD
:109AD0000232606804F164051278134493F922207D
:109AE000036803921B6E98473E493F4B039A012837
:109AF00008BF0B463D49284600934FF4613314F0EC
:109B00005DFE013001D100236366606E0028CDD078
:109B1000F7F782FB0546606803681B6A9847A8420E
:109B2000C4D360682A46616E0368DB6898470023E7
:109B300084F89031BAE7D4E902322D4904F1640087
:109B400012781344012293F9223014F037FED8E73B
:109B500094F85A20274B53F8222009E0A36893F980
:109B60000C30012B0AD0022B0CD0002BCDD1224A75
:109B7000224904F1640014F021FEC2E794F85A204F
:109B80001F4BE8E704232366BFE701F051FE96224E
:109B90004FF4801101F038FEB7E793F90E30022B35
:109BA00084D1184B1B685B6D93F89C301BB101236B
:109BB00084F87C307AE794F87C30002B3FF476AF61
:109BC000636F9B057FF572AF17F00EFBE36D0546E3
:109BD0008342BFF46BAF05F57A752046FFF718FF97
:109BE000E56563E75D7E0808587E0808657E08081D
:109BF000887E0808D87F0808E17E08087FBB0A082D
:109C0000B47F0808F02A003006207047836893F973
:109C100013302BB1D0F8B804B0FA80F04009704787
:109C200001207047004870474080080870470000D6
:109C300090F8BC34822B08D81A0611D4033B012BB0
:109C40000ED9084B01200B607047FF2BF9D1054B53
:109C50000B60836893F91300B0FA80F040097047F5
:109C6000014BEFE7AE47613E8FC2F53D00207047E4
:109C7000704700000120704710B50446FCF75AFAFF
:109C8000204610BD10B40022D0F8B834012101FAEA
:109C900002F41C420AD0C1680748097850F8222013
:109CA000013106485DF8044BF9F766BE0132142A0B
:109CB000EDD15DF8044B704784820808488008089D
:109CC00013B5044601F0F4FC94F88C3463B102F04F
:109CD00039FDE36805491A7804F28D430132009397
:109CE00004F2AB4302F05EF902B010BD70800808C8
:109CF00010B586B0044601F0F9FCC8B31622002165
:109D0000684636F02BFBA3238DF8003095238DF8A1
:109D100001305D238DF8023017F06EFAE368CDF85C
:109D20000710CDF803001B788DF80B30B4F86A30BB
:109D3000ADF80C3094F887308DF80E3094F86F3011
:109D40008DF80F30B4F86C30ADF81030D4F8B8346A
:109D5000CDF81230B4F86E34442B04BF94F88F3031
:109D60008DF80E3002F0EEFC1622694601F0F0FF8D
:109D700006B010BD1FB5044601F0B8FC68B3102250
:109D80000021684636F0EAFAA3238DF800309523C7
:109D90008DF801305E238DF8023017F02DFAE3685C
:109DA000CDF80710CDF803001B788DF80B3094F830
:109DB0005A308DF80C3094F85B308DF80D3094F8F3
:109DC0005C308DF80E3094F85D308DF80F3002F075
:109DD000B9FC1022694601F0BBFF04B010BD0000C1
:109DE00030B591B0044601F081FC002831D002F07A
:109DF000A9FC054617F000FAD4F87230164A0E9303
:109E0000D4F86E300D93D4F86A300C93B4F8603007
:109E10000B93D4F866300A93D4F862300993B4F8FF
:109E20005E300893B4F85C30079394F85B30069387
:109E300094F85A300593E3681B780493074B019319
:109E4000074BCDE9020100932846064B064902F074
:109E5000BDFA11B030BD00BF95800808D780080852
:109E6000E480080888800808D28008082DE9F047B7
:109E70008CB00C4601F03AFC002847D017F0BCF932
:109E8000002507460E464FF0A30A4FF095094FF004
:109E90005A08A279EBB29A4238D98DF815201822C7
:109EA0002168013502FB0343CDF80F101A7FB4F986
:109EB00004108DF804A08DF805908DF80680CDF87B
:109EC0000770CDF80B60ADF813108DF81620996867
:109ED000DA68CDF81710CDF81B205A691969CDF84A
:109EE00023209A69CDF81F10CDF827205A7F8DF8CE
:109EF0002B209A7FDB7F8DF82C208DF82D3002F0FF
:109F000021FC2A2201A901F023FFC2E70CB0BDE821
:109F1000F08700002DE9F04792B00C4601F0E6FB17
:109F200000287CD017F068F95B2322684FF0A30962
:109F30008DF806304FF09508636800274FF05C0AF3
:109F40000D46CDF8133006462389CDF80B10ADF839
:109F50001730A37ACDF80F208DF81930E37A8DF8F9
:109F600004908DF81A30237B8DF805808DF81B3016
:109F7000CDF8070002F0E6FB182201A901F0E8FE87
:109F8000E27AFBB29A424AD904EB43138DF81C9053
:109F90008DF81D8001378DF81EA0CDF81F60CDF81B
:109FA000235019695A69CDF82710CDF82B20DA69AA
:109FB0009969CDF833201A6ACDF82F10CDF83720E3
:109FC00093F824208DF83B2093F825208DF83C2031
:109FD00093F827208DF83D2093F8291093F8282036
:109FE00042EA0122ADF83E2093F82A208DF8402065
:109FF00093F82B208DF8412093F82C208DF84220E7
:10A0000093F82D208DF8432093F82E308DF84430AE
:10A0100002F098FB292207A901F09AFEB0E712B0DE
:10A02000BDE8F087C1F302710139C9B204299ABFB2
:10A03000014B585C002070477C82080830B5039CB7
:10A040000A44914209D011F8015B18782844C0B243
:10A050001870257828442070F3E730BD2DE9F041D1
:10A060000446406886B01D4603688846BDF83060E7
:10A0700017461B6A984706F1080398424FF0000004
:10A080003AD3B5238DF813700DF10F0704228DF824
:10A09000103062230DF112018DF80E008DF80F00C3
:10A0A00020468DF811300DF10E0300978DF81280C7
:10A0B000ADF81460FFF7C2FF3246294620460097EC
:10A0C000FFF7BCFF6068062204A90368DB689847B5
:10A0D0006068324629460368DB6898476068012259
:10A0E0000DF10E010368DB6898476068012239466C
:10A0F0000368DB689847012006B0BDE8F0810000E6
:10A1000013B50446406803681B6A9847072806D9B8
:10A110000023062120461A460093FFF79FFF02B056
:10A1200010BD00001FB590F88B34052B05D9FFF743
:10A13000E7FF002005B05DF804FB02238DF80C104A
:10A140008DF80D2006210093012203ABFFF786FF57
:10A15000F0E70000F0B5044640681D4685B003688E
:10A160000F4616461B6A98470A280FD90323012277
:10A1700006212046009303AB8DF80C708DF80D601E
:10A180008DF80E50FFF76AFF05B0F0BD0020FBE729
:10A1900090F8CE340133DBB280F8CE342BB990F88E
:10A1A0006D2490F87214FFF7D5BF70470A2938B5AF
:10A1B0000546184663D004D801290AD0022964D084
:10A1C00038BD0D29FCD1032AFAD14FF48024012394
:10A1D0002EE0122A35D8012AF2D9931E102BEFD87F
:10A1E00001A454F823F000BF4FA204085BA20408A6
:10A1F0002DA20408C1A1040867A204089DA20408B6
:10A20000C1A10408C1A10408C1A10408C1A1040896
:10A21000C1A10408C1A10408C1A10408C1A1040886
:10A22000C1A10408C1A1040873A2040801232024C9
:10A23000834239D1D5F8B83423EA0403C5F8B834D9
:10A24000BEE7202ABCD14FF400440523F0E795F87F
:10A25000D24484F001030224EAE795F8D24484F062
:10A2600001030424E4E795F8D24484F001030824B0
:10A27000DEE795F8D24484F001031024D8E7092AD8
:10A2800010D00B2A9CD18024DFE7102A01D0152A98
:10A2900096D1AB684FF480749B7BC9E701234FF4E0
:10A2A0000054C5E74024D0E72846FFF753FFD5F810
:10A2B000B8342343C5F8B834012385F8D0347FE798
:10A2C0002DE9F04385B0541C9146002602AFC0F83A
:10A2D000E034A40097F82830054680F8D8246A4670
:10A2E00080F8E434E31DC0F8D414013CDB08C0F866
:10A2F000DC644068A4B2A2EBC303884602689D46B2
:10A30000126A02AB7B60904704F1090292B290425C
:10A3100018D3414603AA08EBC9097B680296494550
:10A3200004D051F8080B42F8040BF8E701348B22F3
:10A3300006212846A4B20094FFF790FE0C37BD46D4
:10A34000BDE8F0833046F9E70C23092213B5044633
:10A35000062100930A4BFFF781FE16F045FF94F8A3
:10A360008034C4F87C040133064884F88034E36800
:10A370001978013102B0BDE81040F9F7FDBA00BF0D
:10A380006C830808F480080810B50023082482783C
:10A39000082A0ED8DFE802F00B051217202B3747EA
:10A3A0004D00622902D10223837002E08370B52937
:10A3B00001D0002042E083780133F5E70323C17028
:10A3C00083700171F5E704238370C378194403791E
:10A3D000C9B2C1701944F4E7052302790170837092
:10A3E000C3780B44DBB2C37013440371E1E7062367
:10A3F0008370C37819440379C9B2C170194400232A
:10A4000001714370D5E7C378027819440379C9B262
:10A41000C1701944437801710133DBB29A42437031
:10A42000C7D10723C0E7C27884708A42C1D0837045
:10A43000ADE7027983708A42A9D1012010BD0000E6
:10A44000002307B504220A210093FFF707FE03B09B
:10A450005DF804FB1FB5C368044680681978FDF7F2
:10A4600081FE012306210822ADF80A300023ADF851
:10A4700008002046ADF80C3002AB0091FFF7EEFD6E
:10A4800004B010BDB0F86E24083201F033B90000FA
:10A4900090F8BC0400F0FD00A0F180035842584140
:10A4A000704700002DE9F04F85B006460C469246F5
:10A4B00002AF9B46FFF7ECFF20B900200C37BD46EA
:10A4C000BDE8F08F3046FFF7ADFD00238046C7E9B9
:10A4D000003300F10F0370681FFA88F523F00703BB
:10A4E000ADEB030D03681B6A0DF10809984705F1F0
:10A4F00010039BB29842E0D37C6001233C460835B0
:10A500003B70424687F801B0ADB203CC029004A87C
:10A510000391514635F0FAFE4B468A220621304619
:10A520000095FFF79BFDC9E72DE9F04F2DED028B5C
:10A5300090F8721495B00446052945D190F86D2421
:10A54000012A01D000201FE090F85A30062B0CD0D1
:10A550000A2BF7D190F85B30092B30D00B2BF1D1BF
:10A56000D0F8B83423F0800326E090F85B30312B2C
:10A570001ED00ED8162B00F08A81242B4FF000003D
:10A5800000F05081092B0ED015B0BDEC028BBDE858
:10A59000F08F3E2B00F07681712BD3D1D0F8B834F8
:10A5A00023F4803308E084F8732484F8D004EBE7C4
:10A5B000D0F8B83423F48043C4F8B834C2E7D0F8F4
:10A5C000B83423F04003F7E7062910D190F86D2442
:10A5D000242A00F0F18000F28880082A00F07D81B2
:10A5E0006AD8002A00F07481012A00F0558194F89D
:10A5F00072540A2D40F0FC8194F86D34092B00F060
:10A60000E3810B2B00F0EB81042B40F01C82012333
:10A6100004F2AB4704F28D462A4684F88C3404F1E8
:10A620007801384636F024FA1E2204F15A013046E9
:10A6300036F01EFAE3683A46C248197833460131CB
:10A64000F9F79AF90822C049384636F0FDF9D8B929
:10A650002A46BE49304636F0F7F960B994F8BC3462
:10A66000802B1EBFD4F8B83443F48033C4F8B83418
:10A67000802384F8BC340A22B549304636F0E4F928
:10A6800010B9812384F8BC340822B249384636F028
:10A69000DBF900287FF456AF0922AF49304636F087
:10A6A000D3F900287FF44EAF822384F8BC34D4F869
:10A6B000B83443F40023B9E0162A98D1836893F99B
:10A6C0000C50022D00F0E38090F85A30AB4200F0BD
:10A6D000DE80034603F85A5F08250095FFF7BEFCAD
:10A6E000D4F8B83443F4805394E0712A00F00F8119
:10A6F0008B2A00F033813E2A7FF479AFD0E902CE75
:10A700009EF80030634493F90F20002A00F0BA80CD
:10A7100000F15A0505AE00F192092B46B0462868B3
:10A72000083555F8041C37464D4503C73E46F6D15B
:10A73000286800213860084642FA01F5ED0703D584
:10A7400001291CBF0130C0B201310729F4D14200F8
:10A7500094F85D5000264FF0080A03922246B54255
:10A760007BDD9EF8001092F85E70614491F90F0055
:10A77000F100384110F0010065D0012F59D094F854
:10A780005B900398A9F1030B9BFBF0F094F8BCB429
:10A79000C0B2BBF1040F82F85F0001D8022F4FD086
:10A7A00082F860902144D1F8620040F00100013647
:10A7B0000832C1F86200D2E700238268A0F85A305C
:10A7C00092F901305E1C08D090F85C1099421EBFCF
:10A7D00080F85C300123A0F85A3092F90D30B4F8BB
:10A7E0005A0013F1640F1BD094F966209A4217D0D7
:10A7F00040F0020084F86630A4F85A00242204F1E4
:10A800005A03062120460092FFF728FCD4F8B834FA
:10A8100043F48063C4F8B834012384F8D03491E65B
:10A820000028EBD1D4F8B83423F48063C4F8B834EA
:10A83000AAE64FF0030082F85F7082F86000B1E78B
:10A8400082F860A0AEE7214482F85F0082F86000E1
:10A85000D1F8620020F00100A9E719463C224046E9
:10A86000039335F043FD039B60B1ED003E220621CA
:10A87000204604350095FFF7F1FBD4F8B83443F4D3
:10A880000063C7E7D4F8B83423F4006394E6D4F83F
:10A89000B83423F480538FE6B0F86E34082B10D10F
:10A8A00090F88B34052B02D9FFF72AFC4AE60344C3
:10A8B00090F85B2090F85A1093F85C30FFF776FC24
:10A8C00040E690F85C3090F85B2090F85A10F5E77D
:10A8D00090F85A3080F88B3434E6D0E90213B0F89F
:10A8E0005A201B78083331F913309A4207D1C36DCF
:10A8F000012B04D1D0F8B83423F001035CE62046E4
:10A90000FFF7A8FDD4F8B83443F0010382E7B0F8AC
:10A910005C30002513F001030CD02823A0F85C5014
:10A92000009300F15A03FFF799FBD4F8B83443F4CD
:10A9300080336FE7D0F8B82422F48032C0F8B8240E
:10A9400000E600BF70800808148108081D8108080F
:10A9500028810808338108083C810808B0F86E5443
:10A9600000F15E06B84F4FF00008043DEDB2042D33
:10A970007FF63DAED6F80090B94512D13379F3B1E8
:10A98000072305AA394620468DF81480FFF78AFD73
:10A99000012384F8D034D4F8B83443F48033C4F8B5
:10A9A000B83449462046FFF73DFB00283FF4CAADC6
:10A9B000C0F1FC0304301D440644EDB2D7E7D4F8DF
:10A9C000B83423F48033EAE7B4F86E343C2B02D079
:10A9D000442B7FF4B7AD2046FFF78AF9B2E5B4F80F
:10A9E0006E341C2B7FF4AEAD2046FFF7C3F9A9E50A
:10A9F000022D19D194F86D34102B09D1A36893F965
:10AA00000E3003B304F15A012046FFF72FFA99E5FF
:10AA1000152B18D1A36893F90E30A3B104F15A0194
:10AA20002046FFF777FA8DE50D2D0AD1D4F86C3466
:10AA3000864A23F0FF03934205D12046FFF7D0F961
:10AA400080E5012D03D02046FFF7A2FB7AE594F8BC
:10AA50006D24122A17D8012A1BD9931E102B18D83F
:10AA6000DFE813F02600AF00D3001700E4002C014C
:10AA7000170017001700170017001700170017001E
:10AA8000170017003402202A00F01582302A00F047
:10AA9000888294F8CE040130C5B284F8CE54002DDB
:10AAA0007FF450AD2B4601212046FFF753FB49E5CB
:10AAB00094F8D23433B1D4F8B83443F00203C4F874
:10AAC000B83457E0D4F85A102046FFF7DBFCD4F82E
:10AAD0005A30D4F85E200A21C4F87834E368DFEDF8
:10AAE0005C6A9A61E368D4F862205A61A368E268FC
:10AAF0001B8D13F0100F14BFD4F86630D4F86A30F1
:10AB000093FBF1F313610122E36883F85C20D4F82E
:10AB10006A30D4F86600E1681B1A07EE903AF8EE46
:10AB2000E77A67EEA67AC1ED167AE36894F8CF1457
:10AB30005970D4F86E1094F8CD3407EE101A134300
:10AB4000B8EE477A84F8CD34E36827EE267A83EDB1
:10AB5000117AD4F87210E36807EE901AF8EE677A6B
:10AB600067EEA67AC3ED127AE36883F85220E368B1
:10AB700083F85320E36893F8543063B116F034FB44
:10AB8000D4F8C834C01AB0F5C87F40F23682E36802
:10AB9000002283F8542094F8CD34D9077FF5D2AC45
:10ABA0009A07C3F340007FF5CDACD4F87414D4F801
:10ABB000782491427FF4C6AC23F0030384F8CD34AB
:10ABC000E2E4D4F85A102046FFF75CFC94F8D23443
:10ABD00023B1D4F8B83443F0040370E794F85F105D
:10ABE000E26811F0010F0BD094F85E30032B05D111
:10ABF0008A0700D5042384F8CF34BBE7022BFAD0B0
:10AC0000012384F8CF345370B4E70023D4F85A10EA
:10AC1000204684F8D134FFF735FCE368B4F86620A9
:10AC2000DA85E368B4F864201A86A3E7D4F85A10EA
:10AC30002046FFF727FC94F8D234E26863B1B4F8F9
:10AC40006230138196E700BF0100032000031C005F
:10AC50006F12833AACC5273794F86510CB0728D517
:10AC600094F86430032B22D18F0700D5042384F895
:10AC7000CF3494F8D1341BB1E368B4F88620DA8578
:10AC8000E36894F8892083F8322094F8CF34012BBC
:10AC90007FF670AFE56816F0A7FA2866E368D4F887
:10ACA0005A205A60E368B4F862201A8162E7022BE6
:10ACB000DDD0012384F8CF345370DAE70123D4F8D0
:10ACC0005A1020461FED1E8A84F8D234FFF7DAFBB3
:10ACD000D4F85A30D4F872200A21C4F8C034C4F829
:10ACE0007834E3689A61E368D4F876205A61A368FF
:10ACF000E2681B8D13F0100F14BFD4F87A30D4F82B
:10AD00007E3093FBF1F313610122E36883F85C204A
:10AD1000D4F87E30D4F87A00E1681B1A07EE903A36
:10AD2000F8EEE77A67EE887AC1ED167A94F86E301D
:10AD3000052B00F2BE80DFE803F0BCBC039BB4BC73
:10AD4000E36802225A70E26801251FED3E0A53783B
:10AD500084F8CF3494F8CD3443F0010384F8CD3433
:10AD6000D4F8823007EE903AF8EE677A67EE887A88
:10AD7000C2ED117AD4F88620E36807EE902AF8EE47
:10AD8000677A67EE887AC3ED127AE36883F85250E7
:10AD9000E36883F85350E36894F8712083F8322015
:10ADA000D4F89620D4F85A3007EE902AC4F87434B8
:10ADB000F8EEE77AE36867EE887AC3ED077AD4F8AD
:10ADC0009A30E66807EE903AF8EEE77A27EE800AC6
:10ADD00001F00EFF86ED080AE36883F85050D4F8BE
:10ADE0008A20E36807EE902AF8EEE77A67EE887A21
:10ADF000C3ED0D7AD4F88E20E36807EE902AF8EEC2
:10AE0000E77A67EE887AC3ED0E7AD4F89220E36889
:10AE100007EE902AF8EEE77A67EE887AC3ED0F7AAC
:10AE2000E36883F85150D4F89E20E36807EE902A37
:10AE3000F8EE677A27EE888A83ED108A94F8CD348D
:10AE400043F0020384F8CD3494F8D1343BB1E36885
:10AE5000B4F8A620DA85E368B4F8A6201A86E56877
:10AE600016F0C2F92866E368D4F85A205A6081E6E1
:10AE70000322E3685A7094F86F309E0742BFE3687C
:10AE800004225A7094F86F305D0642BFE3680522D1
:10AE90005A7094F96F30002BBFF655AFE368062265
:10AEA00050E794F86F105948F8F766FDE3680322FD
:10AEB00048E7E36846E72046D4F85A10FFF7E2FA7D
:10AEC00094F8653098077FF555AEEBE694F8D234E8
:10AED00023B1D4F8B83443F01003F0E5D4F85A1095
:10AEE0002046FFF7CFFAD4F86E209FED498A07EE8F
:10AEF000902AD4F85A309FED470AF8EE677AC4F8E2
:10AF00007434E36867EE887AC3ED077AD4F8723058
:10AF1000E56807EE903AF8EEE77A27EE800A01F04E
:10AF200067FE85ED080A0125E368204683F8505046
:10AF3000D4F85E20E36807EE902AF8EEE77A67EE31
:10AF4000887AC3ED0D7AD4F86220E36807EE902A80
:10AF5000F8EEE77A67EE887AC3ED0E7AD4F86620C9
:10AF6000E36807EE902AF8EEE77A67EE887AC3ED99
:10AF70000F7AE16800F046FBE36883F85150D4F89B
:10AF80007620E36807EE902AF8EE677A67EE887A13
:10AF9000C3ED107A94F8CD3443F0020384F8CD3435
:10AFA000E8E5D4F85A102046FFF76CFA94F85F20D1
:10AFB00002F00702022A84F8BC2413D8AAB1D4F8FC
:10AFC000B83423F40063C4F8B834D4F8B834302269
:10AFD0000121204623F40073C4F8B8340023FFF79E
:10AFE000B9F8C7E5D31E012BEFD90B4B0B491B68F2
:10AFF000186C03681B689847E7E7D4F8C424D4F8B2
:10B00000C0349A427FF49EAAC5E500BF4681080875
:10B010000AD7233CACC52737F02A00305A810808EC
:10B020007FB505460E46FFF733FA98B168680024ED
:10B03000CDE9024403681B6A98470F280CD90823FE
:10B040008B220621284600936B44ADF808400396F6
:10B05000FFF704F804B070BD2046FBE713B5836822
:10B06000044693F91330002B4BD0406803681B6AE9
:10B0700098470D2845D9D4F8B834082B05D194F851
:10B08000D23413B10023C4F8B83494F88A345A1C6B
:10B0900084F88A24162B00F2A180DFE803F00C4428
:10B0A0004C144A484E121A263B40327E5052555795
:10B0B000636A32929500072201212046FFF732F899
:10B0C00074E02022F8E7204602B0BDE81040FFF708
:10B0D00017B894F8BC34FF2B13D100233022012180
:10B0E00000932046FEF7BAFF60E0A36893F90C30A6
:10B0F000022B08D000231622062120460093FEF7DB
:10B10000ADFF02B010BDD4F8B83423F48053C4F8B6
:10B11000B834F6E70023242200930621E1E7002358
:10B120003E220093F9E7002308220093F5E702226C
:10B13000C2E70322C0E70622BEE71222BCE70422D0
:10B14000BAE709220A21B8E70B22FBE7A36893F9C3
:10B150000E3023B9D4F8B83423F48073D7E7102223
:10B160000221AAE7A36893F90E30002BF2D0152232
:10B17000F6E794F88C345BB9194B1B685B6D93F858
:10B180009C302BB9204602B0BDE81040FFF758B9FB
:10B19000D4F8B83423F40073B9E72046FFF778F900
:10B1A000034658B10F492046FFF73AFF0028A8D1BF
:10B1B00094F88A34013B84F88A34A2E77122009023
:10B1C000ABE703220D2178E7032308220649204636
:10B1D00000934FF40023FFF773F8E7E70023EAE753
:10B1E000F02A003001000320D482080810B504467C
:10B1F00000F0ACF9114BE16823604FF47F43A06885
:10B20000A4F88A3441F6FF73C4F8B834FF2384F8F5
:10B21000BC349DF8083084F8CC34012384F8CF3452
:10B2200084F8D13484F8D334002309781A46FCF723
:10B2300071FC2046FFF712FF204610BD1C83080852
:10B240002DE9F843044615F0CFFF0546D4F88434C1
:10B25000B4F88824C31A93426AD32046FFF7FEFE4F
:10B26000D4F8B834C4F88454002B36D094F8D224DF
:10B2700082BB13F0170F2DD04FF49673A4F88834C7
:10B2800060684FF0000808260368C14647461B69FE
:10B290009847B0F5005F28BF4FF4005085B21FFA01
:10B2A00088F39D4240F2D880606803685B699847E4
:10B2B0000028C0F2D180C3B20621000280B294F807
:10B2C0006C24082A3ED8DFE802F042384852637402
:10B2D00095B2B90040F2EE23D0E74FF4FA63A4F838
:10B2E0008834A36893F91230002BC9D094F87324E2
:10B2F000002AC5D194F88024042AC1D8D4F87C044B
:10B3000041F288322D1A9542BAD9554A1268526DC7
:10B3100092F89C20002AB3D1012B05D0022BAFD18B
:10B3200094F8D034002BABD02046FFF70DF8A7E7F8
:10B33000D4F8B834002BA3D1D3E7622B05D1022374
:10B3400084F86C3408F10108A9E784F86C74B52B13
:10B35000F8D194F86C340133F2E7032284F87234A4
:10B3600084F86A3484F86C2484F86B34EAE70422A5
:10B3700094F86B1484F86D3484F86C2494F86A247F
:10B380001A44D2B284F86A240A4484F86B24D9E7B8
:10B39000052294F86B14A4F86E3484F86C2494F8A5
:10B3A0006A241A44D2B284F86A240A4484F86B24CA
:10B3B000C8E794F86A2494F86BC41A4484F86C14AF
:10B3C000D2B284F86A24624484F86B24B4F86E2400
:10B3D000024492B2B2F5826FA4F86E2404D9A4F8A4
:10B3E0006E7484F86C746AE7A4F87074002AA9D1AA
:10B3F0000723A5E794F86A2494F86B141A44D2B290
:10B4000084F86A240A4484F86B24B4F87024B2F5F2
:10B41000826F3CBF121982F85A30B4F87034B4F815
:10B420006E2401339BB29A42A4F8703490E794F8EA
:10B430006A2484F86C649A42D3D183E794F86B242D
:10B4400084F86C749A427FF47DAF2046FFF76CF865
:10B45000002818BF814675E74846BDE8F88300BF5D
:10B46000F02A00300320704737B50546406814467F
:10B47000019168B103681B6A9847A04208D96868BF
:10B48000224601990368DB6803B0BDE830401847E5
:10B4900003B030BD034608462DE9F041DB688CB0AF
:10B4A0001A7822B1012A2AD00CB0BDE8F08193F8B5
:10B4B0008510B3F87C50D3F8788093F88440D3E9B2
:10B4C00022ECD3E92476D3F898308DF82E10192188
:10B4D00009932323ADF82A208DF82C20ADF82850AD
:10B4E0008DF82D40CDE90328CDE9003103AA7F2155
:10B4F000CDE905ECCDE9077609F036FCD4E793F801
:10B50000841093F88520B3F87C40D3F87880D3E991
:10B5100022E5D3E92476D3F898308DF82E20E22264
:10B52000099300238DF82D108021ADF82A308DF875
:10B530002C30ADF82840CDE903382323CDE905E5CB
:10B54000CDE90032CDE9077603AAD5E710B5044668
:10B550000B48C4E90212C4E9000364224FF4FA71F3
:10B5600004F1180008F00EF9E2680023204682F882
:10B570005130E26882F85230E26882F8533010BDF0
:10B58000BC83080810B590F83C3013B9C3685868FC
:10B5900010BD846C0CB9806BFAE74FF47A7200230B
:10B5A000D0E91001F5F7EEF92044F1E738B5C568A8
:10B5B0000446DFED137A2DED028B95ED088A28EE17
:10B5C000278AB0EE480A32F0FFF9D5ED077A27EE68
:10B5D000800A85ED0D0AB0EE480AE56832F09EFF5C
:10B5E0000022D5ED077A27EE800A85ED0E0AE36882
:10B5F000DA630022E36883F85020BDEC028B38BD8B
:10B6000035FA8E3C10B5D1ED0D0A0C4691ED0E0ABF
:10B6100033F018F9DFED077A20EE270A01F0E8FA97
:10B6200004F1340084ED080A01F0F4FC84ED070A0B
:10B6300010BD00BFE02E6542F0B5C4684FF0380C75
:10B64000174E87B02578846836686F1C0CFB054E52
:10B650000368766D9EF819E15B6BCDE90412BEF1CB
:10B66000000F12D00CFB054494F8184198470D4B7D
:10B6700053F824300097CDE90103DDE904120A4BA9
:10B68000304611F04FF907B0F0BD9847074BCDE9B0
:10B690000070DDE90412304611F044F9F3E700BF11
:10B6A000F02A00301C7A0808788308089A83080872
:10B6B00000B58FB0332201A9FFF7BEFF01F042F8B9
:10B6C00001A900F05DFC0FB05DF804FB00B58FB080
:10B6D000332201A9FFF7B0FF01A90348F8F74CF99D
:10B6E0000FB05DF804FB00BF858008088068FCF798
:10B6F000A7BB00002DE9F341836B044688468B42CB
:10B7000075D001238163D0E9047680F83C3057EA94
:10B71000060320D0C3685B78012B1CD900220023CC
:10B72000C0E9042315F060FDE56C3223226DC5F1FC
:10B730001905E0640544B5FBF3F55D43636DAB4269
:10B7400019D1B4F85830042B11D80133A4F858306B
:10B75000236D0BBB15E0606830B1036891B29B6F3D
:10B76000984707460E46DDE715F046FDF9E7954296
:10B77000EED02565ECE700236565A4F85830002A73
:10B7800038D1E368A0681978FCF7ECFCC8223221B4
:10B7900000B201F0BDFA2065236D04F1180005EB3D
:10B7A00053024FF47A75B2FBF3F25A43D4E9101303
:10B7B0006A43521843F10003CDE90076C4E910232F
:10B7C00007F0E4FFE3680122C3E91A01E36883F8A4
:10B7D0007020E3685B78934209D94FF47A720023B2
:10B7E000D4E91001F5F7CEF8A8EB0000A06402B090
:10B7F000BDE8F0814FF47A7123682046DB6CB1FB21
:10B80000F2F1C9B29847A3E710B503680281194362
:10B810004368013301604360044B1B685C6DA162A7
:10B82000596D406888855B6DDA8510BDF02A00305F
:10B83000004870473448003070B5732204464FF416
:10B8400000010E48FFF7E0FF0D4E0E4B1D683378E8
:10B850003BB9686D042221464830FAF7B1F901235B
:10B8600033706B6D2A2283F846206B6D93F89C3001
:10B870001BB92146044815F085FC70BD34480030E2
:10B8800040480030F02A00300C84080810B58322AC
:10B8900004464FF080610948FFF7B6FF084B1B686C
:10B8A0005B6D93F89C303BB92146064812F09CFF33
:10B8B0002146054815F066FC10BD00BF3448003035
:10B8C000F02A0030208408083C840808002307B5CB
:10B8D0000093012301F054F803B05DF804FB00006D
:10B8E00038B514460D4659220021204634F036FD65
:10B8F000A323601D04222370952363708023A3700B
:10B900002B78E3706B782371D5F80210FAF758F9A9
:10B91000D5F8061004F109001022FAF751F9D5F80C
:10B920000A1004F119004022BDE83840FAF748B97E
:10B9300038B514460D462C220021204634F00EFD69
:10B94000A3232370952363707023A37015F054FC18
:10B95000C4F80300C4F8071004F10C002B7810227F
:10B96000E372D5F80E10FAF72BF9D5F8121004F19E
:10B970001C001022BDE83840FAF722B910B598B083
:10B98000044601AAFFF7ACFF592201A92046FFF7A0
:10B990009DFF18B010BD000010B58CB0044601AA80
:10B9A000FFF7C6FF2C2201A92046FFF78FFF0CB03E
:10B9B00010BD00002DE9F0414FF023088AB0064683
:10B9C0000F464246002101A810EE105A10EE904A90
:10B9D00034F0C4FCA3238DF8043095238DF8053092
:10B9E00020238DF8063015F007FC1022CDF8070053
:10B9F000CDF80B100DF10F003946CDF81F50CDF8E2
:10BA00002340FAF7DDF8424601A93046FFF75EFF12
:10BA10000AB0BDE8F0810000F0B58DB00C460546D7
:10BA200017460021302268461E4634F097FCA323B7
:10BA30008DF8003095238DF801304C238DF80230BD
:10BA400015F0DAFBA37F3022CDF8030028468DF8ED
:10BA50000B30E37FCDF8071069468DF80C3094F871
:10BA600020308DF80D708DF80F30A38B8DF80E609F
:10BA7000ADF810302368CDF812306368CDF8163079
:10BA8000A368CDF81A30E368CDF81E302369CDF8ED
:10BA900022306369CDF82630A369CDF82A309DF8AD
:10BAA00048308DF82E309DF84C308DF82F3000F056
:10BAB0004FF90DB0F0BD000070B54B2694B00446B0
:10BAC0000D463246002101A834F048FCA3238DF82E
:10BAD000043095238DF805303B238DF8063015F0A2
:10BAE0008BFB4022CDF80700CDF80B100DF10F00B5
:10BAF0002946FAF765F8324601A92046FFF7E6FE27
:10BB000014B070BD2DE9F04F8DB0934606464FF04E
:10BB100064089DF858700193FAF726FC04463946EC
:10BB2000FAF75EFB39465FFA80F92046FAF758FBD0
:10BB300004F1300AC0B2394600FB08AA2046FAF7E1
:10BB40004FFB1322C5B2002107A834F007FC08FB05
:10BB50000940019BA322D0ED1B7A3946CDF8133062
:10BB6000FDEEE77ACDF80FB08DF817708DF80C2048
:10BB7000952217EE903AD0ED1C7A8DF80D206B22AD
:10BB8000FDEEE77AADF818308DF80E2017EE903AFA
:10BB9000D0ED1D7A2046FDEEE77AADF81A3017EEAB
:10BBA000903AADF81C30DAED027AFDEEE77A17EE46
:10BBB000903AADF81E30DAED037AFDEEE77A17EE33
:10BBC000903AADF82030DAED047AFDEEE77A17EE20
:10BBD000903AADF8223008FB0543D3ED187AFDEE1C
:10BBE000E77A17EE902AD3ED197AFDEEE77AADF8F1
:10BBF000242017EE902AD3ED1A7AFDEEE77AADF8FD
:10BC0000262017EE903AADF82830FAF7E9FAC3B2D9
:10BC10003946204608FB034393F831308DF82A302B
:10BC2000FAF7DEFAC0B2232203A908FB004430462B
:10BC3000E36FCDF82B3000F08BF80DB0BDE8F08F3E
:10BC40002DE9F3410546002415F0D6FA07460E46C5
:10BC5000FAF78AFB8046E3B298F816209A4207D991
:10BC600000933A46334628460134FFF74BFFF2E78C
:10BC700002B0BDE8F081000038B5104B0025044645
:10BC8000416403630E4B436340F62273C0E90155E0
:10BC90000387483012F032FD04F18C00656612F023
:10BCA0002DFD0849204606F011FB074B1A6812B11A
:10BCB000064815F067FA20461C6038BDF086080873
:10BCC00000860808008808084448003054840808A2
:10BCD00090F83A00003818BF0120704738B590F846
:10BCE0003A30044673B10025EBB204EB8303D86B02
:10BCF00003685B6C984730B9013594F83A20EBB291
:10BD00009A42F1D8002038BD38B590F83A30044650
:10BD10007BB10025EBB204EB8303D86B03689B6C0B
:10BD2000984730B9013594F83A20EBB29A42F1D8ED
:10BD300038BD0120FCE70000027B436E520703D5AB
:10BD4000181E18BF01207047023B584258417047E7
:10BD50002DE9F7430024064688469146274696F883
:10BD60003A00E3B298420AD906EB83050097002314
:10BD70004A464146E86B013400F002FEEFE703B0AB
:10BD8000BDE8F0832DE9F04F054683B01C46084618
:10BD900095F9123002AF1146BBB304F10A03EA462B
:10BDA00022464FF00008DB0803340126C346AAEB05
:10BDB000C303A4B29D46A3230DF108098DF80830F2
:10BDC000952389F802000DF10B0089F8013034F059
:10BDD0009DFA95F83A205FFA88F39A420FD905EB5D
:10BDE0008300CDF800B0012322464946C06B00F025
:10BDF000C7FD002808F1010808BF0026E9E7D5467D
:10BE000030460437BD46BDE8F08F0126F8E7000054
:10BE10002DE9F7430024064688469146274696F8C2
:10BE20003A00E3B298420AD906EB83050097012352
:10BE30004A464146E86B013400F0A2FDEFE703B04B
:10BE4000BDE8F08338B50446002594F83A20EBB2FB
:10BE50009A4207D904EB83030135D86B03685B680A
:10BE60009847F2E738BD000038B50446002594F83D
:10BE70003A20EBB29A4207D904EB83030135D86B21
:10BE800003685B6B9847F2E738BD000010B490F888
:10BE90003A4034B1C06B0468E468A4465DF8044BD2
:10BEA00060475DF8044B704710B490F83A4034B1E5
:10BEB000C06B04682469A4465DF8044B60475DF8D4
:10BEC000044B704730B490F83A40BDF8085034B194
:10BED000C06B046802956469A44630BC6047204684
:10BEE00030BC704790F83A301BB1C06B03689B6957
:10BEF0001847184670470000F8B5967A0546537AF9
:10BF00000F46144643EA0623D67A43EA06437A2BC1
:10BF10000DD8742B0AD903F180730124753B23F0EB
:10BF20007F4304FA03F313F0350F12D1F8BDB92B98
:10BF3000FCD1002695F83A20F3B29A42F6D905EBE7
:10BF40008303224639460136D86B0368DB6B98477A
:10BF5000F0E7BDE8F8401DF00FBE000038B504461C
:10BF6000002594F83A20EBB29A4207D904EB8303F8
:10BF70000135D86B03681B6C9847F2E738BD0000A9
:10BF800070B504460E46002594F83A20EBB29A426A
:10BF900007D904EB830331460135D86BFFF78CFDDD
:10BFA000F2E770BD0EB430B596B0002105463D22D3
:10BFB00019AC06A8059154F8043B039334F0CEF96C
:10BFC000094A05A9039B106841220094406D04941E
:10BFD00010F088FC05A92846FFF7D2FF16B0BDE88F
:10BFE000304003B0704700BFF02A003070B52DED2F
:10BFF000028BF0EE408A04460E4600259FED0A8A29
:10C0000094F83A20EBB29A420BD904EB8303F0EE9A
:10C01000480AB0EE680A3146D86B0135FFF7CAFC12
:10C02000EEE7BDEC028B70BD5241C07FF0B500233E
:10C0300090F82C7017269AB2974209D906FB03F4A0
:10C04000856A01332A192C5D8C42F4D11046F0BD6B
:10C050000022FBE770B5002390F82C6017259AB2F8
:10C06000964208D905FB03F2846A0133A25C8A4236
:10C07000F5D1012070BD406A0028FBD003798B42C6
:10C08000F7D00068F8E7000038B50546FE24E1B2B5
:10C090002846FFF7DFFF08B920B238BD013CA4B243
:10C0A000002CF4D14FF0FF30F7E7000038B50C4614
:10C0B000456A9DB32B79934232D02D68F9E711225E
:10C0C00034F0D6FCA9691122D4F8120029B134F059
:10C0D000CFFC6B790120637038BD34F03FF9D4F8A0
:10C0E0000600F5F799F8112802464FF03F0128BFE6
:10C0F0001122D4F8120034F031F907221D49D4F886
:10C100000A0034F0A1FC0028E3D1D4F80E307322E9
:10C110001A704622D4F812301A70DAE72846DBE7A4
:10C1200022700522A968D4F8020034F0A1FC112283
:10C13000E968D4F8060034F09BFC29694122D4F860
:10C140000A0034F095FC6969D4F80E000029B6D1D4
:10C15000112234F003F9D4F80600F5F75DF8112840
:10C1600002464FF03F0128BF1122D4F80E0034F0F0
:10C17000F5F8A7E77084080810B508460C46F5F7EF
:10C180004BF800220323D1B288422BD961564239A1
:10C190002F2929D8DFE801F01E18281C2828181C90
:10C1A00028281C1E20282824282828282828282831
:10C1B00022282828282828221E18241C1C28181C5D
:10C1C000282828281C2828240233DBB20132DAE789
:10C1D0000433FAE70133F8E71033F6E74033F4E7C6
:10C1E0000833F2E718B210BD4FF0FF30FBE7000054
:10C1F0002DE9F04F85B0054698460F469DF8403032
:10C2000000F14801914603A840F23942DDF83CA014
:10C210009DF84440019310F0E5FA6E6A96B1019BD7
:10C22000B06843B9B8420BD103A810F0FDFA30460C
:10C2300005B0BDE8F08F3946F4F7E4FF0028F3D0ED
:10C240003668EBE71C21012030F0E0FB8346002834
:10C25000EAD02846FFF718FF421C03D1584630F0B9
:10C26000D9FBE1E78BF80400002C42D0792030F0B4
:10C270008DFB04460028F1D03946671D0522F9F7E9
:10C280009FFC112251463846F9F79AFC04F116003A
:10C29000494641228146F9F793FCCBE90247CBF8A6
:10C2A0001090B8F1000F08D004F157071122414651
:10C2B0003846F9F785FCCBF814700E9B3BB1683417
:10C2C000112219462046F9F77BFCCBF8184051465D
:10C2D0002846FFF751FF431CC0D0019B6A6A8BF8C8
:10C2E000050003B96AB9CBF80020C5F824B05E4652
:10C2F0009AE70E9BCBE9027ACBE90498CBF8183089
:10C30000E5E711461268002AFBD1C1F800B0EEE75C
:10C310002DE9F04F89B0002506469DF85840149F3E
:10C320000594139C9DF854800194129CCDE902550C
:10C330000094FFF75DFF044648B9FFF779FA40F231
:10C34000DF32012109B0BDE8F04FFFF75DBA4FF0D1
:10C35000010B96F83A305FFA85FA534522D9A37952
:10C360000AF10E0923FA0AF313F0010F0DD106EBBF
:10C3700089022179506800F0EBF988B1A2790BFAB3
:10C380000AFA42EA0A0A84F806A0059B06EB89002D
:10C3900021793A46009343464068079700F022FB14
:10C3A0000135D6E709B0BDE8F08F000030B589B09F
:10C3B00000250EAC079402940D9C01940C9CCDE9D1
:10C3C00003550094FFF7A4FF09B030BD30B589B024
:10C3D0004FF0010C00250EAC079402940D9C0194C3
:10C3E0000C9CCDE9035C0094FFF792FF09B030BDCF
:10C3F00030B5A3B0FAF732F900231D491A46FAF70F
:10C400004BF8421C044631D0FAF728F9002340F2D9
:10C4100001621849FAF740F8431C054607D1FAF7BC
:10C420001DF92146FAF762F8002023B030BDFAF773
:10C4300015F9802302AA2146FAF766F8031E019334
:10C4400007DDFAF70BF9019B02AA2946FAF76CF807
:10C45000EDE7FAF703F92946FAF748F8FAF7FEF894
:10C460002146FAF743F80448F7F786FA0120DCE79B
:10C47000788408088C8408089F8408082DE9F74F01
:10C480000646002714F0A4FEDFF898B00446804664
:10C49000814614F09DFE031B0546B3F57A7F21D239
:10C4A00004F57A71091AFA2938BFFA21DBF800304D
:10C4B00089B24FF0000A186D019303689B68984792
:10C4C00014F086FE044696F83A105FFA8AF3994211
:10C4D0000AD906EB83030AF1010AD86B03681B6DC6
:10C4E0009847F0E7FA21E1E7A5EB09030B4A9342ED
:10C4F00006D9019BA946586D0368D3F88C3098473C
:10C50000002FC6D1A5EB0803054A9342C1D9304696
:10C51000A846FFF76DFF0746BBE700BFA0860100F6
:10C52000404B4C00F02A003008B5FFF7A7FF000091
:10C5300070B588B0044600F18C0140F28D5205A818
:10C5400010F050F994F86330CBB90F4B012508AACD
:10C5500006941B68186D03681E6D0C4B0793082327
:10C56000CDE9013540F22C630093094B12E9060036
:10C57000B04710B9074814F005FE84F8635005A8C9
:10C5800010F052F908B070BDF02A003029C5040837
:10C59000B4840808BB840808F8B504460D460E307C
:10C5A0000121164605F05CFC154B1B685F6D3B686E
:10C5B00038465B68984738B197F84D3023B1114839
:10C5C000F7F7DAF901236374A562002584F82C607B
:10C5D00094F83A20EBB29A4207D904EB8303013571
:10C5E000D86B03685B6A9847F2E72046FFF7A0FF25
:10C5F00094F8623043F0010384F86230F8BD00BF64
:10C60000F02A0030DC84080830B5002385B00446E9
:10C610000D460393CDE90133A3238DF80430952310
:10C620008DF80530B4238DF8063014F0E5FD0C22AA
:10C63000CDF80700CDF80B10204601A98DF80F505A
:10C64000FFF7E6FB05B030BD7FB504460E46154644
:10C6500000210D22684633F081FEA3238DF80030BF
:10C6600095238DF80130B7238DF8023014F0C4FD06
:10C670000D22CDF80300CDF80710204669468DF84D
:10C680000B608DF80C50FFF7C3FB04B070BD0000C9
:10C6900070B590F862300446C3F340059B0702D59D
:10C6A0000125284670BD90F91130012BF8D0154AAC
:10C6B000022B16681ED014F097FD94F8623043F6F2
:10C6C000982213F0040F104B08BF1346726D92F8B6
:10C6D0009C1029B9D2F8A02012B1821A9A42DFD355
:10C6E000D4F8A420002ADCD0801A834294BF00250D
:10C6F0000125D6E7706C03689B6B98470028DAD158
:10C70000CEE700BFF02A0030F049020010B5436CBC
:10C7100004461B68194201D1002010BD90F860301A
:10C7200053B12046FFF708FB0028F5D194F83A00F2
:10C73000003818BF0120F0E7FFF7AAFF0028F0D16A
:10C74000EAE70000014B1868704700BF444800301A
:10C7500070B5A6B00C460546792207AE00213046DA
:10C7600033F0FCFD1722002101A833F0F7FD0DF195
:10C770002103224601A9CDF80A300DF13203686881
:10C78000CDF80E300DF17303CDF80660CDF8123000
:10C7900021ABCDF81630FFF789FC044640B9FFF70E
:10C7A00047F8C7220221FFF72FF8204626B070BDB8
:10C7B00001A92846FFF7E2F804460028F5D001A9B0
:10C7C0002846FFF7E9F80446EFE7000070B5436834
:10C7D00004460E4693F86230DB0702D40025284653
:10C7E00070BD457E002DF9D0806803689B6898472E
:10C7F00098B16068FFF7A0FAC0B9606836B194F8E4
:10C800003C301BB190F91030002BE8D090F860302C
:10C810000BB3012384F83C30E1E7144B1B68186D1F
:10C8200003681B6C98470028E3D1D7E763689B6EC9
:10C83000002BE2D014F0D8FC63689A6E801A42F2A2
:10C840000F72904204D893F86030002BD5D1C5E721
:10C8500000229A66D1E7FFF71BFF0028BED063686D
:10C8600093F86030002BBAD0D3E700BFF02A003035
:10C8700038B5036805460C461B780BB1002038BD5F
:10C8800014F0B4FC9FED0B6A05EB44010B89C31A4D
:10C890009BB207EE903A6B68D3ED006AF8EEE77A48
:10C8A00086EE267AF4EEC77AF1EE10FAE6D4088125
:10C8B0000120E4E700007A4408B503888B4208D8D9
:10C8C000FEF7B6FF3A224FF40031BDE80840FEF70C
:10C8D0009BBF4B0901F01F0100EB8300012303FA0A
:10C8E00001F143680B43436008BD0000F8B543689D
:10C8F00004460E46D3ED007AF5EEC07AF1EE10FA5A
:10C9000002D803681B78EBB1331DB7B234F813308B
:10C91000D3B9CAB97A0906F01F03012504EB8202D4
:10C9200005FA03F3D2F80C24134218D131462068DB
:10C93000FFF77CFB08B1837D33B9394604F581608C
:10C94000FFF7BAFF01250AE031462046FFF790FFC6
:10C95000054630B1394604F22C40FFF7ADFF2846BA
:10C96000F8BD7F09012306F01F0604EB870403FAD4
:10C9700006F6D4F8303423EA0603C4F83034EEE780
:10C980002DE9F0410E461946044617461D469DF80E
:10C990001880FFF71BFF10B3236820465B6E984793
:10C9A00018B1236820461B6B9847236820461B6EEE
:10C9B0009847A0B155B123683A4631462046D3F88E
